:100000000C9436080C9455080C9455080C9455081B
:100010000C9455080C9455080C94A60A0C94DC0A10
:100020000C9455080C9455080C9455080C945508DC
:100030000C9455080C9455080C9455080C94360EE5
:100040000C9455080C9455080C9455080C945508BC
:100050000C94C1560C94CD4D0C9455080C94550835
:100060000C9455080C94A34E0C9455080C94974E80
:100070000C9455080C9455080C9455080C9455088C
:100080000C9484620C9455080C9455080C945508F3
:100090000C94E14E0C9455080C94D54E0C945508D4
:1000A0000C9455080C9455080C9455080C9455085C
:1000B0000C9455080C9455080C9455080C9455084C
:1000C0000C9455080C9455080C9455080C9455083C
:1000D0000C9455080C9455080C9455080C9455082C
:1000E0000C9455080C947A560C9484560C947056C3
:1000F0000C942A560C94B5560C94A6560C949A5609
:100100000C948E560C9455080C9455080C94550874
:100110000C9455080C9455080C9455080C945508EB
:1001200007634236B79BD8A71A39685618AEBAABE0
:10013000558C1D3CB7CC5763BD6DEDFD753EF61774
:100140007231BF000000803F08000000BE922449C9
:10015000123EABAAAA2ABECDCCCC4C3E00000080F9
:10016000BEABAAAAAA3E00000000BF000000803F6C
:100170000000000000084178D3BB4387D1133D192C
:100180000E3CC3BD4282AD2B3E68EC8276BED98F59
:10019000E1A93E4C80EFFFBE01C4FF7F3F0000009D
:1001A0000000503A20256C642050612020252D3716
:1001B0002E3266206D0A0025630025630049324314
:1001C0003A2000256300256C642050612020252DF5
:1001D000372E3266206D00256C6420432000256395
:1001E00000545F52483D252D342E31662000524880
:1001F0003D252D342E3166200025630025630050F7
:100200007772313D25730A0044656275673D307829
:10021000252D780A00496E7075742050313D257384
:100220000A0048554D5F5057525F414C5741595352
:100230003D25730A0025730A006175746F0A004C2E
:100240006F67206D6F64653D00496E74722E205398
:1002500065633A20202050303D252D372E3366200F
:1002600050313D252D372E33660A00496E74722EAB
:1002700020546F74616C3A2050303D252D6C642001
:1002800050313D252D6C640A005553425F50575242
:100290003D25730A00565F4D43553D252D352E32C1
:1002A000660A00565F494E3D252D352E32660A00FE
:1002B0005265706F7274204D61736B3D3078252DDF
:1002C0007820005265706F727420496E7465727682
:1002D000616C3D252D640A0052494D4520616464DE
:1002E000723D252D642E252D640A004E65696768D0
:1002F000626F72207461626C652073697A653D2556
:10030000640A00545820506F7765723D25640A00D6
:100310004932433A200049443D007478743D2573C6
:100320000A0053797374656D2053756D6D61727930
:100330000A0025630025630043757272656E7420A0
:100340007265706F727420696E74657276616C3D4F
:10035000252D64207365630A004E657720726570F1
:100360006F727420696E74657276616C3D252D64C0
:10037000207365630A002563005573696E672072F8
:1003800065706F72743D3078252D6C7820004E6555
:1003900077207265706F72743D3078255820002583
:1003A0006300256300256300256300204F5343430A
:1003B000414C3D2564200020467573653A206565F3
:1003C0003D253032782068663D25303278206C66D5
:1003D0003D25303278206C623D25303278004D4327
:1003E000553D2530366C7800256300252D31306C65
:1003F0007520252D31306C7520252D31306C752000
:10040000252D31306C75200A007478206C656E20C3
:10041000202020207268206D6973732020202072B4
:1004200068207374616C652020207268206D697388
:10043000630A002563004F4B0A0025630025630013
:10044000256300445F434F4D504153533D30782561
:10045000780A00445F414343454C3D307825780A93
:1004600000445F505245533D307825780A00445F80
:100470005057525F313D307825780A00445F41453E
:10048000533D307825780A00445F50315F4C454435
:100490003D307825780A00445F50305F4C45443D3C
:1004A000307825780A00445F4556454E543D3078F3
:1004B00025780A00445F504F5745523D30782578E3
:1004C0000A00445F4C45443D307825780A00445F7B
:1004D0004F573D307825780A00445F504B543D6EAD
:1004E000307825780A00445F54583D307825780AE2
:1004F00000445F52583D307825780A00445F4F50E1
:1005000045523D307825780A0043757272656E74E5
:100510002064656275673D307825580A004E65771E
:100520002064656275673D307825580A0025730A96
:100530000025372E33662025372E33660025352ECD
:10054000326620004572726F72203020566F6C74D4
:10055000004E6F7420737570706F727465640A005A
:100560004572726F72203020566F6C740045727243
:100570006F72203020566F6C740025730A00545837
:1005800020506F7765723D25640A005465737420AE
:10059000342025730A005465737420332025730AB0
:1005A000005465737420322025730A0054657374F7
:1005B00020312025730A0025730A0025730A0025BF
:1005C000730A0025730A005854414C5F5452494D38
:1005D0003D25640025730A0050413D090930782506
:1005E0006C7800503D09093078256C780041323D27
:1005F0000909307825780041313D0909307825789E
:1006000000565F494E3D0909307825780052483D33
:1006100009093078257800555054494D453D090960
:10062000307825780050315F543D090930782578BD
:100630000050313D0909307825780050305F543D35
:100640000909307825780050303D0909307825783F
:1006500000565F4D43553D09093078257800545FB9
:100660004D43553D0909307825780054313D09093D
:100670003078257800543D090930782578004944C0
:100680003D090930782578005458543D09093078DF
:100690002578005041200050200041322000413197
:1006A0002000565F494E20005248200055505449C2
:1006B0004D45200050315F54200050312000503013
:1006C0005F54200050302000565F4D4355200054A9
:1006D0005F4D4355200054312000542000494420F0
:1006E000005458542000253032780025372E3366C8
:1006F0002025372E33660025352E32662000204E09
:10070000657665722D7573656420737461636B2003
:100710003E2025642062797465730A0055707469FF
:100720006D6520256420646179732C202530326446
:100730003A253032643A253032640A0074657374A5
:10074000205B6F66667C317C327C335D202020200C
:1007500020202020202020202D2074657374206DFF
:100760006F6465730A0D00776474205B6F6E7C6F35
:1007700066667C746573745D202020202020202014
:100780002020202D207761746368646F670A0D0054
:10079000757067722020202020202020202020201B
:1007A0002020202020202020202020202D207265A5
:1007B000626F6F742076696120626F6F746C6F6115
:1007C0006465720A0D00626F6F7420202020202063
:1007D0002020202020202020202020202020202019
:1007E00020202D207265626F6F740A0D0070777281
:1007F00073205B646565707C666F7263655F6964B6
:100800006C655D2020202020202D206D63752073D5
:100810006C656570206D6F64650A0D007265737498
:1008200020656570726F6D20202020202020202000
:1008300020202020202020202D20726573746F72CC
:100840006520656570726F6D0A0D007031205B6FF9
:100850006E7C6F66665D20202020202020202020D6
:10086000202020202020202D2064697361626C6587
:100870002070756C736520703120746F2073617601
:100880006520706F7765720A0D0070777231205B9A
:100890006F6E7C6F66665D20202020202020202047
:1008A0002020202020202D2070696E31207077724A
:1008B0000A0D0074787077205B31352D305D202073
:1008C0002020202020202020202020202020202D1B
:1008D000205458205077722E2048696768657374D9
:1008E000203020283364426D290A0D00747874206A
:1008F0005B737472696E675D2020202020202020A9
:1009000020202020202020202D2053657420726577
:10091000706F7274207465787420737472696E6776
:100920000A0D00737320202020202020202020206A
:100930002020202020202020202020202020202DAA
:100940002073797374656D2073756D6D6172790AAA
:100950000D00727320202020202020202020202025
:1009600020202020202020202020202020202D207A
:10097000726164696F2073746174730A0D00726927
:10098000205B696E745D2020202020202020202004
:10099000202020202020202020202D207265706F14
:1009A000727420696E74657276616C0A0D007265EE
:1009B000205B6D61736B5D20202020202020202093
:1009C000202020202020202020202D206D6F7465E5
:1009D000207265706F72742073657474696E670A33
:1009E0000D006F7720202020202020202020202094
:1009F00020202020202020202020202020202D20EA
:100A00006F6E652D776972652073656E736F727393
:100A10000A0D006C6F67205B6175746F7C6F6E7C74
:100A20006F66665D20202020202020202020202DA1
:100A3000206D6F7465732064617461206F6E205542
:100A400053420A0D006E65205B666C7573685D200D
:100A50002020202020202020202020202020202096
:100A6000202D206E65696768626F72207461626C08
:100A7000650A0D0065727220202020202020202091
:100A80002020202020202020202020202020202066
:100A90002D206572726F7220696E666F0A0D006D8F
:100AA00063752020202020202020202020202020AE
:100AB00020202020202020202020202D206D637544
:100AC00020696E666F0A0D006964205B726573654C
:100AD000745D202020202020202020202020202085
:100AE000202020202D2069642068616E646C696E6E
:100AF000670A0D0068756D70205B6F6E7C6F6666AF
:100B00005D202020202020202020202020202020A8
:100B10002D2068756D6964697479207065726D2027
:100B200073656E736F72207077720A0D0068756D51
:100B300020202020202020202020202020202020B5
:100B40002020202020202020202D2068756D696421
:100B50006974792073656E736F720A0D0064652085
:100B60005B6D61736B5D20202020202020202020E1
:100B70002020202020202020202D20646562756701
:100B80000A0D0063616C69205B5B765F696E7C6156
:100B9000317C61325D20766F6C747C726573657434
:100BA0007C6E6F6E655D202D2063616C6962726181
:100BB00074650A0D0061646320202020202020201D
:100BC0002020202020202020202020202020202025
:100BD000202D2073686F7720765F696E2C2061313D
:100BE0002C20613220766F6C74616765730A0D008A
:100BF000616573205B6F6E7C6F66665D20202020D0
:100C00002020202020202020202020202D20696E40
:100C1000746567726574790A0D00752020202020A4
:100C200020202020202020202020202020202020C4
:100C30002020202020202D20757074696D650A0DFC
:100C4000007620202020202020202020202020206E
:100C5000202020202020202020202020202D207631
:100C6000657273696F6E0A0D0068202020202020B5
:100C70002020202020202020202020202020202074
:100C800020202020202D2068656C700A0D0025632F
:100C900000756E6B6E6F776E20636D640A004E4850
:100CA00044433032313620004C3347343230304404
:100CB0002000484D433538383320004144584C33E8
:100CC00034352000424D50303835200048494836F0
:100CD0003133302000415432344D4143200020252F
:100CE00073002025362E3266200025303278002011
:100CF0002573002025362E3266204F6E2D426F61FF
:100D000072640025303278000A00452025642E25C3
:100D10006420636C6F636B20256C75206370752095
:100D2000256C75206C706D20256C752069727120A2
:100D3000256C7520676C656420256C7520796C6561
:100D40006420256C7520726C656420256C75207498
:100D50007820256C75206C697374656E20256C7520
:100D60002073656E736F727320256C7520736572C6
:100D700069616C20256C750A00532025642E25645A
:100D800020636C6F636B20256C7520747820256C54
:100D90007520727820256C752072747820256C750A
:100DA0002072727820256C75207265786D697420C8
:100DB000256C752061636B747820256C75206E6FCF
:100DC00061636B747820256C752061636B72782089
:100DD000256C752074696D65646F757420256C755C
:100DE0002062616461636B727820256C7520746F7A
:100DF0006F6C6F6E6720256C7520746F6F73686FF2
:100E0000727420256C752062616473796E6368204A
:100E1000256C752062616463726320256C752063A4
:100E20006F6E74656E74696F6E64726F7020256C7E
:100E3000752073656E64696E6764726F7020256CCF
:100E400075206C6C747820256C75206C6C72782021
:100E5000256C750A00257325730A004F6E6C696E48
:100E6000650A000A002C20636865636B2072617458
:100E70006520257520487A0025732025732C206372
:100E800068616E6E656C20257520706F77657220C5
:100E90002575000A0025783A004D414320616464BD
:100EA00072657373200052616E646F6D2045554901
:100EB000363420616464726573732067656E657291
:100EC000617465640A000A2A2A2A2A2A2A2A426F99
:100ED0006F74696E672025732A2A2A2A2A2A2A0A09
:100EE00000020000FFFE00000141544D4547413122
:100EF000323872666131006C6F63616C686F737455
:100F000000454550524F4D20697320636F727275D2
:100F100070742C20726577726974696E67207769C6
:100F200074682064656661756C74732E0A006E6166
:100F30006E00696E660000407A10F35A00A0724E8F
:100F400018090010A5D4E80000E87648170000E46E
:100F50000B54020000CA9A3B000000E1F5050000B6
:100F600080969800000040420F000000A08601001B
:100F70000000102700000000E803000000006400EB
:100F8000000000000A000000000001000000000056
:100F90002C76D888DC674F0823DFC1DFAE59E1B17A
:100FA000B796E5E3E453C63AE651997696E8E6C289
:100FB0008426EB898C9B62ED407C6FFCEFBC9C9F90
:100FC00040F2BAA56FA5F490055A2AF75C936B6CB2
:100FD000F9676DC11BFCE0E40D47FEF520E6B500A6
:100FE000D0ED902E0300943577050080841E080014
:100FF00000204E0A000000C80C333333330F986EC4
:1010000012831141EF8D2114893BE65516CFFEE680
:10101000DB18D1844B381BF77C1D901DA4BBE42446
:10102000203284725E228100C9F124ECA1E53D27C3
:10103000494E46494E4954594E414ECDCCCC3D0ABD
:10104000D7233C17B7D13877CC2B329595E6241FA0
:10105000B14F0A000020410000C84200401C462059
:10106000BCBE4CCA1B0E5AAEC59D740011241FBED7
:10107000CFEFD1E4DEBFCDBF16E0A0E0B2E0E2E901
:10108000FBEF00E00BBF02C007900D92A23DB1073D
:10109000D9F71DE2A2EDB6E001C01D92A638B10756
:1010A000E1F70E94874C0C94C77D0C94000029E066
:1010B000FC0120935700C895802D0895E091AB174F
:1010C000F0E0EF71F070E050F84E80838091AB1744
:1010D0008F5F8093AB178091C02488608093C02479
:1010E00042EE54E0CA0161E10E94CF3D80E090E011
:1010F00008954F925F926F927F928F929F92AF92DC
:10110000BF92CF92DF92EF92FF920F931F93DF93E4
:10111000CF93CDB7DEB760970FB6F894DEBF0FBEA2
:10112000CDBF3B018091D2069091D30681FD74988A
:101130000E9497446C01DC018C91982F92959F70CE
:10114000913009F05CC190E08F709070009709F4C5
:1011500056C185EC94E2B3010E949C3B009709F0D4
:101160004EC187EF96E00E94C63E1CC0C8010296A1
:10117000B3010E949C3B009791F0C8010D9660E07E
:1011800074E649E25AE098010E948B41F601918190
:10119000D80118968C911897981761F530C1C8013D
:1011A0000E948C3F082F192F01151105F9F62FC148
:1011B000C8010296B3010E94933BF60181818150E0
:1011C000D80118968C9380E091E0A0E0B0E0F8019F
:1011D00081879287A387B48787EF96E0B8010E9442
:1011E0004D3FC8010D9660E074E649E25AE098016F
:1011F0000E948B4184E00E94CB45D80115969C93B8
:101200008E93149783E00E94CB452C01F8019783BD
:101210008683D60111968C908085881A9924AA24F9
:10122000BB2486E0880C991CAA1CBB1C8A95D1F7AC
:10123000618572858385948520EC30E040E050E044
:101240000E94D976672F782F892F9927860E971EAF
:10125000A81EB91EF80181869286A386B486D6019F
:1012600011968C91119780878091D2069091D30628
:1012700081FD08C08091BC0480FD04C081FFBFC017
:101280001D9BBDC0EDB7FEB774970FB6F894FEBFB7
:101290000FBEEDBFEDB6FEB60894E11CF11C80E078
:1012A00092E092838183C6010296D70113969C93A4
:1012B0008E931297F301808114968C931497159650
:1012C0001C921597818116968C93169717961C92EF
:1012D000D60111968C911197F701808711868C9118
:1012E00090E08F70907093878287D80114968D91CB
:1012F0009C9115979587848757864686BB27AB2D8B
:101300009A2D892D918B808BC501B40124E630E0A4
:1013100040E050E00E94D976672F782F892F9927D7
:101320000E941F77F701738B628B0E949F7A209136
:101330009F048DB79EB744960FB6F8949EBF0FBE1C
:101340008DBF2223A9F000D000D0EDB7FEB73196B3
:101350008AEB91E0ADB7BEB712969C938E9311972E
:10136000228313820E94B17A0F900F900F900F90FA
:101370008091491C86FF43C00E947D4AC6010596A4
:101380000E943C4AEDB7FEB73C970FB6F894FEBFFB
:101390000FBEEDBF31967E010894E11CF11CADB784
:1013A000BEB71296FC92EE92119780E190E0938383
:1013B000828384E492E095838483D80114968D918E
:1013C0009C9115979783868316968D919C9117977C
:1013D00091878087D60111968C91828713860E940F
:1013E0000F7BEDB7FEB73C960FB6F894FEBF0FBE6D
:1013F000EDBF82E00E94594AC7010E943C4A809199
:10140000D2069091D30681FF0DC0749A0BC08BE475
:1014100095E00E945A3E082F192F0115110509F079
:10142000C7CEEDCF60960FB6F894DEBF0FBECDBF2E
:10143000CF91DF911F910F91FF90EF90DF90CF90B0
:10144000BF90AF909F908F907F906F905F904F90E4
:101450000895EF92FF92CF93DF93E82EE7017E018C
:10146000F92EE7018091D2069091D30687FF2FC015
:101470008DB79EB70C970FB6F8949EBF0FBE8DBF69
:10148000EDB7FEB7319687E592E0ADB7BEB71296DD
:101490009C938E9311978A81828313828B8184839C
:1014A00015828885868317828C819D8191878087AC
:1014B0008E819F81938782870E949F7A2DB73EB746
:1014C000245F3F4F0FB6F8943EBF0FBE2DBF87EF8E
:1014D00096E0BE010E94143F8BE495E0BE010E949D
:1014E000803EDF91CF91FF90EF90089587EE93E0DB
:1014F0008115910511F00197F1F70895882369F09E
:101500006D987598ED9A80916A00886080936A0062
:10151000809168008160809368008091BC04909104
:10152000BD0491FF10C06E988EB18F6B8EB9EE9A8C
:1015300080916A00806280936A0080916800816077
:10154000809368000895769AEE9808951F920F92FE
:101550000FB60F9211248F939F93AF93BF938091F7
:10156000680080FF20C08091A0249091A124A091C8
:10157000A224B091A3240196A11DB11D8093A024A3
:101580009093A124A093A224B093A3248091D20687
:101590009091D30690FF07C0749882E090E09093FA
:1015A000920480939104BF91AF919F918F910F907E
:1015B0000FBE0F901F9018951F920F920FB60F92AB
:1015C00011248F939F93AF93BF938091680080FF06
:1015D00020C08091A4249091A524A091A624B0912C
:1015E000A7240196A11DB11D8093A4249093A52446
:1015F000A093A624B093A7248091D2069091D306FD
:1016000091FF07C0739882E090E0909392048093DA
:101610009104BF91AF919F918F910F900FBE0F904A
:101620001F90189580937C0080917B00877F80932A
:101630007B0080917C00806C80937C0085E08093AF
:101640007A0080917A00806880937A0080917B0094
:1016500087FFFCCF80917B0085FFFCCF80917A00D3
:10166000806480937A0080917A0086FDFCCF10928E
:1016700079001092780084E090E060E070E02091C2
:101680007A00206420937A0020917A0026FDFCCF16
:101690002091780030917900620F731F019779F7DC
:1016A00010927C0080917A008F7780937A007695F3
:1016B00067957695679580E090E00E945F74089545
:1016C00080E00E94120B2091930430919404409189
:1016D0009504509196040E94117521EE3AE744E971
:1016E0005EE30E948F73089580E18093510180939F
:1016F00051019091510195FF03C08F5F8F31B9F770
:101700006BE4869FB0011124882777FD8095982F80
:101710000E94617420E030E64FE954E40E948F7328
:1017200020E030E04AE754E40E94F7730895809186
:10173000B60484FF4BC080917B00886080937B005F
:1017400089EC80937C0085E080937A0080917A0018
:10175000806880937A0080917B0087FFFCCF809126
:101760007B0085FFFCCF80917A00806480937A00B3
:1017700080917A0086FDFCCF80917A00806480930E
:101780007A0080917A0086FDFCCF6091780070919C
:10179000790080E090E00E945F7427ED33EA40E931
:1017A0005FE30E94117526E636E648E853E40E949E
:1017B0008E736093A0177093A1178093A2179093D4
:1017C000A31780917A008F7780937A0008956F92A3
:1017D0007F928F929F92AF92BF92CF92DF92EF92C1
:1017E000FF920F931F93DF93CF93CDB7DEB72A9766
:1017F0000FB6F894DEBF0FBECDBF3C011092DA06E3
:101800008FEF89835CEBC52E57E1D52E00E010E009
:1018100042E0E42EF12CEC0EFD1E4E010894811CDA
:10182000911C3AE0A32EB12CAC0EBD1E3FC0083077
:10183000110509F441C0C401B7012A870E948947F4
:1018400089812A858F3F11F08E3F19F48093DA0643
:1018500034C06114710479F4C7010E94A3478093D6
:10186000BD24F701A5EBB4E281918D93EA15FB0548
:10187000D9F721E022C0C7010E94A347F601808367
:10188000D701F80123E0EE0FFF1F2A95E1F7E00FE3
:10189000F11FEC54F84E8D918193AA15BB05D9F731
:1018A0000F5F1F4F89E090E0C80ED91E202F89815D
:1018B000882309F0BCCF01C028E0822F2A960FB6FA
:1018C000F894DEBF0FBECDBFCF91DF911F910F9176
:1018D000FF90EF90DF90CF90BF90AF909F908F9050
:1018E0007F906F90089500D088E09DE0EDB7FEB73F
:1018F000928381830E94B17A0F900F9008952F9266
:101900003F924F925F926F927F928F929F92AF928F
:10191000BF92CF92DF92EF92FF920F931F93DF93CC
:10192000CF9300D000D0CDB7DEB78C01009741F443
:1019300089E290E06BE270E04AE250E027E00AC002
:101940008130910549F489E290E06BE270E04AE26F
:1019500050E026E00E946546C8010E94E70BF801AE
:10196000E852F94F808301151105A1F01CEBC12E3F
:1019700017E1D12E00E010E04F01BAEE6B2EBCE073
:101980007B2EA2EE4A2EACE05A2EFEED2F2EFCE06E
:101990003F2EFAC085EB94E20E94D5489C01B90124
:1019A000882777FD8095982F0E946174C82EE92EB4
:1019B000E5EBAE2EE4E2BE2E03E01DE0D5018D91F5
:1019C0005D0100D000D0EDB7FEB73196ADB7BEB720
:1019D00012961C930E931197828313826B837C83E0
:1019E0000E94B17A0F900F900F900F906B817C81C5
:1019F000BDEBAB16B4E2BB0609F700D000D000D0B7
:101A00000DB71EB70F5F1F4F23EF3CE0EDB7FEB7DA
:101A1000328321838C2D9E2D20E030E048EC52E46F
:101A20000E94F773D80112966D937D938D939C93CA
:101A300015970E94B17AEDB7FEB736960FB6F894B7
:101A4000FEBF0FBEEDBF8091BD24882319F086E84C
:101A500092E002C08FE892E000D000D02FEE3CE090
:101A6000ADB7BEB712963C932E93119714969C93E4
:101A70008E9313970E94B17A0F900F900F900F9052
:101A80000E94730C88C0780163E0EE0CFF1C6A951D
:101A9000E1F7E00EF11EE4EBF7E1EE0EFF1EC701E9
:101AA0000E94D5489C01B901882777FD8095982F21
:101AB0000E9461745C0120E030E0D7018D917D01CE
:101AC00000D000D0EDB7FEB73196ADB7BEB71296D5
:101AD0007C926E9211978283138229833A836B835F
:101AE0007C830E94B17A29813A812F5F3F4F0F900A
:101AF0000F900F900F906B817C8128303105E9F6B3
:101B000000D000D000D0EDB6FEB60894E11CF11C68
:101B1000EDB7FEB7528241828A2D9B2D20E030E046
:101B200048EC52E40E94F773D70112966D937D93AF
:101B30008D939C9315970E94B17AEDB7FEB73696B8
:101B40000FB6F894FEBF0FBEEDBFD6018C9188236F
:101B500019F086E892E002C08FE892E000D000D051
:101B6000EDB7FEB732822182948383830E94B17ADB
:101B70000F900F900F900F900E94730C0F5F1F4FEC
:101B800029E030E0C20ED31ED4018C9190E00817FA
:101B900019070CF478CF0F900F900F900F90CF9102
:101BA000DF911F910F91FF90EF90DF90CF90BF904A
:101BB000AF909F908F907F906F905F904F903F90ED
:101BC0002F900895DF93CF9300D0CDB7DEB78091EB
:101BD000B62489838091BC248A83CE0101960E9419
:101BE000AE3B0F900F90CF91DF910895CF93DF938D
:101BF000EC018091B5248F3FB1F58091B6248F3FE1
:101C000091F58091B7248F3F71F58091B8248F3F73
:101C100051F58091B9248F3F31F58091BA248F3FDF
:101C200011F58091BB248F3FF1F48091BC248F3F4C
:101C3000D1F489E290E06BE270E04AE250E027E004
:101C40000E94654680E090E00E94E70BC852D94FA1
:101C5000888385EB94E267E170E049E050E00E9400
:101C6000017C0E94E20DDF91CF9108951F920F92A7
:101C70000FB60F920BB60F9211242F933F934F93F1
:101C80005F936F937F938F939F93AF93BF93EF93E4
:101C9000FF938091C02482608093C0248091BC0413
:101CA00086FD2B9A8091BC0487FD2B9A809191042C
:101CB000909192041816190614F4749A739A8091EC
:101CC000D2069091D30685FF02C0749873988091D4
:101CD00053059091540501979093540580935305B3
:101CE000009709F068C08091060790910707019658
:101CF000909307078093060720914B2030914C204A
:101D000040914D2050914E202F5F3F4F4F4F5F4FDE
:101D100020934B2030934C2040934D2050934E20E5
:101D200020E130E030935405209353052091BC040A
:101D300020FD02C01D9B05C01092D6061092D5064C
:101D400006C021E030E03093D6062093D50660919E
:101D5000BA047091BB046115710599F001960E9457
:101D6000F876009771F477988091D2069091D30617
:101D700093FF07C0749884E090E09093920480935E
:101D800091046091BA047091BB046115710579F0FA
:101D900080910607909107070E94F876009739F422
:101DA0008EEF94E062E140E050E00E94CF3D8091F0
:101DB000BC0486FD2B988DE695E060E040E050E0A5
:101DC0000E94CF3DFF91EF91BF91AF919F918F9175
:101DD0007F916F915F914F913F912F910F900BBE2B
:101DE0000F900FBE0F901F9018958091AB17909198
:101DF0005F20891B08950E94F50E882379F0E091F9
:101E00005F20F0E0EF71F070E050F84E208130E09C
:101E100080915F208F5F80935F2002C02FEF3FEFA4
:101E2000C9010895CF93DF93EC011092FA06109246
:101E3000F90688819981009731F022E0843C92076D
:101E400009F0B9C009C00E94F50E882341F484EC62
:101E500092E099838883B3C0613109F0B0C0F894EF
:101E600078940E94FB0E90E09093FE068093FD060E
:101E70008D3009F47CC08F3F31F38231910569F1D7
:101E80008F37910521F08830910509F053C080917A
:101E9000010790910207181619060CF060C06091B6
:101EA000802D7091812D88E090E00E94737A60917E
:101EB000802D7091812D80E290E00E94737A609174
:101EC000802D7091812D88E090E00E94737A80913E
:101ED00001079091020701973EC06091802D70919B
:101EE000812D8DE090E00E94737A1092000710928D
:101EF000FF0614C0805A9F4DFC0180816091802DA7
:101F00007091812D90E00E94737A8091FF069091EC
:101F100000070196909300078093FF068091FF06CB
:101F200090910007209101073091020782179307D3
:101F30000CF315C06091802D7091812D0E94737AF1
:101F400080910107909102072091FD06FC01E05A63
:101F5000FF4D2083019690930207809301078091A3
:101F60000107909102078F33910509F06CCF109211
:101F70005F2080915F208093AB1780910107909143
:101F80000207FC01E05AFF4D10829093FA068093FD
:101F9000F90610920207109201078091BE249091D9
:101FA000BF24009709F44FCF6091FB0640E050E05A
:101FB0000E94CF3D48CF1982188283E001C081E0A2
:101FC000DF91CF91089578948091D5069091D606AF
:101FD000009731F08091BC049091BD0490FF03C044
:101FE00083B7817F03C083B7817F866083BFF89406
:101FF00083B7816083BF7894889583B78E7F83BFD2
:1020000078940895CF93DF93EC01888199810097AC
:1020100021F02AE08E33920799F40E94DE4F0E944D
:10202000E30F80918C0E90918D0E65E840E050E0BA
:102030000E94CF3D8EE39AE09983888381E003C0BC
:102040001982188283E0DF91CF910895CF93DF93B7
:102050000E94DE4F80EB0E9455498823B1F40E9414
:10206000BB498091491C90914A1C816090934A1C05
:102070008093491C00D085ED9CE0EDB7FEB79283BC
:1020800081830E94B17A0F900F908EB1C82FD0E05B
:10209000C470D070729A0E94DE4F8EE40E9455493F
:1020A0008823B1F40E94BB498091491C90914A1C3D
:1020B000826090934A1C8093491C00D08CEC9CE079
:1020C000EDB7FEB7928381830E94B17A0F900F9093
:1020D000209709F472980E94DE4F8EEE0E945549B7
:1020E0008823B1F40E94BB498091491C90914A1CFD
:1020F000846090934A1C8093491C00D084EC9CE03F
:10210000EDB7FEB7928381830E94B17A0F900F9052
:1021100086EA0E9455498823B1F40E94BB49809108
:10212000491C90914A1C886090934A1C8093491CDA
:1021300000D08BEB9CE0EDB7FEB7928381830E94C9
:10214000B17A0F900F900E94DE4F8CE30E945549A8
:102150008823B1F40E94BB498091491C90914A1C8C
:10216000806190934A1C8093491C00D082EB9CE0D4
:10217000EDB7FEB7928381830E94B17A0F900F90E2
:102180000E94DE4F82ED0E9455498823B1F40E94DF
:10219000BB498091491C90914A1C806290934A1CD3
:1021A0008093491C00D088EA9CE0EDB7FEB792838B
:1021B00081830E94B17A0F900F90C7E0D0E00E9417
:1021C000DE4F8CE70E9455498823B9F40E94BB4931
:1021D0008091491C90914A1C806490934A1C809382
:1021E000491C00D08EE99CE0EDB7FEB79283818355
:1021F0000E94B17A0F900F9002C0219701F70E94C0
:10220000BB490E94730CDF91CF910895DF93CF9368
:1022100000D0CDB7DEB74A8369830E9491496981B6
:10222000862F0E94C3494A81842F0E94C3490E947D
:10223000BB490F900F90CF91DF910895AF92BF925D
:10224000DF92EF92FF920F931F93DF93CF9300D013
:102250000F92CDB7DEB7082FD22E4A835B836983F6
:102260000E9491496981862F0E94C349802F816015
:102270000E94B8494A815B81042F152FAA24BB24F0
:10228000ED2CFF240894E108F1080FC0AE14BF0440
:1022900019F40E94DE4902C00E94D449F8018083EB
:1022A0000894A11CB11C0F5F1F4FAD1478F30E945E
:1022B000BB490F900F900F90CF91DF911F910F911D
:1022C000FF90EF90DF90BF90AF9008958F929F9214
:1022D000AF92BF92CF92DF92EF92FF920F931F9334
:1022E000DF93CF93CDB7DEB760970FB6F894DEBF1C
:1022F0000FBECDBF8E010F5F1F4F80E1D8011D9231
:102300008A95E9F780EB68E9A80128E00E941E1190
:1023100000D080E992E0EDB7FEB7928381830E94FE
:102320009F7A680198E0892E912C8C0E9D1E0F904B
:102330000F90780187E9A82E82E0B82ED7018D9101
:102340007D0100D000D0EDB7FEB73196ADB7BEB776
:102350001296BC92AE921197828313820E949F7A4A
:102360000F900F900F900F90E814F90439F700D0F8
:1023700000D0EDB7FEB731968DE992E0ADB7BEB7AC
:1023800012969C938E9311978885828313820E9464
:102390009F7AAE014F5F5F4F80E1FA0111928A95FB
:1023A000E9F70F900F900F900F9080EB60E828E016
:1023B0000E941E1100D083EA92E0ADB7BEB712961C
:1023C0009C938E9311970E949F7A015F1F4F0F90ED
:1023D0000F908A2CEB2CF60181916F0100D000D078
:1023E000EDB7FEB73196ADB7BEB711968C92119787
:1023F0001296EC92828313820E949F7A0F900F9024
:102400000F900F90C016D10631F700D000D0EDB775
:10241000FEB731968DE992E0ADB7BEB712969C93A8
:102420008E9311978885828313820E949F7A0F90E2
:102430000F900F900F9060960FB6F894DEBF0FBE0E
:10244000CDBFCF91DF911F910F91FF90EF90DF9063
:10245000CF90BF90AF909F908F9008950F931F9350
:10246000DF93CF9300D0CDB7DEB71A8219828EEEFC
:102470006AEA8E010F5F1F4FA80122E00E941E1121
:10248000398120E08A8190E0822B932B9093211850
:10249000809320188EEE6CEAA80122E00E941E11A3
:1024A000398120E08A8190E0822B932B909323182E
:1024B000809322188EEE6EEAA80122E00E941E117F
:1024C000398120E08A8190E0822B932B909325180C
:1024D000809324188EEE60EBA80122E00E941E116A
:1024E000398120E08A8190E0822B932B90933318DE
:1024F000809332188EEE62EBA80122E00E941E113A
:10250000398120E08A8190E0822B932B90933518BB
:10251000809334188EEE64EBA80122E00E941E1115
:10252000398120E08A8190E0822B932B9093371899
:10253000809336188EEE66EBA80122E00E941E11F1
:10254000398120E08A8190E0822B932B9093271889
:10255000809326188EEE68EBA80122E00E941E11DF
:10256000398120E08A8190E0822B932B9093291867
:10257000809328188EEE6AEBA80122E00E941E11BB
:10258000398120E08A8190E0822B932B90932D1843
:1025900080932C188EEE6CEBA80122E00E941E1195
:1025A000398120E08A8190E0822B932B90932F1821
:1025B00080932E188EEE6EEBA80122E00E941E1171
:1025C000398120E08A8190E0822B932B90933118FF
:1025D000809330180F900F90CF91DF911F910F9142
:1025E00008952F923F924F925F926F927F928F92B7
:1025F0009F92AF92BF92CF92DF92EF92FF920F9392
:102600001F93DF93CF93CDB7DEB76C970FB6F894D7
:10261000DEBF0FBECDBFA82E4A8B2B8FFE01319699
:1026200083E0DF011D928A95E9F7809144188823A1
:1026300039F46C8F0E942E1281E0809344186C8DC7
:10264000662309F475C08EEE64EF4EE20E94061117
:1026500069E07AE180E090E00E9442498EEE66EF08
:10266000AE014F5F5F4F22E00E941E11698170E052
:1026700080E090E0982F872F762F66272A8130E020
:1026800040E050E0622B732B842B952B2091361861
:102690003091371840E050E0621B730B840B950BB0
:1026A000209134183091351840E050E00E94D976DE
:1026B0007B018C013FE015950795F794E7943A95D7
:1026C000D1F760912E1870912F18882777FD80958B
:1026D000982F2BE0660F771F881F991F2A95D1F737
:1026E0002091301830913118442737FD4095542FF0
:1026F0002E0D3F1D401F511F0E9441772E0D3F1D83
:1027000030932B1820932A18285F3F4FB4E035955B
:102710002795BA95E1F779010027F7FC0095102F6E
:10272000E0923818F092391800933A1810933B1839
:10273000BA2DB295BB0FBB0FB07CBC5CB9872A2DFC
:1027400030E03E8B2D8B63E070E00A2C02C0660FF8
:10275000771F0A94E2F7882777FD8095982F25E365
:1027600035E040E050E00E94D976DC01CB010296D2
:10277000A11DB11D8A879B87AC87BD8720E533ECFF
:1027800040E050E004C05595479537952795AA94A9
:10279000D2F72E873F87488B598B18861C821D8263
:1027A0001E821F8248E050E08D899E89481B590B8C
:1027B0005C8B4B8B69C18EEE64EF49850E940611DC
:1027C0006A857B858C859D850E9442498EEE66EFE9
:1027D000AE014F5F5F4F23E00E941E1180912A18C7
:1027E00090912B18805A9F401C01442437FC409440
:1027F000542CC201B101A20191010E94D9766F8BC4
:10280000788F898F9A8F209124183091251844272A
:1028100037FD4095542FC201B1010E94D9767B014A
:102820008C01ADE015950795F794E794AA95D1F73B
:1028300022E030E040E050E0E20EF31E041F151FDE
:102840006F89788D898D9A8DFCE095958795779520
:102850006795FA95D1F720912618309127184427CB
:1028600037FD4095542F0E94D976BC01992777FDFA
:102870009095892FE60EF71E081F191F72E0159517
:102880000795F794E7947A95D1F780E090E8A0E077
:10289000B0E0E80EF91E0A1F1B1F2091321830917C
:1028A000331840E050E0C801B7010E94D9763B01DF
:1028B0004C016FE096948794779467946A95D1F76A
:1028C000A980BB24CC24DD246501BB24AA248A81F1
:1028D00090E0A0E0B0E0BA2FA92F982F8827A82A6F
:1028E000B92ACA2ADB2A8B8190E0A0E0B0E0A82AAE
:1028F000B92ACA2ADB2A0B8804C0D594C794B79496
:10290000A7940A94D2F720912218309123184427D3
:1029100037FD4095542FC201B1010E94D9767B0149
:102920008C013BE015950795F794E7943A95D1F71C
:102930008091201890912118AA2797FDA095BA2F71
:1029400022E0880F991FAA1FBB1F2A95D1F7E80E16
:10295000F91E0A1F1B1F209128183091291844279F
:1029600037FD4095542F6F89788D898D9A8D0E94FF
:10297000D976A7E19595879577956795AA95D1F72B
:10298000E60EF71E081F191F0D8804C0EE0CFF1C71
:10299000001F111F0A94D2F722E030E040E050E01F
:1029A000E20EF31E041F151FF2E015950795F7942C
:1029B000E794FA95D1F7AE18BF08C00AD10AC6014C
:1029C000B5012E853F85488959890E94D97697FDA2
:1029D0000BC0660F771F881F991FA40193010E94E7
:1029E0001F7779018A010AC0A40193010E941F7711
:1029F00079018A01EE0CFF1C001F111F552717FDDE
:102A00005A95412F302F2F2DCA01B9010E94D97636
:102A10002EED3BE040E050E00E94D9765B016C0176
:102A2000C801B70123E433EE4FEF5FEF0E94D97680
:102A3000BC01992777FD9095892F6153714F8F4F76
:102A40009F4F5601DD24B7FCD094CD2C6A0D7B1D21
:102A50008C1D9D1D24E095958795779567952A9502
:102A6000D1F76E0D7F1D801F911F2C813D814E81FE
:102A70005F81260F371F481F591F2C833D834E83CC
:102A80005F8338853F5F388748855A89451708F442
:102A900092CE552391F0252F30E040E050E06C813C
:102AA0007D818E819F810E941F7720933C183093F7
:102AB0003D1840933E1850933F188B8D8823C9F1E1
:102AC00060913C1870913D1880913E1890913F188C
:102AD000611571058105910561F10E94617420E81D
:102AE00036EE45EC57E40E94F77321E03EED42E4F8
:102AF0005EE30E947475562F472F382F292F60E010
:102B000070E080E89FE3DA01F9012B2F3A2F4F2F75
:102B10005E2F0E948E732BE43AE34DEB57E30E9445
:102B2000F773609340187093411880934218909304
:102B300043186C960FB6F894DEBF0FBECDBFCF9191
:102B4000DF911F910F91FF90EF90DF90CF90BF909A
:102B5000AF909F908F907F906F905F904F903F903D
:102B60002F900895DF93CF9300D000D000D0CDB741
:102B7000DEB7FE01319686E0DF011D928A95E9F706
:102B80008091AA17882399F486EA61E340E00E94C5
:102B9000061186EA6CE24AE00E94061181E0809309
:102BA000AA176CE77EE380E090E00E94424986EA43
:102BB0006DE248E00E9406116CE77EE380E090E061
:102BC0000E94424986EA62E3AE014F5F5F4F26E012
:102BD0000E941E1186EA6DE247E00E9406119A816A
:102BE00080E0498150E0482B592B5093A517409322
:102BF000A4179C8180E02B8130E0282B392B309367
:102C0000A7172093A6177E8160E08D8190E0862B28
:102C1000972B9093A9178093A8176DB77EB768502C
:102C200070400FB6F8947EBF0FBE6DBFEDB7FEB714
:102C3000319667EA72E0ADB7BEB712967C936E9399
:102C400011975383428335832483978386830E941D
:102C50009F7A6DB77EB7685F7F4F0FB6F8947EBFDF
:102C60000FBE6DBF26960FB6F894DEBF0FBECDBF68
:102C7000CF91DF9108950F931F93DF93CF9300D0EF
:102C800000D000D0CDB7DEB78E010F5F1F4F86E0BA
:102C9000D8011D928A95E9F78CE362E041E00E9439
:102CA00006118CE360E048E50E94061162E174E3DE
:102CB00080E090E00E9442498CE363E0A80126E0B6
:102CC0000E941E118CE362E043E00E94061199818C
:102CD00080E04A8150E0482B592B50938117409354
:102CE00080179B8180E02C8130E0282B392B30939A
:102CF0008317209382177D8160E08E8190E0862B80
:102D0000972B9093851780938417EDB7FEB738976C
:102D10000FB6F894FEBF0FBEEDBF319665EB72E0C3
:102D2000ADB7BEB712967C936E93119753834283CF
:102D300035832483978386830E949F7AEDB7FEB7FD
:102D400038960FB6F894FEBF0FBEEDBF26960FB6AD
:102D5000F894DEBF0FBECDBFCF91DF911F910F91D1
:102D60000895CF93DF93EC0188819981009731F02A
:102D70002AE08732920709F071C00BC08BED96E014
:102D800060E870E00E94854087E29AE0998388833A
:102D900069C08BED96E00E94B040009709F462C0D4
:102DA0008091D2069091D30694FF3FC08091491C38
:102DB00082FF3BC083E061E048E021E00E94F11225
:102DC0008DB79EB70A970FB6F8949EBF0FBE8DBF02
:102DD000EDB7FEB7319682EA91E0ADB7BEB7129675
:102DE0009C938E93119780913C1890913D18A091DF
:102DF0003E18B0913F1882839383A483B58380915A
:102E0000401890914118A0914218B09143188683C0
:102E10009783A087B1870E94B17A8DB79EB70A9633
:102E20000FB6F8949EBF0FBE8DBF8091D2069091D1
:102E3000D30695FF06C08091491C83FF02C00E9403
:102E4000B2158091D2069091D30696FF97CF8091CC
:102E5000491C84FF93CF0E943B1690CF19821882A1
:102E600083E001C081E0DF91CF910895CF92DF929E
:102E7000FF920F931F93CF93DF93729A8091BC04BC
:102E800083FD06C0C0E5D0E00E94760A2197E1F7F5
:102E90008EE40E9455498823B1F080914F20909193
:102EA0005020A0915120B09152200196A11DB11D3A
:102EB00080934F2090935020A0935120B0935220A4
:102EC00021E030E084C0C0E5D0E00E94760A21977E
:102ED000E1F78FE40E9455490E94D449F82E82956B
:102EE0008695869583708130A9F420915320309186
:102EF000542040915520509156202F5F3F4F4F4F07
:102F00005F4F20935320309354204093552050938B
:102F1000562016C08230A0F02091572030915820C2
:102F20004091592050915A202F5F3F4F4F4F5F4F94
:102F300020935720309358204093592050935A2083
:102F40000E94D4491F2D1F7300E0080F111D0E941D
:102F5000D4490E94DE4920E0E901C80FD11DD69571
:102F6000C795D695C7950E94BB498091BC0483FF45
:102F70007298B80180E090E00E945F7420E134E034
:102F800048EC5BE30E9411756093451870934618F6
:102F90008093471890934818BE0180E090E00E940B
:102FA0005F7424EA3CEF44E25CE30E94117520E088
:102FB00030E040E252E40E948E736093C12470932B
:102FC000C2248093C3249093C42420E030E0C9013C
:102FD000DF91CF911F910F91FF90DF90CF900895D7
:102FE0007298729A8EE40E94554980EA0E94C34901
:102FF00080E00E94C34980E00E94C3498FE40E94A0
:1030000055490E94D4498295869586958370813072
:10301000A9F4209153203091542040915520509193
:1030200056202F5F3F4F4F4F5F4F209353203093D9
:103030005420409355205093562016C08230A0F063
:1030400020915720309158204091592050915A207A
:103050002F5F3F4F4F4F5F4F2093572030935820A3
:103060004093592050935A2000D000D0EDB7FEB7BE
:10307000319623EC32E0ADB7BEB712963C932E9357
:103080001197828313820E949F7A0F900F900F9066
:103090000F908EE40E94554980E80E94C34980E069
:1030A0000E94C34980E00E94C3490E94BB4980E05E
:1030B00090E0089500D081E99CE0ADB7BEB71296CC
:1030C0009C938E9311970E94B17A20919F040F9048
:1030D0000F902223A9F000D000D0EDB7FEB73196B3
:1030E0008EE89CE0ADB7BEB712969C938E93119775
:1030F000228313820E94B17A0F900F900F900F904D
:10310000089500D089E69CE0EDB7FEB792838183F5
:103110000E94B17A81E49CE0EDB7FEB7928381838F
:103120000E94B17A8AE19CE0EDB7FEB79283818379
:103130000E94B17A80EF9BE0EDB7FEB79283818366
:103140000E94B17A85EB9BE0EDB7FEB79283818355
:103150000E94B17A83E89BE0EDB7FEB7928381834A
:103160000E94B17A8DE59BE0EDB7FEB79283818333
:103170000E94B17A8DE29BE0EDB7FEB79283818326
:103180000E94B17A84EF9AE0EDB7FEB79283818313
:103190000E94B17A88EC9AE0EDB7FEB79283818302
:1031A0000E94B17A8FE99AE0EDB7FEB792838183EE
:1031B0000E94B17A84E79AE0EDB7FEB792838183EB
:1031C0000E94B17A85E49AE0EDB7FEB792838183DD
:1031D0000E94B17A83E19AE0EDB7FEB792838183D2
:1031E0000E94B17A82EE99E0EDB7FEB792838183B7
:1031F0000E94B17A8EEA99E0EDB7FEB7928381839F
:103200000E94B17A8EE799E0EDB7FEB79283818391
:103210000E94B17A82E599E0EDB7FEB7928381838F
:103220000E94B17A83E299E0EDB7FEB79283818381
:103230000E94B17A8CEE98E0EDB7FEB7928381835D
:103240000E94B17A83EB98E0EDB7FEB79283818359
:103250000E94B17A8AE898E0EDB7FEB79283818345
:103260000E94B17A8BE498E0EDB7FEB79283818338
:103270000E94B17A8CE198E0EDB7FEB7928381832A
:103280000E94B17A8DEE97E0EDB7FEB7928381830D
:103290000E94B17A86EC97E0EDB7FEB79283818306
:1032A0000E94B17A80E997E0EDB7FEB792838183FF
:1032B0000E94B17A87E697E0EDB7FEB792838183EB
:1032C0000E94B17A8CE397E0EDB7FEB792838183D9
:1032D0000E94B17A0F900F90089583ED92E00E94C2
:1032E000D87A08952F923F924F925F926F927F9279
:1032F0008F929F92AF92BF92CF92DF92EF92FF9206
:103300000F931F93CF93DF9360914B2070914C20CC
:1033100080914D2090914E20A0904B20B0904C2059
:10332000C0904D20D0904E2060904B2070904C204B
:1033300080904D2090904E2020904B2030904C203B
:1033400040904D2050904E202DB73EB72A5030402F
:103350000FB6F8943EBF0FBE2DBFCDB7DEB7219696
:103360002CE137E0EDB7FEB732832183A0E8EA2EE7
:10337000A1E5FA2EA1E00A2F112DA80197010E94C4
:103380001F773B832A83C601B501A80197010E94DC
:103390001F77F0E1EF2EFEE0FF2E012D112DA80189
:1033A00097010E941F77332727FD30953D832C839B
:1033B000C401B301A80197010E941F77ECE3EE2E30
:1033C000F12C012D112DA80197010E941F773327A1
:1033D00027FD30953F832E83C201B101A8019701DB
:1033E0000E941F77772767FD7095798768870E940D
:1033F000B17A2DB73EB7265F3F4F0FB6F8943EBF68
:103400000FBE2DBFDF91CF911F910F91FF90EF90D5
:10341000DF90CF90BF90AF909F908F907F906F90F4
:103420005F904F903F902F900895E6E8FDE28081F5
:10343000918122E482349207B9F000D000D08EEF5F
:1034400096E0ADB7BEB712969C938E931197E6584F
:10345000FD421496FC93EE9313970E94B17A0F905D
:103460000F900F900F9008953A96B1E4E53FFB0757
:10347000F0F20895EF92FF920F931F93CF93DF9393
:103480000E94600B00D000D000D027EF36E0ADB72F
:10349000BEB712963C932E931197EDB7FEB7638398
:1034A0007483858396830E94B17A8DB79EB7069602
:1034B0000FB6F8949EBF0FBE8DBF81E00E94120B25
:1034C00020919704309198044091990450919A0466
:1034D0000E9411757B018C0182E00E94120B9B01FE
:1034E000AC01ADB7BEB71A970FB6F894BEBF0FBE0A
:1034F000ADBFCDB7DEB72196EBEEF6E01296FC93AA
:10350000EE9311978E2D9F2DA02FB12F8A839B8331
:10351000AC83BD83CA01B90120919B0430919C0406
:1035200040919D0450919E040E9411756E837F838B
:10353000888799870E94B17AEDB7FEB73A960FB6A1
:10354000F894FEBF0FBEEDBF0E94730CDF91CF91C8
:103550001F910F91FF90EF9008950F931F93CF93BA
:10356000DF93882389F085EB94E26FEF70E049E008
:1035700050E00E941A7A85EB94E267E170E049E03E
:1035800050E00E94017C1CC0C5EBD4E206EE16E0C0
:10359000899100D000D0EDB7FEB73196ADB7BEB778
:1035A00012961C930E931197828313820E94B17A14
:1035B0000F900F900F900F90B4E2CD3BDB0741F7D7
:1035C0000E94730CDF91CF911F910F910895EF929C
:1035D000FF920F931F936091A4047091A50480E063
:1035E00090E00E940C7A67EF72E00E94217A0097C7
:1035F00009F098C086E294E1A0E0B0E08093B604C0
:103600009093B704A093B804B093B90486EB94E008
:103610006EE070E042E050E00E94017C8CE390E0BC
:103620009093BB048093BA048AEB94E062E170E06B
:1036300042E050E00E94017C8AE090E09093BD045B
:103640008093BC048CEB94E064E170E042E050E0D5
:103650000E94017C1092D3061092D20682ED96E071
:1036600060E070E042E050E00E94017C0F2EF2E248
:10367000EF2EFFEFFF2EFCEC0F2FFBE31F2FF02DA3
:10368000E0929704F09298040093990410939A049E
:1036900087E994E066E070E044E050E00E94017C3D
:1036A000E0929B04F0929C0400939D0410939E046E
:1036B0008BE994E06AE070E044E050E00E94017C15
:1036C0008DEE97E4AAE8BCE380939304909394046E
:1036D000A0939504B093960483E994E062E070E0CF
:1036E00044E050E00E94017C1092D70687ED96E0FE
:1036F00066E170E041E050E00E94017C86E997E1DC
:103700002AE0FC0111922A95E9F760E270E04AE0B4
:1037100050E00E94017C81E00E94AD1A80E090E0C0
:103720000E94F60D1F910F91FF90EF90089588234E
:1037300009F436C18091B60480FF0BC000D081EE41
:1037400096E0EDB7FEB7928381830E94B17A0F9025
:103750000F908091B60481FF0BC000D08DED96E0F4
:10376000EDB7FEB7928381830E94B17A0F900F90DC
:103770008091B60482FF0BC000D08AED96E0EDB7D1
:10378000FEB7928381830E94B17A0F900F9080914F
:10379000B60483FF0BC000D086ED96E0EDB7FEB710
:1037A000928381830E94B17A0F900F908091B6042A
:1037B00084FF0BC000D08FEC96E0EDB7FEB792838C
:1037C00081830E94B17A0F900F908091B60485FF9B
:1037D0000BC000D088EC96E0EDB7FEB792838183F2
:1037E0000E94B17A0F900F908091B60486FF0BC0B3
:1037F00000D084EC96E0EDB7FEB7928381830E94FF
:10380000B17A0F900F908091B60487FF0BC000D063
:103810008EEB96E0EDB7FEB7928381830E94B17A7A
:103820000F900F908091B6049091B704A091B804C6
:10383000B091B90490FF0BC000D08AEB96E0EDB7D1
:10384000FEB7928381830E94B17A0F900F9080918E
:10385000B6049091B704A091B804B091B90491FF57
:103860000BC000D084EB96E0EDB7FEB79283818366
:103870000E94B17A0F900F908091B6049091B70496
:10388000A091B804B091B90492FF0BC000D08CEAAB
:1038900096E0EDB7FEB7928381830E94B17A0F90D4
:1038A0000F908091B6049091B704A091B804B091A4
:1038B000B90493FF0BC000D088EA96E0EDB7FEB7DD
:1038C000928381830E94B17A0F900F908091B60409
:1038D0009091B704A091B804B091B90494FF0BC0C3
:1038E00000D082EA96E0EDB7FEB7928381830E9412
:1038F000B17A0F900F908091B6049091B704A09187
:10390000B804B091B90495FF0BC000D08EE996E0E1
:10391000EDB7FEB7928381830E94B17A0F900F902A
:103920008091B6049091B704A091B804B091B90405
:1039300096FF0BC000D08AE996E0EDB7FEB7928300
:1039400081830E94B17A0F900F908091B60490917C
:10395000B704A091B804B091B90497FF0BC000D090
:1039600087E996E0EDB7FEB7928381830E94B17A32
:103970000F900F908091B6049091B704A091B80475
:10398000B091B904A0FFF7C100D083E996E0EDB78C
:10399000FEB7928381830E94B17A0F900F90EBC1A2
:1039A00000D000D000D088E896E0EDB7FEB7928353
:1039B000818381E090E0A0E0B0E083839483A583DD
:1039C000B6830E94B17A8DB79EB706960FB6F8946B
:1039D0009EBF0FBE8DBF0E94730C00D000D000D0E0
:1039E0008EE796E0EDB7FEB79283818382E090E0A8
:1039F000A0E0B0E083839483A583B6830E94B17A6C
:103A00008DB79EB706960FB6F8949EBF0FBE8DBFBA
:103A10000E94730C00D000D000D085E796E0EDB78F
:103A2000FEB79283818384E090E0A0E0B0E08383DE
:103A30009483A583B6830E94B17A8DB79EB706960C
:103A40000FB6F8949EBF0FBE8DBF0E94730C00D0BE
:103A500000D000D08BE696E0EDB7FEB7928381836D
:103A600088E090E0A0E0B0E083839483A583B683F0
:103A70000E94B17A8DB79EB706960FB6F8949EBF96
:103A80000FBE8DBF0E94730C00D000D000D08EE519
:103A900096E0EDB7FEB79283818380E190E0A0E0ED
:103AA000B0E083839483A583B6830E94B17A8DB7F7
:103AB0009EB706960FB6F8949EBF0FBE8DBF0E94AC
:103AC000730C00D000D000D081E596E0EDB7FEB7D2
:103AD0009283818380E290E0A0E0B0E083839483CE
:103AE000A583B6830E94B17A8DB79EB706960FB6AE
:103AF000F8949EBF0FBE8DBF0E94730C00D000D003
:103B000000D087E496E0EDB7FEB79283818380E42E
:103B100090E0A0E0B0E083839483A583B6830E9405
:103B2000B17A8DB79EB706960FB6F8949EBF0FBEBA
:103B30008DBF0E94730C00D000D000D08BE396E0C4
:103B4000EDB7FEB79283818380E890E0A0E0B0E01B
:103B500083839483A583B6830E94B17A8DB79EB781
:103B600006960FB6F8949EBF0FBE8DBF0E94730CD1
:103B700000D000D000D081E396E0EDB7FEB792838D
:103B8000818380E091E0A0E0B0E083839483A5830B
:103B9000B6830E94B17A8DB79EB706960FB6F89499
:103BA0009EBF0FBE8DBF0E94730C00D000D000D00E
:103BB00085E296E0EDB7FEB79283818380E092E0E4
:103BC000A0E0B0E083839483A583B6830E94B17A9A
:103BD0008DB79EB706960FB6F8949EBF0FBE8DBFE9
:103BE0000E94730C00D000D000D087E196E0EDB7C2
:103BF000FEB79283818380E094E0A0E0B0E083830D
:103C00009483A583B6830E94B17A8DB79EB706963A
:103C10000FB6F8949EBF0FBE8DBF0E94730C00D0EC
:103C200000D000D08DE096E0EDB7FEB7928381839F
:103C300080E098E0A0E0B0E083839483A583B6831E
:103C40000E94B17A8DB79EB706960FB6F8949EBFC4
:103C50000FBE8DBF0E94730C00D000D000D081E059
:103C600096E0EDB7FEB79283818380E090E1A0E01B
:103C7000B0E083839483A583B6830E94B17A8DB725
:103C80009EB706960FB6F8949EBF0FBE8DBF0E94DA
:103C9000730C00D000D000D087EF95E0EDB7FEB7F1
:103CA0009283818380E090E2A0E0B0E083839483FC
:103CB000A583B6830E94B17A8DB79EB706960FB6DC
:103CC000F8949EBF0FBE8DBF0E94730C00D000D031
:103CD00000D08DEE95E0EDB7FEB79283818380E052
:103CE00090E4A0E0B0E083839483A583B6830E9430
:103CF000B17A8DB79EB706960FB6F8949EBF0FBEE9
:103D00008DBF0E94730C00D000D000D083EE95E0F0
:103D1000EDB7FEB79283818380E090E8A0E0B0E049
:103D200083839483A583B6830E94B17A8DB79EB7AF
:103D300006960FB6F8949EBF0FBE8DBF0E94730CFF
:103D400000D000D000D088ED95E0EDB7FEB79283AB
:103D5000818380E090E0A1E0B0E083839483A58339
:103D6000B6830E94B17A8DB79EB706960FB6F894C7
:103D70009EBF0FBE8DBF0E94730C08952F923F927D
:103D80004F925F926F927F928F929F92AF92BF926B
:103D9000CF92DF92EF92FF920F931F93DF93CF9317
:103DA00000D0CDB7DEB79A838983DC018D919C91D9
:103DB0001197009711F00C94B8316091A4047091A0
:103DC000A50480E690E20E940C7A80E690E260E42E
:103DD00070E00E94397A009759F46091802D7091BB
:103DE000812D8AE090E00E94737A81E00C94BE31CC
:103DF0008130910549F420906020332444245524D7
:103E0000662477244301BFC18230910599F4309133
:103E1000602020916120932F80E0820F911D1C0172
:103E2000892F880F880B482E582E682E782E882EC2
:103E3000982EA9C18330910509F09CC02091602083
:103E4000A09061208090622030E040E050E060E08F
:103E500070E080E090E000E10E942B6FF22E132FC3
:103E6000E42ED52EC62EB72E282E992E2A2D30E0E0
:103E700040E050E060E070E080E090E008E00E9408
:103E80002B6F2F0DB1E02F1508F0B0E0310FE1E0FE
:103E9000311708F0E0E0B30FF1E0B31708F0F0E0FD
:103EA000EF2B4E0D31E04E1508F030E0E40FF1E05D
:103EB000E41708F0F0E03F2B5D0D41E05D1508F0E0
:103EC00040E0A32FA50F31E0A51708F030E0432B09
:103ED0006C0D31E06C1508F030E0F42FF60F41E086
:103EE000F61708F040E0342B7B0D41E07B1508F01D
:103EF00040E0532F570F31E0571708F030E0432BC5
:103F0000820D31E0821508F030E0480F61E048177B
:103F100008F060E0362B990D930F022F080D11E089
:103F2000021708F010E01B0F81E01B1708F080E07B
:103F3000B82FBE0F71E0BE1708F070E07A0F61E095
:103F40007A1708F060E06F0F31E06F1708F030E08B
:103F5000350F21E0351708F020E0240F81E0241709
:103F600008F080E018014B2E572E662E732E822EFD
:103F7000982EFEC08430910509F0FCC0209160208D
:103F8000A0906120709062208090632030E040E03B
:103F900050E060E070E080E090E008E10E942B6F6C
:103FA000F22E132FE42ED52EC62EB72E282E992EA4
:103FB0002A2D30E040E050E060E070E080E090E0EA
:103FC00000E10E942B6F2F0DF1E02F1508F0F0E0BB
:103FD000310FE1E0311708F0E0E0F30FA1E0F31753
:103FE00008F0A0E0EA2B4E0D31E04E1508F030E06D
:103FF000E40FA1E0E41708F0A0E03A2B5D0D41E0EA
:104000005D1508F040E0B32FB50F31E0B51708F0AB
:1040100030E0432B6C0D31E06C1508F030E0A42F3C
:10402000A60F41E0A61708F040E0342B7B0D41E0DD
:104030007B1508F040E0532F570F31E0571708F079
:1040400030E0432B820D31E0821508F030E0480F5C
:1040500061E0481708F060E0362B990E930E122F9E
:10406000180D81E0121708F080E0282E2F0E81E055
:104070002F1608F080E0F82EFE0E81E0FE1608F004
:1040800080E0E82EEB0E81E0EB1608F080E0D82E01
:10409000DA0E81E0DA1608F080E0C82EC50E81E065
:1040A000C51608F080E0B82EB40E81E0B41608F012
:1040B00080E0980E272D30E040E050E060E070E0B6
:1040C00080E090E008E00E942B6F210FE1E02117D3
:1040D00008F0E0E0320DF1E0321508F0F0E0E30F17
:1040E000A1E0E31708F0A0E0FA2B4F0D31E04F15E7
:1040F00008F030E0F40FA1E0F41708F0A0E03A2B4C
:104100005E0D41E05E1508F040E0A32FA50F31E001
:10411000A51708F030E0432B6D0D31E06D1508F068
:1041200030E0542F560F41E0561708F040E0342B92
:104130007C0D41E07C1508F040E0632F670F31E013
:10414000671708F030E0432B8B0D31E08B1508F03A
:1041500030E0480F71E0481708F070E0372B990DF8
:10416000222E3E2E4F2E5A2E652E762E842E932EE4
:10417000990E09C01AE0212E3324442455246624C4
:104180007724882499240E94730CB22DB33689F4C5
:10419000E32DE23371F4F42DF93659F4552049F446
:1041A000662039F4772029F4882019F4992009F43D
:1041B0004EC59101A201B301C401B3E6AB2EA2E347
:1041C000BA2EF9E6CF2EDD24EE24FF2400E010E025
:1041D0000E949C6F823008F073C2822D853689F46C
:1041E000932D923771F4442061F4552051F46620E8
:1041F00041F4772031F4882021F4992011F40C94B3
:104200003F2D9101A201B301C401E5E6AE2E02E704
:10421000B02ECC24DD24EE24FF2400E010E00E9428
:104220009C6F823008F008C1A22DA53681F4B32D11
:10423000B43669F4442059F4552049F4662039F421
:10424000772029F4882019F4992009F4CDC691012A
:10425000A201B301C40115E6A12EB4E6BB2ECC2405
:10426000DD24EE24FF2400E010E00E949C6F8230E9
:1042700008F062C0E22DE53779F4332069F4442078
:1042800059F4552049F4662039F4772029F4882020
:1042900019F4992009F4EAC79101A201B301C401FC
:1042A000A5E7AA2EBB24CC24DD24EE24FF2400E0C5
:1042B00010E00E949C6F823010F5F22DF83611F05C
:1042C0000C94B631332011F00C94B631442011F027
:1042D0000C94B631552011F00C94B631662011F0D3
:1042E0000C94B631772011F00C94B631882011F07F
:1042F0000C94B631992011F00C94B63192C7822DEE
:10430000863779F4332069F4442059F4552049F470
:10431000662039F4772029F4882019F4992009F4CB
:10432000BEC7922D943611F00C94B631A32DA13650
:1043300011F00C94B6317BC0B22DB73789F4E32D60
:10434000EF3671F4442061F4552051F4662041F4B5
:10435000772031F4882021F4992011F40C94D52B86
:104360009101A201B301C401F7E7AF2EEFE6BE2E23
:10437000CC24DD24EE24FF2400E010E00E949C6F9A
:104380008230B8F5F22DF43681F4832D893669F444
:10439000442059F4552049F4662039F4772029F453
:1043A000882019F4992009F440C7922D953611F010
:1043B0000C94B631A32DAE3611F00C94B6314420D6
:1043C00011F00C94B631552011F00C94B6316620E2
:1043D00011F00C94B631772011F00C94B63188208E
:1043E00011F00C94B631992011F00C94B6310C9464
:1043F000292CB22DB13389F4E32DE03771F4442038
:1044000061F4552051F4662041F4772031F488207E
:1044100021F4992011F40C94BA2CF22DF33311F0FD
:104420000C94B631832D813711F00C94B6314420B1
:1044300011F00C94B63195C0922D983789F4A32DC4
:10444000A43671F4B42DB13659F4552049F46620E0
:1044500039F4772029F4882019F4992009F4F3C35A
:104460009101A201B301C40108E7A02E14E6B12E08
:10447000B1E6CB2EDD24EE24FF2400E010E00E9404
:104480009C6F823008F083C0E22DE33789F4F32D6E
:10449000F23771F4442061F4552051F4662041F460
:1044A000772031F4882021F4992011F40C940B2EFC
:1044B0009101A201B301C401A3E7AA2EF2E7BF2E26
:1044C000CC24DD24EE24FF2400E010E00E949C6F49
:1044D000823020F5822D893611F00C94B631932D5F
:1044E000923711F00C94B631442011F00C94B6318F
:1044F000552011F00C94B631662011F00C94B631B1
:10450000772011F00C94B631882011F00C94B6315C
:10451000992011F00C94B6310C94B82DA22DA3372C
:1045200089F4B32DB33771F4442061F4552051F46C
:10453000662041F4772031F4882021F4992011F489
:104540000C941A2EE22DE33611F00C94B631F32DB3
:10455000F43611F00C94B631842D813611F00C94A0
:10456000B631552011F00C94B631662011F00C9440
:10457000B631772011F00C94B631882011F00C94EC
:10458000B631992011F00C94B6310C942E30922D46
:10459000923791F4A32DA23779F4B42DB53661F496
:1045A000552051F4662041F4772031F4882021F41D
:1045B000992011F40C94F82A9101A201B301C401CD
:1045C000E2E7AE2E02E7B02E15E6C12EDD24EE2482
:1045D000FF2400E010E00E949C6F8230C0F5E22DC5
:1045E000E33789F4F32DF53671F4842D813659F4CF
:1045F000552049F4662039F4772029F4882019F4ED
:10460000992009F45CC6922D923611F00C94B631C3
:10461000A32DA53611F00C94B631B42DB43611F09B
:104620000C94B631552011F00C94B631662011F07F
:104630000C94B631772011F00C94B631882011F02B
:104640000C94B631992011F00C94B631CDC4E22D02
:10465000E33689F4F32DFD3671F4842D883659F450
:10466000552049F4662039F4772029F4882019F47C
:10467000992009F4F0C2922D9D3611F00C94B631B8
:10468000A32DA53711F00C94B631B42DB83611F026
:104690000C94B631552011F00C94B631662011F00F
:1046A0000C94B631772011F00C94B631882011F0BB
:1046B0000C94B631992011F00C94B6310C943D3025
:1046C000E22DE03791F4F32DFC3679F4842D853614
:1046D00061F4952D983649F4662039F4772029F451
:1046E000882019F4992009F49CC59101A201B30115
:1046F000C401B0E7AB2EACE6BA2EF5E6CF2EE8E665
:10470000DE2EEE24FF2400E010E00E949C6F823039
:1047100008F047C1A22DA13389F4B32DB13371F450
:10472000E42DE13759F4552049F4662039F4772017
:1047300029F4882019F4992009F4BDC79101A20138
:10474000B301C40101E3A02E11E3B12EB1E7CB2EDA
:10475000DD24EE24FF2400E010E00E949C6F8230F4
:1047600008F083C0F22DF73689F4832D8F3671F46B
:10477000942D9C3659F4552049F4662039F477205D
:1047800029F4882019F4992009F4DFC69101A201C7
:10479000B301C401A7E6AA2EFFE6BF2EECE6CE2E9B
:1047A000DD24EE24FF2400E010E00E949C6F8230A4
:1047B00020F5A22DA43611F00C94B631B32DB336EA
:1047C00011F00C94B631E42DEC3611F00C94B631A6
:1047D000552011F00C94B631662011F00C94B631CE
:1047E000772011F00C94B631882011F00C94B6317A
:1047F000992011F00C94B631A5C6F22DF53789F445
:10480000832D833671F4942D9D3659F4552049F447
:10481000662039F4772029F4882019F4992009F4C6
:104820004AC7A22DA03311F00C94B631B32DB13389
:1048300011F00C94B631E42DE13711F00C94B6313F
:10484000552011F00C94B631662011F00C94B6315D
:10485000772011F00C94B631882011F00C94B63109
:10486000992011F00C94B631C3C6F22DF43791F4AF
:10487000832D843679F4942D973761F4552051F4C3
:10488000662041F4772031F4882021F4992011F436
:104890000C9449319101A201B301C40104E7A02E97
:1048A00014E6B12EB7E7CB2EDD24EE24FF2400E082
:1048B00010E00E949C6F8230D0F5A22DA03791F4B9
:1048C000B32DB53679F4E42DE23761F4552051F477
:1048D000662041F4772031F4882021F4992011F4E6
:1048E0000C943F2DF22DF43711F00C94B631832D3A
:1048F000883711F00C94B631942D943711F00C9444
:10490000B631552011F00C94B631662011F00C949C
:10491000B631772011F00C94B631882011F00C9448
:10492000B631992011F00C94B6310C941E31A22DA1
:10493000A43791F4B32DBF3679F4E42DEF3661F44A
:10494000F52DF23649F4662039F4772029F48820D1
:1049500019F4992009F40CC5822D893611F00C94B4
:10496000B631932D9C3611F00C94B631A42DA1369E
:1049700011F00C94B631B52DB33611F00C94B6315C
:10498000662011F00C94B631772011F00C94B631FA
:10499000882011F00C94B631992011F00C94B631A6
:1049A00086C1E22DE33799F4F32DF23781F4842D9B
:1049B000873769F4952D903751F4662041F47720BC
:1049C00031F4882021F4992011F40C94072D9101E1
:1049D000A201B301C401A3E7AA2EF2E7BF2EE7E7C5
:1049E000CE2E00E7D02EEE24FF2400E010E00E943F
:1049F0009C6F823008F089C0A22DA03791F4B32DAE
:104A0000BD3679F4E42DE53761F4F52DF83649F437
:104A1000662039F4772029F4882019F4992009F4C4
:104A2000EAC69101A201B301C40110E7A12EBDE6BF
:104A3000BB2EA5E7CA2EF8E6DF2EEE24FF2400E009
:104A400010E00E949C6F823028F5822D813611F093
:104A50000C94B631932D9D3611F00C94B631A42DE3
:104A6000A53711F00C94B631B52DB83611F00C9471
:104A7000B631662011F00C94B631772011F00C9409
:104A8000B631882011F00C94B631992011F00C94B5
:104A9000B631A0C6E22DE33799F4F32DF53681F453
:104AA000842D823769F4952D903751F4662041F4B6
:104AB000772031F4882021F4992011F40C94873068
:104AC000A22DA13311F00C94B631B32DB23711F0F1
:104AD0000C94B631E42DE73711F00C94B631F52D76
:104AE000F03711F00C94B631662011F00C94B63109
:104AF000772011F00C94B631882011F00C94B63167
:104B0000992011F00C94B631AAC0822D873791F408
:104B1000932D903779F4A42DA83761F4B52DB437CF
:104B200049F4662039F4772029F4882019F4992073
:104B300009F4F5C39101A201B301C401E7E7AE2E68
:104B400000E7B02E18E7C12EB4E7DB2EEE24FF24D9
:104B500000E010E00E949C6F8230D0F5E22DE43737
:104B600091F4F32DF33779F4842D853661F4952D86
:104B7000923749F4662039F4772029F4882019F413
:104B8000992009F4F4C6A22DA43711F00C94B63183
:104B9000B32DB33711F00C94B631E42DE53611F096
:104BA0000C94B631F52DF43711F00C94B631662023
:104BB00011F00C94B631772011F00C94B6318820A6
:104BC00011F00C94B631992011F00C94B631D4C385
:104BD000822D823791F4932D973679F4A42DA03746
:104BE00061F4B52DB53749F4662039F4772029F4FE
:104BF000882019F4992009F476C4E22DEC3611F0DE
:104C00000C94B631F32DF13611F00C94B631842D9D
:104C1000843711F00C94B631952D983711F00C941F
:104C2000B631662011F00C94B631772011F00C9457
:104C3000B631882011F00C94B631992011F00C9403
:104C4000B6310C94E2300E94B2150C94B8310E9437
:104C500026100C94B8310E943B160C94B831609128
:104C6000A4047091A50480E090E00E940C7A8C016D
:104C70006EEF72E00E94217A009719F477980C94F5
:104C8000B831C80161E073E00E94217A009719F4FD
:104C9000779A0C94B831779903C08EEF92E002C0F6
:104CA00081E093E000D000D02DE235E011C46091A6
:104CB000A4047091A50480E090E00E940C7A8C011D
:104CC00068E173E00E94217A009709F052C0609178
:104CD000A4047091A50480E090E00E940C7A8C01FD
:104CE000009711F40C94B8316BE173E00E94217AC3
:104CF000009729F482E29FEFACECBBE30BC0C80144
:104D000061E273E00E94217A009769F482E29FEFEA
:104D1000ACECBAE38093970490939804A093990421
:104D2000B0939A041DC0C8010E94FF787B018C01DA
:104D300020E030E0A9010E94F3738823B1F081E004
:104D40000E94120B9B01AC01C801B7010E94F773CE
:104D500060939704709398048093990490939A04B5
:104D600087E994E066E070E0BEC000D08DE695E093
:104D70008CC0C80166E273E00E94217A009709F0B6
:104D800052C06091A4047091A50480E090E00E945C
:104D90000C7A8C01009711F40C94B8316BE173E03C
:104DA0000E94217A009729F482E29FEFACECBBE3EA
:104DB0000BC0C80161E273E00E94217A009769F498
:104DC00082E29FEFACECBAE380939B0490939C0447
:104DD000A0939D04B0939E041DC0C8010E94FF785B
:104DE0007B018C0120E030E0A9010E94F37388234D
:104DF000B1F082E00E94120B9B01AC01C801B70127
:104E00000E94F77360939B0470939C0480939D04AD
:104E100090939E048BE994E06AE070E064C000D057
:104E200080E695E067C0C80169E273E00E94217ADC
:104E3000009709F06BC06091A4047091A50480E014
:104E400090E00E940C7A8C01009711F40C94B83118
:104E50006BE173E00E94217A009769F48DEE97E48C
:104E6000AAE8BCE38093930490939404A0939504E0
:104E7000B093960434C0C80161E273E00E94217AC5
:104E8000009741F400D081E595E0EDB7FEB792833D
:104E9000818336C0C8010E94FF781B012C0120E0ED
:104EA00030E0A9010E94F373882309F180E00E9499
:104EB000120B7B018C01C201B10121EE3AE744E9FA
:104EC0005EE30E948E73A80197010E94F7736093BE
:104ED000930470939404809395049093960483E9CB
:104EE00094E062E070E044E050E00C948C3100D03B
:104EF00084E495E0ADB7BEB712969C938E9311975C
:104F00000E94B17A0F900F900C94B8310E94600B00
:104F100000D000D000D02DE335E0EDB7FEB73283EE
:104F20002183ADB7BEB713966D937D938D939C93FC
:104F300016970E94B17AEDB7FEB736960FB6F89481
:104F4000FEBF0FBEEDBF81E00E94120B20919704BF
:104F5000309198044091990450919A040E941175DF
:104F60007B018C0182E00E94120B9B01AC018DB78A
:104F70009EB70A970FB6F8949EBF0FBE8DBFCDB6F1
:104F8000DEB60894C11CD11C81E395E0ADB7BEB775
:104F900012969C938E9311978E2D9F2DA02FB12F3B
:104FA000F60182839383A483B583CA01B90120915A
:104FB0009B0430919C0440919D0450919E040E945A
:104FC0001175D60116966D937D938D939C931997C9
:104FD0000E94B17AEDB7FEB73A960FB6F894FEBFCD
:104FE0000FBEEDBF0C941B316091A4047091A50419
:104FF00080E090E00E940C7A009761F160E070E040
:1050000040E150E00E94F1772091D2063091D30622
:105010002617370799F17093D3066093D20682ED75
:1050200096E060E070E042E050E00E94017C8091F8
:10503000D2069091D30600D000D02DE135E0ADB777
:10504000BEB712963C932E93119714969C938E9311
:1050500013970EC08091D2069091D30600D000D055
:1050600029E035E0EDB7FEB7328321839483838353
:105070000E94B17A0F900F900F900F900E94730CC6
:1050800000D000D08CEF94E0ADB7BEB712969C93E1
:105090008E93119781E090E014969C938E931397D2
:1050A0000E94B17A81EF94E0EDB7FEB792838183DD
:1050B00082E090E0948383830E94B17A86EE94E04C
:1050C000ADB7BEB712969C938E93119784E090E093
:1050D00014969C938E9313970E94B17A89ED94E075
:1050E000EDB7FEB79283818388E090E09483838359
:1050F0000E94B17A8EEC94E0ADB7BEB712969C9345
:105100008E93119780E190E014969C938E93139761
:105110000E94B17A82EC94E0EDB7FEB7928381836E
:1051200080E290E0948383830E94B17A84EB94E0E0
:10513000ADB7BEB712969C938E93119780E490E022
:1051400014969C938E9313970E94B17A86EA94E00A
:10515000EDB7FEB79283818380E890E094838383E8
:105160000E94B17A87E994E0ADB7BEB712969C93DE
:105170008E93119780E091E014969C938E931397F1
:105180000E94B17A88E894E0EDB7FEB792838183FC
:1051900080E092E0948383830E94B17A8CE794E06C
:1051A000ADB7BEB712969C938E93119780E094E0B2
:1051B00014969C938E9313970E94B17A8EE694E096
:1051C000EDB7FEB79283818380E098E09483838378
:1051D0000E94B17A81E694E0ADB7BEB712969C9377
:1051E0008E93119780E090E114969C938E93139781
:1051F0000E94B17A83E594E0EDB7FEB79283818394
:1052000080E090E2948383830E94B17A83E494E007
:10521000ADB7BEB712969C938E93119780E090E441
:105220005DC10E9481180C94B8316091A404709102
:10523000A50480E090E00E940C7A6BE173E00E948C
:10524000217A009711F481E001C080E00E94AD1A3C
:1052500020919F04222311F40C94B83100D000D087
:10526000EDB7FEB7319680E494E00FC00E9472194A
:1052700020919F04222311F40C94B83100D000D067
:10528000EDB7FEB731968DE394E0ADB7BEB7129699
:105290009C938E931197228313820C94AF310E94BA
:1052A0006D1920919F04222311F40C94B83100D081
:1052B00000D0EDB7FEB731968AE394E0E6CF609177
:1052C000A4047091A50480E090E00E940C7A8C0107
:1052D0006EEF72E00E94217A009739F48091BC044D
:1052E0009091BD0484600C948231C80161E073E048
:1052F0000E94217A4091BC045091BD04009711F4A2
:105300004B7FA6C342FF03C08EEF92E002C081E054
:1053100093E000D000D02AE735E00C94A9316091E9
:10532000A4047091A50480E090E00E940C7A0E9491
:105330000379803160F48093D70690E00E9437545F
:1053400087ED96E066E170E041E050E0E5C700D00F
:1053500000D0EDB7FEB731968EE795E0ADB7BEB79A
:1053600012969C938E9311978091D706828394CF47
:105370000C9400000C94B8316091A4047091A504C1
:1053800080E090E00E940C7A8C016EE273E00E9453
:10539000217A009739F4219A8091BC049091BD0440
:1053A0008061B0C7C80160E373E00E94217A009772
:1053B00039F4229A8091BC049091BD048062A2C706
:1053C000C80162E373E00E94217A009739F4239ABE
:1053D0008091BC049091BD04806494C7C80164E3CB
:1053E00073E00E94217A009739F4239A8091BC04DB
:1053F0009091BD04806886C7C80161E073E00E9497
:10540000217A4091BC045091BD04009739F44F704B
:105410005093BD044093BC042B9A78C744FF03C04B
:105420008EEF92E002C081E093E000D000D02CEA41
:1054300035E0EDB7FEB732832183948383830E94E6
:10544000B17A8091BC040F900F900F900F9085FF60
:1054500003C08EEF92E002C081E093E000D000D064
:1054600021EA35E0ADB7BEB712963C932E93119763
:1054700014969C938E9313970E94B17A8091BC04EA
:105480000F900F900F900F9086FF03C08EEF92E069
:1054900002C081E093E000D000D026E935E0EDB70E
:1054A000FEB732832183948383830E94B17A8091F3
:1054B000BC040F900F900F900F9087FF03C08EEFEA
:1054C00092E002C081E093E000D000D02BE835E00C
:1054D000ADB7BEB712963C932E93119714969C933A
:1054E0008E9313973CC700D086E394E0EDB7FEB7E8
:1054F000928381830E94B17A20919F040F900F9034
:105500002223A9F000D000D0EDB7FEB7319683E397
:1055100094E0ADB7BEB712969C938E9311972283F9
:1055200013820E94B17A0F900F900F900F9088E134
:105530000FB6F89480936000109260000FBE0C9438
:10554000007C16C70E94E14A13C76091A4047091C1
:10555000A50480E090E00E940C7A1C016EEF72E0DE
:105560000E94217A009749F40E948E518091BC04D8
:105570009091BD0481608D7FC5C6C10161E073E07B
:105580000E94217A009741F40E94F0508091BC045F
:105590009091BD048C7FB6C606E313E0C101B8014B
:1055A0000E94217A009749F40E94F0508091BC0437
:1055B0009091BD048E7F8260A5C68091BC0481FF5E
:1055C0000BC000D000D08BEB95E0EDB7FEB7928317
:1055D000818314830383C3C680FF03C08EEF92E0F0
:1055E00002C081E093E000D000D027EB35E070CF1F
:1055F00000D089E094E0EDB7FEB7928381830E94EA
:10560000B17A8DB79EB740970FB6F8949EBF0FBE84
:105610008DBFEDB7FEB731968BEE93E0ADB7BEB759
:1056200012969C938E93119780915B2090915C20B1
:10563000A0915D20B0915E2082839383A483B58383
:1056400080914F2090915020A0915120B0915220F4
:1056500086839783A087B1878091532090915420AF
:10566000A0915520B091562082879387A487B58753
:105670008091572090915820A0915920B0915A20A4
:1056800086879787A08BB18B0E94B17A20919F0467
:10569000EDB7FEB772960FB6F894FEBF0FBEEDBF22
:1056A000222309F465C600D000D0EDB7FEB73196CD
:1056B00088EE93E0EACDF89481E090E00E945708EC
:1056C000182F80E090E00E945708082F7894F894F3
:1056D00083E090E00E945708F82E82E090E00E945C
:1056E0005708E82E789400D000D000D02EED33E09B
:1056F000EDB7FEB7328321832091FC173091FD175F
:105700004091FE175091FF17ADB7BEB713962D937A
:105710003D934D935C9316970E94B17A00D000D0D0
:10572000EDB7FEB7319627EB33E0ADB7BEB71296B3
:105730003C932E931197E2821382F48215820683A2
:105740001782108711860E94B17AEDB7FEB73A969C
:105750000FB6F894FEBF0FBEEDBF0E94151A209140
:10576000660000D000D0EDB7FEB731968BEA93E02B
:10577000ADB7BEB712969C938E9311972283138276
:105780000E94B17A0F900F900F900F900E94730CAF
:1057900020919F04222309F4EBC500D000D0EDB77F
:1057A000FEB7319688EA93E070CD80E090E00E94E9
:1057B0007F0C81E090E00E947F0C20919F042223C7
:1057C00009F4D6C500D000D0EDB7FEB7319685EA12
:1057D00093E05BCD0E94F0170E94730C20919F0410
:1057E000222309F4C5C500D000D0EDB7FEB731962D
:1057F00082EA93E04ACD6091A4047091A50480E010
:1058000090E00E940C7A8C016EEF72E00E94217A87
:10581000009731F48091BC049091BD04886072C5FA
:10582000C80161E073E00E94217A4091BC0450916C
:10583000BD04009711F4477F0BC143FF03C08EEFF7
:1058400092E002C081E093E000D000D02FEB35E081
:1058500080C56091A4047091A50480E090E00E944E
:105860000C7A6BE373E00E94217A009741F5F8947B
:1058700087EF96E00E94C63E0CC0C8010D960E94BC
:1058800012428BE495E0B8010E94803EC8010E945C
:105890008C3F082F192F0115110579F704C087EFE8
:1058A00096E00E94073F87EF96E00E946C3F0097CA
:1058B000B1F787EF96E00E94C23E78944BC087EF25
:1058C00096E00E94C63E482F592F7A0101E413E06A
:1058D0003DC08DB79EB70C970FB6F8949EBF0FBE14
:1058E0008DBFEDB7FEB73196ADB7BEB712961C931C
:1058F0000E931197D70112968C911297828313827F
:1059000013968C9113978483158218968C9118970F
:105910008683178214968D919C9115979187808725
:1059200016968D919C911797938782870E949F7AF4
:10593000EDB7FEB73C960FB6F894FEBF0FBEEDBFB5
:10594000C7010E948C3F482F592F7A01E114F104BE
:1059500009F0BFCF20919F04222309F409C500D08C
:1059600000D0EDB7FEB731968FE993E08ECC0E9460
:10597000E71AFEC46091A4047091A50480E090E051
:105980000E940C7A8C016EEF72E00E94217A0097DF
:1059900051F48091BC049091BD0492609093BD0439
:1059A0008093BC0410C0C80161E073E00E94217ABA
:1059B0004091BC045091BD04009771F45D7F5093F9
:1059C000BD044093BC048CEB94E064E170E042E0E1
:1059D00050E00E94017C17C051FF03C08EEF92E09F
:1059E00002C081E093E000D000D023EC35E0EDB7B9
:1059F000FEB732832183948383830E94B17A0F9010
:105A00000F900F900F9081E00E947E0AB1C46091C8
:105A1000A4047091A50480E090E00E940C7A8C01AF
:105A200060E173E00E94217A009731F48091BC0418
:105A30009091BD049E7F66C4C80165E073E00E943A
:105A4000217A4091BC045091BD04009731F451601B
:105A50005093BD044093BC0459C450FF03C085E07B
:105A600093E002C080E193E000D000D028E633E06C
:105A7000ADB7BEB712963C932E93119703C46091B5
:105A8000A4047091A50480E090E00E940C7A009735
:105A9000A9F160E070E040E150E00E94F17760938E
:105AA000B6047093B7048093B8049093B90400D0FF
:105AB00000D000D02EE833E0EDB7FEB7328321836B
:105AC000ADB7BEB713966D937D938D939C93169748
:105AD0000E94B17AEDB7FEB736960FB6F894FEBFC6
:105AE0000FBEEDBF86EB94E06EE070E044E050E066
:105AF0000E94017C81E00E94971B3AC480E00E94D2
:105B0000971B0E94730C00D000D000D089E793E06F
:105B1000ADB7BEB712969C938E9311978091B60441
:105B20009091B704A091B804B091B904EDB7FEB755
:105B300083839483A583B6830E94B17A8DB79EB781
:105B400006960FB6F8949EBF0FBE8DBF81E00E94EF
:105B5000971B0E94730C20919F04222309F408C410
:105B600000D000D0EDB7FEB7319686E793E08DCB3D
:105B70006091A4047091A50480E090E00E940C7AEA
:105B8000009741F160E070E04AE050E00E94F17758
:105B90007093BB046093BA0400D000D0EDB7FEB799
:105BA000319629E533E0ADB7BEB712963C932E93FC
:105BB0001197738362830E94B17A0F900F900F90B8
:105BC0000F908AEB94E062E170E042E050E00E94C6
:105BD000017C14C000D000D088E393E0EDB7FEB79D
:105BE000928381838091BA049091BB0494838383D0
:105BF0000E94B17A0F900F900F900F9020919F0408
:105C0000222309F4B5C300D000D0EDB7FEB731961A
:105C100085E393E03ACB0E944F4220919F042223D8
:105C200009F4A6C300D000D0EDB7FEB7319682E3E9
:105C300093E02BCB00D082E293E0EDB7FEB79283E6
:105C400081830E94B17A0F900F900E946D1900D04D
:105C500000D08AE193E0ADB7BEB712969C938E93C5
:105C6000119786E997E114969C938E9313970E945F
:105C7000B17A0F900F9086E193E0EDB7FEB7928373
:105C800081830E94B17A0F900F9080E00E94AD1A3C
:105C900000D080E193E0ADB7BEB712969C938E938F
:105CA00011970E94B17A0F900F900E942610809158
:105CB000491C80FF02C00E9466110E94721900D028
:105CC00000D0EDB7FEB7319683E093E0ADB7BEB735
:105CD00012969C938E9311978091D706828313829C
:105CE0000E94B17A8BEE92E0EDB7FEB7928381838A
:105CF00080E490E0948383830E94B17A00D0EDB772
:105D0000FEB7319688ED92E0ADB7BEB712969C9380
:105D10008E9311978091C524828313828091C6242B
:105D2000848315820E94B17A0F900F9083EC92E0E9
:105D3000EDB7FEB7928381838091BA049091BB0442
:105D4000948383830E94B17A00D080EB92E0ADB758
:105D5000BEB712969C938E9311978091B604909142
:105D6000B704A091B804B091B904EDB7FEB783832E
:105D70009483A583B6830E94B17A8DB79EB70696A9
:105D80000FB6F8949EBF0FBE8DBF81E00E94971B97
:105D90000E94600B00D000D000D023EA32E0ADB703
:105DA000BEB712963C932E931197EDB7FEB763835F
:105DB0007483858396830E94B17A8DB79EB70696C9
:105DC0000FB6F8949EBF0FBE8DBF0E94970B0E9426
:105DD000740B00D000D000D025E932E0ADB7BEB7DB
:105DE00012963C932E931197EDB7FEB7638374839D
:105DF000858396830E94B17A8DB79EB706960FB6BB
:105E0000F8949EBF0FBE8DBF1D9B03C085E193E03C
:105E100002C081E093E000D000D029E832E0ADB7C5
:105E2000BEB712963C932E93119714969C938E9323
:105E300013970E94B17A2091A0243091A12440911F
:105E4000A2245091A3248091A4249091A524A091F0
:105E5000A624B091A72400D000D000D00DB71EB763
:105E60000F5F1F4F6BE672E0EDB7FEB77283618381
:105E7000F801228333834483558386839783A087E5
:105E8000B1870E94B17AEDB7FEB7319689E492E00E
:105E9000ADB7BEB712969C938E9311978091AD24A7
:105EA0009091AE24A091AF24B091B02482839383CB
:105EB000A483B5838091B1249091B224A091B3249E
:105EC000B091B42486839783A087B1870E94B17A6A
:105ED000EDB7FEB738960FB6F894FEBF0FBEEDBF14
:105EE0008FE392E0928381830E94B17A8091BC0417
:105EF0000F900F9081FF0EC000D089E392E0ADB704
:105F0000BEB712969C938E9311970E94B17A0F9010
:105F10000F9017C080FF03C08EEF92E002C081E0B7
:105F200093E000D000D025E332E0EDB7FEB7328336
:105F30002183948383830E94B17A0F900F900F90F6
:105F40000F908091BC0483FF03C08EEF92E002C0EB
:105F500081E093E000D000D022E232E0ADB7BEB7DE
:105F600012963C932E93119714969C938E931397AD
:105F70000E94B17A8091BC049091BD040F900F9063
:105F80000F900F9091FF03C08EEF92E002C081E06E
:105F900093E000D000D025E132E0EDB7FEB73283C8
:105FA0002183948383830E94B17A8091D206909159
:105FB000D30628E032E0ADB7BEB712963C932E93DD
:105FC000119714969C938E9313970E94B17A0F9019
:105FD0000F900F900F90779903C08EEF92E002C060
:105FE00081E093E000D000D02FEF31E0EDB7FEB7B5
:105FF00032832183948383830E94B17A8091BC048D
:106000009091BD040F900F900F900F9090FF03C0E0
:1060100085E093E002C080E193E000D000D028E664
:1060200033E0ADB7BEB712963C932E9311971496FA
:106030009C938E9313970E949F7A20919F040F90B8
:106040000F900F900F90222309F492C100D000D03E
:10605000EDB7FEB731968CEF91E017C90E943A1A5E
:1060600020919F04222309F483C100D000D0EDB712
:10607000FEB7319689EF91E008C90E943617009764
:10608000B9F500D000D000D08EEE91E0EDB7FEB7AC
:10609000928381838091451890914618A09147186A
:1060A000B091481883839483A583B6830E94B17A04
:1060B00081EE91E0ADB7BEB712969C938E93119787
:1060C0008091C1249091C224A091C324B091C42492
:1060D000EDB7FEB783839483A583B6830E94B17A1C
:1060E0008DB79EB706960FB6F8949EBF0FBE8DBFB4
:1060F0000E94730C20919F04222309F439C100D01F
:1061000000D0EDB7FEB731968EED91E0BEC883E0CA
:1061100061E048E021E00E94F11200D000D000D000
:1061200087ED91E0EDB7FEB79283818380913818B7
:1061300090913918A0913A18B0913B1883839483B9
:10614000A583B6830E94B17A00D000D0EDB7FEB728
:10615000319686EC91E0ADB7BEB712969C938E93C4
:10616000119780913C1890913D18A0913E18B091E4
:106170003F1882839383A483B583809140189091C4
:106180004118A0914218B091431886839783A08745
:10619000B1870E94B17AEDB7FEB73A960FB6F89480
:1061A000FEBF0FBEEDBF0E94730C20919F042223FF
:1061B00009F4DEC000D000D0EDB7FEB7319683EC15
:1061C00091E063C86091A4047091A50480E090E020
:1061D0000E940C7A61E773E00E94217A0097B1F483
:1061E0006091A4047091A50480E090E00E940C7A74
:1061F000009709F4BDC00E940379803108F0B8C04F
:1062000090915201982B90935201B2C0809152010B
:1062100000D000D027EC35E0EDB7FEB73283218304
:1062200090E08F709070948383830E94B17A0F9076
:106230000F900F900F900E94730C9AC06091A4046D
:106240007091A50480E090E00E940C7ABC01009758
:1062500069F086E997E14AE050E00E942A7A86E9EF
:1062600097E160E270E04AE050E056C000D000D014
:1062700086E793E0ADB7BEB712969C938E931197C5
:1062800086E997E114969C938E9313970E949F7AC8
:1062900068C06091A4047091A50480E090E00E9421
:1062A0000C7A8C016EEF72E00E94217A009741F423
:1062B0000E94D24F8091BC049091BD04946022C092
:1062C000C80161E073E00E94217A009741F5F894DB
:1062D0000E94E04F88E10FB6F8948093600010921E
:1062E00060000FBE84B7877F84BF809160008861A3
:1062F000809360001092600078948091BC0490912B
:10630000BD049B7F9093BD048093BC048CEB94E010
:1063100064E170E042E050E00E94017C29C0C801C5
:106320006EE773E00E94217A4091BC045091BD0455
:10633000009721F452FF1CC0F894FFCF52FF03C016
:106340008EEF92E002C081E093E000D000D024ED17
:1063500035E0EDB7FEB732832183948383830E94B7
:10636000B17A0F900F900F900F9002C00E945A18B0
:10637000A981BA8111961C921E9283E00F900F9012
:10638000CF91DF911F910F91FF90EF90DF90CF9011
:10639000BF90AF909F908F907F906F905F904F9045
:1063A0003F902F900895F89491E2E0E0F0E0909310
:1063B00057008491E2E0F0E0909357002491E4E0EC
:1063C000F0E090935700E49190E0A0E0B0E0DC01B1
:1063D0009927882730E040E050E0542F432F322F98
:1063E0002227820F931FA41FB51F8E0F911DA11D81
:1063F000B11D8093FC179093FD17A093FE17B093E7
:10640000FF1778940895DF93CF93CDB7DEB76197E8
:106410000FB6F894DEBF0FBECDBFCE0102966EE080
:1064200070E042E050E00E94E37B8A819B812FEF85
:106430008F3F920749F486EB94E06EE070E042E013
:1064400050E00E94017C0AC0A0E0B0E08093B60456
:106450009093B704A093B804B093B904CE01029608
:1064600062E170E042E050E00E94E37B8A819B8120
:106470002FEF8F3F920779F48CE390E09093BB0469
:106480008093BA048AEB94E062E170E042E050E06D
:106490000E94017C04C09093BB048093BA04CE0197
:1064A000029664E170E042E050E00E94E37B8A8162
:1064B0009B812FEF8F3F920779F48AE090E09093D1
:1064C000BD048093BC048CEB94E064E170E042E096
:1064D00050E00E94017C04C09093BD048093BC04F2
:1064E000CE01029660E070E042E050E00E94E37B63
:1064F0008A819B812FEF8F3F920769F41092D30618
:106500001092D20682ED96E060E070E042E050E04A
:106510000E94017C04C09093D3068093D20685EB41
:1065200094E267E170E049E050E00E94E37B0E9462
:10653000E20DCE01049666E070E044E050E00E9477
:10654000E37B8C819D81AE81BF818F3F2FEF9207CE
:106550002FEFA2072FEFB20749F487E994E066E036
:1065600070E044E050E00E94017C08C087E994E0BC
:1065700066E070E044E050E00E94E37BCE010496C8
:106580006AE070E044E050E00E94E37B8C819D81F2
:10659000AE81BF818F3F2FEF92072FEFA2072FEF22
:1065A000B20749F48BE994E06AE070E044E050E01F
:1065B0000E94017C08C08BE994E06AE070E044E04E
:1065C00050E00E94E37BCE01049662E070E044E07C
:1065D00050E00E94E37B8C819D81AE81BF818F3F23
:1065E0002FEF92072FEFA2072FEFB20749F483E9AD
:1065F00094E062E070E044E050E00E94017C08C05A
:1066000083E994E062E070E044E050E00E94E37BC4
:10661000CE01019666E170E041E050E00E94E37B2C
:1066200089818F3F49F487ED96E066E170E041E0B3
:1066300050E00E94017C08C087ED96E066E170E0C2
:1066400041E050E00E94E37BCE01089660E270E0FA
:106650004AE050E00E94E37B88858F3F49F486E959
:1066600097E160E270E04AE050E00E94017C08C0DF
:1066700086E997E160E270E04AE050E00E94E37B47
:1066800061960FB6F894DEBF0FBECDBFCF91DF91FC
:1066900008950E94C64F6C9A6B9A6A9A6F9A729A82
:1066A000749A739A779A809880B3897F80BB87E0C9
:1066B00080937E00549A0E94D3310E94033281E07D
:1066C0000E947E0A80E090E00E94F60D0E944F49F1
:1066D0008091BC0486FD239A0895CF93DF93EC014B
:1066E00088819981009731F02AE08831920709F07A
:1066F00092C088C00E9449338091BC0480FD06C0CE
:1067000081FF02C01D9902C00E94F050809170006C
:106710008C7F809370008091B60080628093B60079
:106720001092B20082E08093B1008091B60090E0B8
:10673000877090700097C9F7809170008160809396
:10674000700080E090E06EE578E00E94A94F0E9422
:106750006D1980E00E94AD1A00D08DEB91E0ADB7CD
:10676000BEB712969C938E9311970E94B17A0F90A8
:106770000F900E9426108091491C86FF02C00E9443
:106780008C4A8091D70690E00E9437548AE180932A
:1067900005078AE190E00E94AF5200D000D000D0FF
:1067A000EDB7FEB7319683E893E0ADB7BEB712966A
:1067B0009C938E9311978091050782831382809119
:1067C000D706848315820E949F7A10920407109244
:1067D0000307EDB7FEB736960FB6F894FEBF0FBEAF
:1067E000EDBF8AEC94E09093BF248093BE2483E2B3
:1067F00090E09093FC068093FB0688E19AE09983F1
:1068000088830DC0633259F483E097E060E070E064
:106810000E94BE1EE6CF1982188283E001C081E08B
:10682000DF91CF9108958436910564F12091D206CD
:106830003091D30620FF10C000D000D025E933E00E
:10684000EDB7FEB732832183948383830E949F7ABE
:106850000F900F900F900F9080915B2090915C2093
:10686000A0915D20B0915E200196A11DB11D809385
:106870005B2090935C20A0935D20B0935E2021E08C
:1068800030E002C020E030E0C90108956F927F92AD
:106890008F929F92AF92BF92CF92DF92EF92FF9230
:1068A0000F931F93DF93CF93CDB7DEB7CB57D04075
:1068B0000FB6F894DEBF0FBECDBF3C01633851F474
:1068C00083EE96E0EC966FAFEC970E94063CEC9658
:1068D0006FADEC97D3018D919C911197B8E08A3FF1
:1068E0009B07E9F0E8E08B3F9E0718F4009761F002
:1068F000FDC6F9E08E3D9F0709F4D1C629E0853E2B
:10690000920709F0F3C6E4C683EE96E061E870E012
:1069100047E455E00E94EB3B8AEF98E0D4C6623131
:1069200009F0E9C60E94970B8091B6049091B704D4
:10693000A091B804B091B90493FF02C00E94361729
:106940008091B6049091B704A091B804B091B904B5
:1069500094FF0AC00E94600B6093A8247093A9243E
:106960008093AA249093AB248091B60480FF32C018
:10697000EDB7FEB738970FB6F894FEBF0FBEEDBF68
:106980003196CE010396ADB7BEB712969C938E9307
:10699000119787E790E09383828389EA93E0958358
:1069A000848386E997E1978386830E940F7BE82E94
:1069B000092FEDB7FEB738960FB6F894FEBF0FBE9D
:1069C000EDBF0E941334009709F0A6CF802F0E2D43
:1069D000182F02C000E010E08091B60481FF5FC074
:1069E00083E0C82ED12CCC0EDD1E00D000D000D00C
:1069F000EDB7FEB73196C601800F911FADB7BEB798
:106A000012969C938E93119787E790E093838283ED
:106A100081EB93E0958384830E940F7B080F191FFD
:106A2000B5EBEB2EB4E2FB2EEDB7FEB736960FB604
:106A3000F894FEBF0FBEEDBFA7E7AA2EB12CF5EB71
:106A40008F2EF3E09F2ED7012D917D01EDB7FEB77C
:106A500038970FB6F894FEBF0FBEEDBF3196C60152
:106A6000800F911FADB7BEB712969C938E9311976E
:106A7000B382A28295828482268317820E940F7B32
:106A8000080F191FEDB7FEB738960FB6F894FEBF82
:106A90000FBEEDBFFDEBEF16F4E2FF06A1F680910D
:106AA000B6049091B704A091B804B091B9040097CE
:106AB000A105B10581F12DB73EB7285030400FB682
:106AC000F8943EBF0FBE2DBFEDB7FEB73196CE0195
:106AD0000396800F911FADB7BEB712969C938E930D
:106AE000119787E790E0938382838AEB93E0958305
:106AF00084838091D5069091D606978386830E94E1
:106B00000F7B080F191FEDB7FEB738960FB6F89434
:106B1000FEBF0FBEEDBF8091B60482FF50C089E278
:106B200090E06BE270E04AE250E027E00E946546A8
:106B300085EB94E20E94D5482DB73EB72A503040ED
:106B40000FB6F8943EBF0FBE2DBFEDB6FEB608944B
:106B5000E11CF11C9E012D5F3F4F200F311FADB78F
:106B6000BEB712963C932E93119727E730E0F701BA
:106B70003383228321EC33E0358324839C01B901E4
:106B8000882777FD8095982F0E94617420E030E07F
:106B900048EC52E40E94F773D70116966D937D93EB
:106BA0008D939C9319970E940F7B080F191FEDB7C7
:106BB000FEB73A960FB6F894FEBF0FBEEDBF8091B8
:106BC000B60483FF56C089E290E06BE270E04AE2CF
:106BD00050E026E00E94654681E090E00E94E70BCD
:106BE0008093D90684EB97E10E94D5482DB73EB734
:106BF0002A5030400FB6F8943EBF0FBE2DBFEDB601
:106C0000FEB60894E11CF11C9E012D5F3F4F200F42
:106C1000311FADB7BEB712963C932E93119727E75D
:106C200030E0F701338322832BEC33E03583248378
:106C30009C01B901882777FD8095982F0E94617487
:106C400020E030E048EC52E40E94F773D70116963A
:106C50006D937D938D939C9319970E940F7B080FE2
:106C6000191FEDB7FEB73A960FB6F894FEBF0FBEE8
:106C7000EDBF8091B60484FF36C02DB73EB72A50D1
:106C800030400FB6F8943EBF0FBE2DBFEDB7FEB734
:106C90003196CE010396800F911FADB7BEB7129605
:106CA0009C938E93119787E790E09383828386ED80
:106CB00093E0958384838091A0179091A117A09170
:106CC000A217B091A31786839783A087B1870E94EC
:106CD0000F7B080F191FEDB7FEB73A960FB6F89461
:106CE000FEBF0FBEEDBF8091B60485FF31C00E948C
:106CF000740B2DB73EB72A5030400FB6F8943EBF04
:106D00000FBE2DBFEDB7FEB731969E012D5F3F4FF1
:106D1000200F311FADB7BEB712963C932E9311973B
:106D200027E730E03383228324EE33E03583248366
:106D300066837783808791870E940F7B080F191FD6
:106D4000EDB7FEB73A960FB6F894FEBF0FBEEDBF93
:106D50008091B60486FF3AC0F8948091A024909167
:106D6000A124A091A224B091A32478942DB73EB77A
:106D70002A5030400FB6F8943EBF0FBE2DBF4DB71E
:106D80005EB74F5F5F4F9E012D5F3F4F200F311F5A
:106D9000EDB7FEB73283218327E730E0FA01338372
:106DA000228322EF33E03583248386839783A08771
:106DB000B1870E940F7B080F191F2DB73EB7265FC2
:106DC0003F4F0FB6F8943EBF0FBE2DBF8091B60463
:106DD00087FF8AC08091BA049091BB04009709F4A0
:106DE00083C0F894C090A024D090A124E090A22465
:106DF000F090A32478948091AC179091AD17A09156
:106E0000AE17B091AF17A7019601281B390B4A0B9B
:106E10005B0BCA01B9010E945F74862EA72EB82EA3
:106E2000992E6091BA047091BB0480E090E00E94BA
:106E30005F749B01AC01682D7A2D8B2D992D0E94DA
:106E4000F7735C014DB75EB74A5050400FB6F894E7
:106E50005EBF0FBE4DBFEDB7FEB73196CE010396B4
:106E6000800F911FADB7BEB712969C938E9311976A
:106E700087E790E0938382838BEF93E0958384830D
:106E8000262F372F4A2D5B2D268337834087518746
:106E9000EC966FAFEC97EB967FAFEB970E940F7B72
:106EA000080F191FEC966FADEC97EB967FADEB9743
:106EB000862F972FAA2DBB2D8093AD249093AE24BF
:106EC000A093AF24B093B024C092AC17D092AD176A
:106ED000E092AE17F092AF17EDB7FEB73A960FB645
:106EE000F894FEBF0FBEEDBF8091B6049091B70439
:106EF000A091B804B091B90490FF40C0F89480917B
:106F0000A4249091A524A091A624B091A7247894BC
:106F10002DB73EB72A5030400FB6F8943EBF0FBE93
:106F20002DBF4DB75EB74F5F5F4F9E012D5F3F4F47
:106F3000200F311FEDB7FEB73283218327E730E002
:106F4000FA013383228328E034E035832483868367
:106F50009783A087B1870E940F7B080F191F2DB759
:106F60003EB7265F3F4F0FB6F8943EBF0FBE2DBF12
:106F7000C8010E941334009709F0CECC8091B6046A
:106F80009091B704A091B804B091B90491FF88C062
:106F90008091BA049091BB04009709F481C0F894E1
:106FA000C090A424D090A524E090A624F090A7241B
:106FB00078948091B0179091B117A091B217B091C9
:106FC000B317A7019601281B390B4A0B5B0BCA01AB
:106FD000B9010E945F745B014C016091BA04709129
:106FE000BB0480E090E00E945F749B01AC016A2DBD
:106FF0007B2D882D992D0E94F7735C014DB75EB7EC
:107000004A5050400FB6F8945EBF0FBE4DBFEDB76B
:10701000FEB73196CE010396800F911FADB7BEB774
:1070200012969C938E93119787E790E093838283C7
:1070300081E194E095838483262F372F4A2D5B2DA1
:107040002683378340875187EC966FAFEC97EB969A
:107050007FAFEB970E940F7B080F191FEC966FAD67
:10706000EC97EB967FADEB97862F972FAA2DBB2D34
:107070008093B1249093B224A093B324B093B4240A
:10708000C092B017D092B117E092B217F092B31736
:10709000EDB7FEB73A960FB6F894FEBF0FBEEDBF40
:1070A0008091B6049091B704A091B804B091B9044E
:1070B00092FF3EC080914B2090914C20A0914D209A
:1070C000B0914E202DB73EB72A5030400FB6F894FD
:1070D0003EBF0FBE2DBF4DB75EB74F5F5F4F9E01E6
:1070E0002D5F3F4F200F311FEDB7FEB73283218355
:1070F00027E730E0FA01338322832EE134E0358341
:10710000248386839783A087B1870E940F7B080F13
:10711000191F2DB73EB7265F3F4F0FB6F8943EBFFD
:107120000FBE2DBFC8010E941334009709F0F4CBA5
:107130008091B6049091B704A091B804B091B904BD
:1071400093FF3CC04DB75EB74A5050400FB6F8941D
:107150005EBF0FBE4DBFEDB7FEB73196CE010396B1
:10716000800F911FADB7BEB712969C938E93119767
:1071700087E790E09383828387E294E0958384831A
:107180008091451890914618A0914718B0914818E1
:1071900086839783A087B1870E940F7B080F191FF2
:1071A000EDB7FEB73A960FB6F894FEBF0FBEEDBF2F
:1071B000C8010E941334009709F0AECB8091B60449
:1071C0009091B704A091B804B091B90494FF3CC069
:1071D0002DB73EB72A5030400FB6F8943EBF0FBED1
:1071E0002DBFEDB7FEB73196CE010396800F911FEC
:1071F000ADB7BEB712969C938E93119787E790E038
:107200009383828382E394E0958384838091A8248E
:107210009091A924A091AA24B091AB24868397834E
:10722000A087B1870E940F7B080F191FEDB7FEB72B
:107230003A960FB6F894FEBF0FBEEDBFC8010E948C
:107240001334009709F068CB8091B6049091B7048D
:10725000A091B804B091B90495FF48C081E00E94A4
:10726000120B2DB73EB72A5030400FB6F8943EBFF0
:107270000FBE2DBFEDB6FEB60894E11CF11C9E01B9
:107280002D5F3F4F200F311FADB7BEB712963C9315
:107290002E93119727E730E0F701338322832FE302
:1072A00034E03583248320919704309198044091F1
:1072B000990450919A040E941175D70116966D9306
:1072C0007D938D939C9319970E940F7B080F191F34
:1072D000EDB7FEB73A960FB6F894FEBF0FBEEDBFFE
:1072E000C8010E941334009709F016CB8091B604B0
:1072F0009091B704A091B804B091B90496FF48C02A
:1073000082E00E94120B2DB73EB72A5030400FB6D4
:10731000F8943EBF0FBE2DBFEDB6FEB60894E11C3B
:10732000F11C9E012D5F3F4F200F311FADB7BEB73F
:1073300012963C932E93119727E730E0F7013383A1
:1073400022832CE434E03583248320919B04309104
:107350009C0440919D0450919E040E941175D70198
:1073600016966D937D938D939C9319970E940F7B36
:10737000080F191FEDB7FEB73A960FB6F894FEBF87
:107380000FBEEDBFC8010E941334009709F0C4CAB4
:107390008091B6049091B704A091B804B091B9045B
:1073A00097FF06C083E061E046E020E00E94F11212
:1073B0008091B6049091B704A091B804B091B9043B
:1073C000A0FF06C083E061E046E021E00E94F112E8
:1073D0008091B6049091B704A091B804B091B9041B
:1073E00097FF3CC02DB73EB72A5030400FB6F894F7
:1073F0003EBF0FBE2DBFEDB7FEB73196CE0103964F
:10740000800F911FADB7BEB712969C938E931197C4
:1074100087E790E09383828389E594E09583848372
:1074200080913C1890913D18A0913E18B0913F1862
:1074300086839783A087B1870E940F7B080F191F4F
:10744000EDB7FEB73A960FB6F894FEBF0FBEEDBF8C
:10745000C8010E941334009709F05ECA8091B604F7
:107460009091B704A091B804B091B904A0FF3CC0BA
:107470002DB73EB72A5030400FB6F8943EBF0FBE2E
:107480002DBFEDB7FEB73196CE010396800F911F49
:10749000ADB7BEB712969C938E93119787E790E095
:1074A0009383828381E694E095838483809140185E
:1074B00090914118A0914218B09143188683978308
:1074C000A087B1870E940F7B080F191FEDB7FEB789
:1074D0003A960FB6F894FEBF0FBEEDBFC8010E94EA
:1074E0001334009709F018CA779A8091D2069091C8
:1074F000D30693FD749A8091D2069091D30682FDB3
:1075000008C08091BC0480FD04C081FF31C01D9B78
:107510002FC000D000D08CE694E0ADB7BEB7129675
:107520009C938E931197CE01039614969C938E9301
:1075300013970E949F7A20919F040F900F900F90B5
:107540000F902223A9F000D000D0EDB7FEB73196FE
:1075500087EB91E0ADB7BEB712969C938E931197CF
:10756000228313820E94B17A0F900F900F900F9098
:107570008FE189838091F6068A83FE01E00FF11F77
:10758000138278010894E11CF11C8091D20690913D
:10759000D30680FF12C000D000D083E794E0EDB79F
:1075A000FEB7928381830D5F1F4F148303830E9474
:1075B0009F7A0F900F900F900F9022E030E0E20E34
:1075C000F31E8E010F5F1F4FC801B7010E94634574
:1075D0008091BC0482FF42C086EA94E0B801A70112
:1075E00020EA30E20E94E8498091D2069091D306C9
:1075F00092FF34C000EA10E2E4E8CE2EE4E0DE2E92
:10760000D8018D918D0100D000D0EDB7FEB7319635
:10761000ADB7BEB71296DC92CE92119782831382D9
:107620000E949F7A0F900F900F900F90B0E2003B56
:107630001B0731F78AE090E00E94D17A00D000D099
:1076400089E894E0EDB7FEB792838183F482E38208
:107650000E949F7A0F900F900F900F908091D2060A
:107660009091D30682FD73980E948E5183EE96E02E
:107670000E94093C8091D5069091D606009711F0A2
:107680000E94F0508091F6068F5F8093F6068091FD
:10769000D2069091D30682FF3FC9739A3DC98EEE00
:1076A00096E00E94B040009731F10E948E51809187
:1076B000BC0487FD2B988EEE96E060E470E00E949B
:1076C000854085EE99E0D30111969C938E9313C06B
:1076D0008EEE96E00E94B040009769F00E94F05054
:1076E0008091BC0487FF18C92B9A16C9F301118237
:1076F000108283E001C081E0C558DF4F0FB6F894D7
:10770000DEBF0FBECDBFCF91DF911F910F91FF90D4
:10771000EF90DF90CF90BF90AF909F908F907F9031
:107720006F9008950895FC01DB018C918083119680
:107730008C91119781830895FC01DB0190818C91DC
:10774000981741F421E030E0918111968C911197C6
:10775000981711F020E030E0C9010895FC01808104
:107760008093C52481818093C6240895DC011996F5
:10777000ED91FC911A970280F381E02D309709F08A
:1077800009950895EF92FF920F931F93DF93CF9384
:1077900000D0CDB7DEB78C0188E10E94DE45BC0188
:1077A0007E010894E11CF11CC7010E94933BD801A3
:1077B0001996ED91FC911A970190F081E02DC80186
:1077C000B70109950F900F90CF91DF911F910F9105
:1077D000FF90EF900895EF92FF920F931F93CF9336
:1077E000DF93EC018B017A0147E555E00E94173CDD
:1077F000FA86E986C8016BE575E00E94763CDF9168
:10780000CF911F910F91FF90EF9008950E94303C0F
:107810000895CF93DF93EC0188E165EC74E20E9458
:10782000D445CE010E94333CDF91CF910895EF9271
:10783000FF920F931F93CF93DF93EC018B017A019B
:107840000E944F3CF886EF82C8016FE575E00E9408
:10785000763CDF91CF911F910F91FF90EF900895AB
:107860000E94583C08950E9465570895FC01A78125
:10787000B0852D913C91F90109950895DC01179689
:10788000ED91FC9118970280F381E02D309709F07B
:107890000995089588E89EE00E94C23E0895FC0183
:1078A0007383628388E89EE0BF010E944D3F089584
:1078B000BC0188E89EE00E94143F0895CF93DF93B7
:1078C000EC0188E89EE00E94C63E08C08281938158
:1078D0008C179D0739F0CF010E948C3FE82FF92FBC
:1078E0003097A1F7CF01DF91CF9108950F931F93A8
:1078F000CF93DF938B010E945E3CEC01009731F047
:107900001D830C83C8010E94BD598E83DF91CF91E6
:107910001F910F9108951F93CF93DF93EC01162FC2
:10792000888580FF1DC0EC81FD813097C9F0D09320
:107930008D0EC0938C0E82E08887CE010696099545
:10794000992787FD909502978230910510F01338A2
:1079500029F4CE01BE010E94B43C02C081E08887B8
:10796000DF91CF911F910895CF92DF92EF92FF9216
:107970000F931F93CF93DF93EC017B01C0908C0E8C
:10798000D0908D0E00918A0E10918B0EF80103C0DD
:107990000190F081E02DEC17FD0719F03097C1F749
:1079A00046C0209709F443C08885882309F11886CA
:1079B0000BC0C017D10729F0C80167E8AE010E94CB
:1079C0008B3CF801008111810115110591F7EC81C3
:1079D000FD81309769F0CE15DF0551F0D0938D0E03
:1079E000C0938C0ECE01069663E840E050E0099506
:1079F000E0918A0EF0918B0ECE17DF0791F488810B
:107A0000998190938B0E80938A0E0DC08081918115
:107A10008C179D0729F4888199819183808303C005
:107A2000FC01309799F7D0928D0EC0928C0EDF91A9
:107A3000CF911F910F91FF90EF90DF90CF9008951D
:107A40001F93CF93DF9310928E0EC0918A0ED09128
:107A50008B0E11E00EC08985882341F018871986A6
:107A6000CE0162E840E050E00E948B3C0990D88152
:107A7000C02D209781F7DF91CF911F9108958091BC
:107A8000390F982F9F5F9093390F089560918C0E56
:107A900070918D0E0E94B43C08958AE88093390F4E
:107AA0001092900E10928F0E10928B0E10928A0EE2
:107AB00010928D0E10928C0E089580918E0E882358
:107AC00011F00E94203D70918F0E772309F455C06C
:107AD0002091900E30E0F901EE0FFF1FEE0FFF1F17
:107AE000E20FF31FEF56F14F60816093380F418131
:107AF00052815093370F4093360F83819481909336
:107B0000350F8093340F2F5F3F4F2F7130702093CC
:107B1000900E715070938F0E009741F580918A0EF0
:107B200090918B0E18C080918E0E882311F00E94C8
:107B3000203D4091360F5091370F8091320F909138
:107B4000330F6091380F0E948B3CE091320FF0911F
:107B5000330F808191819093330F8093320F809106
:107B6000320F9091330F0097F1F607C0613819F486
:107B700021E0FC0120870E948B3C80918E0E209199
:107B80008F0E30E0280F311DC901089580918E0EAF
:107B900020918F0E30E0280F311DC901089570919A
:107BA0008F0E7032D9F02091900E270F2F712093F5
:107BB000310F30E0F901EE0FFF1FEE0FFF1FE20F54
:107BC000F31FEF56F14F6083528341839483838385
:107BD0007F5F70938F0E20E030E002C021E030E044
:107BE000C9010895CF93DF93C0918C0ED0918D0E73
:107BF0000E948B3CD0938D0EC0938C0EDF91CF9161
:107C00000895FC01AB0190918A0E80918B0E9C012E
:107C1000A32FB22F03C00D90BC91A02DAE17BF07AC
:107C200091F01097C1F7309771F090838183F093B2
:107C30008B0EE0938A0E81E0808717821682CF0137
:107C400061E80E94F23D0895FC01009741F08085B3
:107C50008150823020F481E0818780938E0E0895D8
:107C600021E030E0FC018085882311F420E030E041
:107C7000C9010895CF93DF93EC014A815B818C8128
:107C80009D8160E070E00E941A7A4A815B81888160
:107C90009981489F9001499F300D589F300D1124C4
:107CA0008E819F8160E070E0A9010E941A7ADF91C5
:107CB000CF910895FC018281938120E030E019C0CA
:107CC000A481B581A20FB31F4C91442381F481E0BC
:107CD0008C9340815181249FC001259F900D349F3A
:107CE000900D112426813781280F391F07C02F5F7F
:107CF0003F4F2817390720F320E030E0C9010895ED
:107D0000FC01268137814281538180E090E018C0D8
:107D10002617370781F4A481B581A80FB91F2C91CC
:107D2000121614F421502C930480F581E02DE80FF5
:107D3000F91F80810895A081B1812A0F3B1F019610
:107D40008417950728F38FEF0895FC01CB01268156
:107D500037816217730790F0A081B18162817381CE
:107D6000A69FA001A79F500DB69F500D1124420F52
:107D7000531F21E030E08417950710F020E030E039
:107D8000C9010895FC01118210820895FC018081CF
:107D900091810895FB0120813181FC013183208391
:107DA0000895FC01208131812115310511F407C0AE
:107DB0009C01F901808191810097D1F702C020E0F8
:107DC00030E0C9010895CF93DF93DC012D913C9100
:107DD000119721153105A9F0F90180819181009752
:107DE00029F411961C921E920EC0F9012081318156
:107DF000D9018D919C9111970097B9F7118210824A
:107E000002C020E030E0C901DF91CF910895DC018C
:107E1000ED91FC911197309729F080819181119615
:107E20009C938E93CF010895CF93DF93FC01A081A3
:107E3000B1811097D9F0C0E0D0E016C0A617B707FF
:107E400071F48D919C911197209719F491838083FF
:107E500002C09983888311961C921E9207C0ED017F
:107E600098818981A92FB82F109741F7DF91CF9181
:107E700008950F931F93CF93DF938C01EB010E9422
:107E8000143FF8018081918199838883D183C083D5
:107E9000DF91CF911F910F910895EF92FF920F9371
:107EA0001F93CF93DF93EC017B010E94143FF701F6
:107EB00011821082CE010E94D13EFC01009719F47C
:107EC000E882F98202C0F182E082DF91CF911F91B6
:107ED0000F91FF90EF900895DC01ED91FC911197C7
:107EE00020E030E005C02F5F3F4F0190F081E02D92
:107EF0003097C9F7C9010895FB01309721F4BA0101
:107F00000E94393F0895DA018081918111969C93F6
:107F10008E93518340830895009721F0FC012081C6
:107F2000318102C020E030E0C901089580913A0F0C
:107F300090913B0F009729F410923D0F10923C0F47
:107F400008950E94524EE0913A0FF0913B0F22812A
:107F5000338140815181240F351F281B390B0CC000
:107F60004281538160817181460F571F481B590B15
:107F70004217530708F49A010480F581E02D3097E9
:107F800079F7280F391F30933D0F20933C0F089548
:107F90008DE695E00E94243E0895CF92DF92EF9205
:107FA000FF920F931F93CF93DF937C01FC0180819D
:107FB0009181009729F08A35910509F06EC00BC0B8
:107FC00010923B0F10923A0F8AE590E0F7019183EF
:107FD000808381E066C0673849F5CA01E0913A0FB5
:107FE000F0913B0F03C00480F581E02D309741F301
:107FF0002681378128173907B1F3E0933A0FF093C0
:108000003B0F0FC016962D913C91179728173907F3
:1080100039F414962D913C91159735832483DF0113
:10802000FD01A481B581109769F7CECF623861F662
:10803000C0913A0FD0913B0F00E010E02BC0CE0171
:108040000E94B55D0097F1F08E819F8168E8AE01D6
:108050000E94CF3D0097A1F41F821E828C819D81DA
:108060000115110521F0F8019583848304C09093D4
:108070003B0F80933A0F1D821C820E94963FD8CFFF
:108080000E94C83F8E019C818D81C92EE6016E0140
:10809000D82EE601209799F697CFF701118210822A
:1080A00083E0DF91CF911F910F91FF90EF90DF90D0
:1080B000CF900895CF93DF93EC010E94C83F8E814B
:1080C0009F81009769F0E0913A0FF0913B0F06C055
:1080D000EC17FD07A9F00480F581E02D3097C1F77A
:1080E00080918C0E90918D0E9F838E8380913A0F9C
:1080F00090913B0F9D838C83D0933B0FC0933A0F9D
:108100000E94963FDF91CF910895CF93DF93EC01CA
:108110000E94955DCE010E945A40DF91CF91089553
:10812000CF93DF93EC010E94A15DCE010E945A40E3
:10813000DF91CF910895CF93DF93EC010E94AB5D67
:10814000CE010E945A40DF91CF910895FC018081B9
:108150009181860F971F918380830E94963F089597
:1081600021E030E0FC0186819781009711F020E04A
:1081700030E0C9010895FC01228133818081918121
:10818000280F391FC9010895FC018081918108954C
:1081900021E030E080913A0F90913B0F009711F46D
:1081A00020E030E0C901089580913A0F90913B0F93
:1081B000009729F020913C0F30913D0F02C020E044
:1081C00030E0C9010895CF93DF93EC01E0913A0FBD
:1081D000F0913B0F8E179F0741F48C819D81909306
:1081E0003B0F80933A0F14C0FC01309731F084812B
:1081F00095818C179D07C1F707C01D821C821F82C5
:108200001E82DF91CF9108958C819D819583848317
:108210000E94963FF2CFCF92DF92EF92FF920F93A0
:108220001F93CF93DF938C017A01FC0180819181B0
:10823000009729F08B34910509F051C01EC08FE3DF
:108240009FE00E94C63EC82EE6017E01F92EE7019E
:1082500009C06C817D81CE0102960E948540099003
:10826000D881C02D2097A9F781E080933E0F8BE441
:1082700090E0F8019183808337C06838A9F58FE3D7
:108280009FE00E94C63EC82EE6016E01D92EE6018F
:1082900023C0CE010296E816F906D9F48FE39FE0D9
:1082A000BE010E94143FE0908C0EF0908D0E8A85E6
:1082B0009B8590938D0E80938C0EEC85FD85309779
:1082C00019F08E859F850995F0928D0EE0928C0EA7
:1082D000CECF0990D881C02D2097D9F6C8CFF8010C
:1082E0001182108283E001C081E0DF91CF911F9164
:1082F0000F91FF90EF90DF90CF90089510923E0F76
:108300008FE39FE00E94C23E86E895E060E070E067
:108310000E94013E08950F931F93CF93DF93EC01CA
:1083200000918C0E10918D0E1B870A875D874C87FC
:108330003F872E8780913E0F882379F086E895E06D
:1083400090938D0E80938C0ECE0102960E948540F4
:1083500010938D0E00938C0E02C07D836C838FE38F
:108360009FE0BE010E94143F8FE39FE0BE010E9488
:108370004D3FDF91CF911F910F9108950F931F9360
:10838000CF93DF93EC0180913E0F882391F0009111
:108390008C0E10918D0E86E895E090938D0E809353
:1083A0008C0ECE0102960E94904010938D0E009389
:1083B0008C0E8FE39FE0BE010E94143F8FE39FE08D
:1083C000BE010E944D3FDF91CF911F910F91089503
:1083D0000F931F93CF93DF93EC0180913E0F88237F
:1083E00091F000918C0E10918D0E86E895E090939F
:1083F0008D0E80938C0ECE0102960E949B401093AE
:108400008D0E00938C0E8FE39FE0BE010E94143FFF
:108410008FE39FE0BE010E944D3FDF91CF911F91FE
:108420000F910895CF93DF93EC0180913E0F882345
:1084300029F0CE0102960E94E34004C01F821E82F2
:10844000198618868FE39FE0BE010E94143FDF91DA
:10845000CF910895CF93DF93EC0180913E0F882355
:1084600031F0CE0102960E94B0409C0114C08FE30F
:108470009FE00E94C63EE82FF92F06C0EC17FD07CB
:1084800041F00190F081E02D3097C1F721E030E01C
:1084900002C020E030E0C901DF91CF9108950F9331
:1084A0001F930091C5241091C6240E947F4E2DB7C2
:1084B0003EB7225530400FB6F8943EBF0FBE2DBFD9
:1084C000EDB7FEB7319629E73DE0ADB7BEB71296DE
:1084D0003C932E9311970283138214831582668333
:1084E0007783808791878091B8269091B926A09153
:1084F000BA26B091BB2682879387A487B5878091DF
:10850000BC269091BD26A091BE26B091BF2686873D
:108510009787A08BB18B8091C0269091C126A091A6
:10852000C226B091C326828B938BA48BB58B80918E
:10853000C4269091C526A091C626B091C726868BE9
:10854000978BA08FB18F8091C8269091C926A0915A
:10855000CA26B091CB26828F938FA48FB58F80913E
:10856000CC269091CD26A091CE26B091CF26868F95
:10857000978FA0A3B1A38091D0269091D126A091EE
:10858000D226B091D32682A393A3A4A3B5A38091AE
:10859000D4269091D526A091D626B091D72686A331
:1085A00097A3A0A7B1A78091D8269091D926A09192
:1085B000DA26B091DB2682A793A7A4A7B5A780915E
:1085C000DC269091DD26A091DE26B091DF2686A7DD
:1085D00097A7A0ABB1AB8091E0269091E126A09146
:1085E000E226B091E32682AB93ABA4ABB5AB80910E
:1085F000E4269091E526A091E626B091E72686AB89
:1086000097ABA0AFB1AF8091E8269091E926A091F9
:10861000EA26B091EB2682AF93AFA4AFB5AFEDB72A
:10862000FEB7FF968091EC269091ED26A091EE2664
:10863000B091EF2680839183A283B383EDB7FEB719
:10864000ED5BFF4F8091F0269091F126A091F226EC
:10865000B091F32680839183A283B383EDB7FEB7F5
:10866000E95BFF4F8091F4269091F526A091F626C4
:10867000B091F72680839183A283B383EDB7FEB7D1
:10868000E55BFF4F8091F8269091F926A091FA269C
:10869000B091FB2680839183A283B383EDB7FEB7AD
:1086A000E15BFF4F8091FC269091FD26A091FE2674
:1086B000B091FF2680839183A283B3830E94B17A15
:1086C0000091C5241091C6242DB73EB72E5A3F4FB6
:1086D0000FB6F8943EBF0FBE2DBF0E947F4EADB7C0
:1086E000BEB7D2970FB6F894BEBF0FBEADBFEDB701
:1086F000FEB731962AE03DE012963C932E931197F7
:10870000028313821483158266837783808791871F
:108710008091002790910127A0910227B091032713
:1087200082879387A487B587809104279091052736
:10873000A0910627B091072786879787A08BB18BDA
:108740008091082790910927A0910A27B0910B27C3
:10875000828B938BA48BB58B80910C2790910D27E6
:10876000A0910E27B0910F27868B978BA08FB18F8A
:108770008091102790911127A0911227B091132773
:10878000828F938FA48FB58F809114279091152796
:10879000A0911627B0911727868F978FA0A3B1A31A
:1087A0008091182790911927A0911A27B0911B2723
:1087B00082A393A3A4A3B5A380911C2790911D2706
:1087C000A0911E27B0911F2786A397A3A0A7B1A7AA
:1087D0008091282790912927A0912A27B0912B27B3
:1087E00082A793A7A4A7B5A780912C2790912D27A6
:1087F000A0912E27B0912F2786A797A7A0ABB1AB4A
:108800000E94B17A2DB73EB72E5C3F4F0FB6F89459
:108810003EBF0FBE2DBF1F910F91089580E380933F
:10882000410F0895EF92FF92CF93DF932091410F74
:1088300030E0C0E3D0E0C21BD30B2A5B304FB9015C
:10884000AE010E94117ACE01DF91CF91FF90EF909F
:108850000895AF92BF92CF92DF92EF92FF920F9363
:108860001F93CF93DF937C01C090420FD090430FB2
:108870002091410F30E08601005D1F4F021B130B5A
:1088800001381105E0F4C0E3D0E0C21BD30B2A5B32
:10889000304FB901AE010E94117ACE0DDF1D20913B
:1088A000440F3091450F8091F80F9091F90F280FE8
:1088B000391FCE01B901A6010E94117A02C000E061
:1088C00010E0C801DF91CF911F910F91FF90EF90C1
:1088D000DF90CF90BF90AF9008959091410F980F87
:1088E0009093410F08954091420F5091430F9C0186
:1088F0004817590798F08091F80F9091F90F820F5F
:10890000931F9093F90F8093F80F421B530B5093D2
:10891000430F4093420F21E030E002C020E030E0FE
:10892000C90108959093430F8093420F08952091B9
:10893000F80F3091F90F2A58304FC901089520914E
:10894000410F30E02A5B304FC901089521E030E04B
:108950008091440F9091450F4FE08637940711F4B2
:1089600020E030E0C90108950E94A644009771F00C
:1089700026E73FE06091440F7091450F4091420F10
:108980005091430FC9010E94117A0895A091F80FE8
:10899000B091F90F1097B9F02091420F3091430F29
:1089A000205D3F4FAA58B04FE6E7FFE080E390E03C
:1089B00003C04D914193019682179307D4F310920F
:1089C000F90F1092F80F08958091440F9091450F80
:1089D00008958091420F9091430F08959091410F17
:1089E00080E3891B089580E39091410F891B2091BA
:1089F000420F3091430F280F311DC90108951F9375
:108A0000CF93DF93EC011091410F812F90E08C17F1
:108A10009D076CF00E94F3448C0F9D1F81389105D7
:108A200030F41C1B1093410F21E030E002C020E025
:108A300030E0C901DF91CF911F910895CF93DF936B
:108A4000EFECF4E21192119284E2EF3FF807D1F7D4
:108A5000C0E0D0E0CE01880F991F89539B4D65E59A
:108A600075E00E94933B2196C430D10599F7DF91C0
:108A7000CF9108951092F90F1092F80F1092430FB2
:108A80001092420F80E38093410F86E79FE090931E
:108A9000450F8093440F0E941E4508950F931F9326
:108AA000CF93DF93EC018B010E943A45D093450FA1
:108AB000C093440F1093430F0093420FDF91CF9167
:108AC0001F910F910895CF92DF92EF92FF920F9333
:108AD0001F93DF93CF9300D0CDB7DEB78C016983AE
:108AE0007A830E943A4569817A81C62ED72E21E881
:108AF000C216D10418F030E8C32ED12C8091440F57
:108B00009091450FB801A6010E94117AD092430FAF
:108B1000C092420FC6010F900F90CF91DF911F912D
:108B20000F91FF90EF90DF90CF900895282F392F6D
:108B3000D901EFECF4E280E301900D928150E1F76E
:108B4000862F972FDC01E7ECF4E288E001900D928C
:108B50008150E1F70895EFECF4E2282F392FD90185
:108B600080E30D9001928150E1F7A7ECB4E2862FEB
:108B7000972FFC0188E001900D928150E1F7089554
:108B8000E82FF0E0EE0FFF1FE153FB4D7183608390
:108B900081E090E00895E82FF0E0EE0FFF1FE15331
:108BA000FB4D80819181089590E0880F991F89562F
:108BB0009B4D0E94933B81E090E00895282F30E088
:108BC000220F331F29563B4DC90108958115910588
:108BD00011F00197F1F70895E0910225F091032536
:108BE00090818091012589230895E091FF24F091DF
:108BF0000025808190910125892B8083E0910425B7
:108C0000F0910525808190910125892B808308951D
:108C1000E091FF24F09100259081809101258095BD
:108C200089238083E0910425F0910525908180912E
:108C300001258095892380830895FF920F931F93C8
:108C4000E091FF24F091002590818091012580958D
:108C500089238083E0910425F091052580819091FE
:108C60000125892B80838FEB93E00E94E645FFB6B8
:108C7000F894E0910425F0910525908180910125DB
:108C800080958923808383E890E00E94E645E09107
:108C90000225F0910325008110910125FFBE7894F3
:108CA0008BE393E00E94E645E0910225F0910325D5
:108CB000808190910125892319F0802F812301C0A3
:108CC00081E01F910F91FF900895509305254093E7
:108CD0000425709300256093FF24909303258093CF
:108CE000022581E090E002C0880F991F2A95E2F7E3
:108CF000809301250E941D4608950F931F93182FFE
:108D00000FB7F894E0910425F091052580819091AA
:108D10000125892B808383E090E00E94E6451123A2
:108D200051F0E0910425F091052590818091012575
:108D300080958923808387E190E00E94E645E09159
:108D40000225F0910325808190910125892309F462
:108D500010E089E590E00E94E645E0910425F0915D
:108D600005259081809101258095892380830FBFFF
:108D70008BE390E00E94E645812F1F910F910895AB
:108D80000F931F93182F08E0812F81700E947D465A
:108D90001695811110680150B9F7812F1F910F911D
:108DA00008958FEF0E94C0460895DF92EF92FF92E0
:108DB0000F931F93CF93DF93182FEB010E941D4653
:108DC000882389F580EF0E94C046EE2400E498EFE6
:108DD000D92ED00E81E00E947D46F82E81E00E94BF
:108DE0007D46882319F0FF2069F020C0FF2051F450
:108DF000011728F0888180FF05C0101719F0E02EB8
:108E0000FF24F3948F2D0E947D4688818695888368
:108E1000FF2011F08068888301500D15D9F60023DA
:108E200039F02196D4CFEE24EA9402C08EEFE82EDA
:108E30008E2DDF91CF911F910F91FF90EF90DF90DA
:108E400008950F931F93CF93DF93182FEB010E9488
:108E50001D46209751F085E50E94C04608E08991A3
:108E60000E94C0460150D9F703C08CEC0E94C04656
:108E7000812F0E94C046DF91CF911F910F910895DD
:108E80000F931F93CF93DF93FB01DA01E801408139
:108E900050E0718160E0462B572B803171F4BA01AC
:108EA0006E7F13E0660F771F1A95E1F796814CE00D
:108EB00050E0491B5109460F571F57FF06C091E06C
:108EC0009C93509541955F4F01C01C92883289F464
:108ED000848190E0BC01607670706036710549F065
:108EE00086FF02C04E7F05C085FF02C04C7F01C0D7
:108EF000487FCA0154E0969587955A95E1F7F901A4
:108F000080834F70488380E0DF91CF911F910F9154
:108F100008950F931F93CF93DF938C01EB01F8011A
:108F20008081BE010E94D546F801808381508D3F2B
:108F300028F48881883211F0803189F7DF91CF9150
:108F40001F910F9108951F93CF93DF93EC010E941F
:108F50001D4684EBBE010E94214781E00E947D46B0
:108F6000182F0E941D4681E0112309F480E0DF9153
:108F7000CF911F9108951F93CF93DF93182FEB018B
:108F80000E941D460E94EC45882349F084E4BE01FE
:108F90000E942147113029F00E94F54502C082E06D
:108FA00001C080E0DF91CF911F9108956F927F9271
:108FB0008F929F92AF92BF92CF92DF92EF92FF92E9
:108FC0000F931F93DF93CF93CDB7DEB729970FB6DB
:108FD000F894DEBF0FBECDBF7C014B013A015901B1
:108FE0000E941D468EEBB7010E9421478E010F5F44
:108FF0001F4F8AE0C82ED12CCC0EDD1E0E94D14618
:10900000F80181938F01EC15FD05C1F78E010F5F0B
:109010001F4FC80169E070E00E946662882351F426
:10902000F7018081B801A401930185010E944047A6
:1090300080E001C083E029960FB6F894DEBF0FBE32
:10904000CDBFCF91DF911F910F91FF90EF90DF90F7
:10905000CF90BF90AF909F908F907F906F9008952A
:109060007F928F929F92AF92BF92CF92DF92EF92B8
:10907000FF920F931F93DF93CF93CDB7DEB729975E
:109080000FB6F894DEBF0FBECDBF782E5B014A014C
:1090900079018EEB60E070E00E9421478E010F5F46
:1090A0001F4F9AE0C92ED12CCC0EDD1E0E94D14656
:1090B000F80181938F01EC15FD05C1F78E010F5F5B
:1090C0001F4FC80169E070E00E946662882349F47E
:1090D000872DB801A501940187010E94404780E0D7
:1090E00001C083E029960FB6F894DEBF0FBECDBF56
:1090F000CF91DF911F910F91FF90EF90DF90CF9074
:10910000BF90AF909F908F907F9008950F931F9383
:10911000DF93CF93CDB7DEB728970FB6F894DEBFB5
:109120000FBECDBF182F062FDE011196E8E9F5E03E
:1091300088E001900D928150E1F7242F332727FD1D
:10914000309541E752E0249FC001259F900D349F48
:10915000900D112464E670E00E940C77AB0164E688
:10916000069FB0011124460F571FFE013196CE0114
:109170000996619170E02617370719F44F5F5F4F2A
:1091800003C0E817F907A9F7112319F05095419585
:109190005F4FCA0128960FB6F894DEBF0FBECDBF51
:1091A000CF91DF911F910F9108950F931F93DF933C
:1091B000CF93CDB7DEB72B970FB6F894DEBF0FBEB7
:1091C000CDBF182F092F885F612F792F0E94BB47D1
:1091D000882309F049C066E471E48FE090E00E94C2
:1091E0004249812F902FBE016F5F7F4FAE014E5FCE
:1091F0005F4F9E012D5F3F4F0E94D6478823A1F508
:10920000DE011496E0E9F5E088E001900D928150CE
:10921000E1F74B81642F70E021E732E0629FC001EB
:10922000639F900D729F900D112464E670E00E9480
:109230000C779A8184E6989FC0011124680F791FEA
:10924000FE013496CE010C962191421719F46F5FFE
:109250007F4F03C0E817F907B9F78981882331F0F8
:10926000709561957F4F02C064E371E2CB012B964C
:109270000FB6F894DEBF0FBECDBFCF91DF911F9127
:109280000F910895DC01CB0181159105A105B10570
:1092900029F081509040A040B040D9F70895109235
:1092A000B90080E28093B800089594EA9093BC00DE
:1092B00020EA36E841E050E005C02150304040400F
:1092C0005040F1F09091BC0097FFF7CF1DC0903156
:1092D000B9F48093BB0084E88093BC0080EA96E8F0
:1092E000A1E0B0E004C00197A109B10959F02091B3
:1092F000BC0027FFF8CF0EC081E0903421F40FC0EE
:1093000081E0089581E008959091B900987F9830A8
:10931000F1F6DFCF9091B900987F983169F780E03E
:10932000089544EA34E824E94093BC009091BC00DD
:1093300097FFFCCF9091B900987F983011F0903151
:1093400099F78093BB003093BC009091BC0097FFCD
:10935000FCCF9091B900987F903211F0983539F494
:109360002093BC009091BC0094FDFCCFDDCF08950C
:109370000E945549089584E98093BC008091BC0007
:1093800084FDFCCF08958093BB0084E88093BC00EB
:109390008091BC0087FFFCCF9091B900987F81E05D
:1093A000983209F480E0089584EC8093BC008091A9
:1093B000BC0087FFFCCF8091BB00089584E88093B8
:1093C000BC008091BC0087FFFCCF8091BB0008955A
:1093D000E82FF92F80E1919190933F018150D9F7C7
:1093E00080913C018F7D80933C0180913C01877F7F
:1093F00080933C01862F972FFC0180E191919093FF
:109400003E018150D9F780913C01806880933C01F6
:1094100080913D0180FFFCCF4051504080913C0144
:10942000806280933C0180913C01877F80933C0166
:1094300014C0862F972FFC0180E1919190933E01FB
:109440008150D9F780913C01806880933C018091E4
:109450003D0180FFFCCF40515040141615064CF3DF
:10946000822F932FFC0180E190913E0191938150D6
:10947000D9F781E090E008950F931F93CF93DF9386
:109480008C018CE70E9491498CE70E94C349C0E09F
:10949000D0E0F80181918F010E94C3492196C0312B
:1094A000D105B9F70E94BB49DF91CF911F910F9170
:1094B0000895813039F48CE790E060E070E040E09E
:1094C00050E006C08CE790E060E070E040EC50E0D7
:1094D0000E9406110895813039F48CE790E060E035
:1094E00070E04EE050E006C08CE790E060E070E095
:1094F00048E050E00E94061108958CE790E060E09B
:1095000070E041E050E00E9406116AE67AE080E0F7
:1095100090E00E94424908958CE790E060E070E09E
:1095200048E350E00E9406118CE790E060E070E0B4
:1095300049E350E00E9406118CE790E060E070E0A3
:1095400044E150E00E9406118CE790E060E070E09A
:1095500048E750E00E9406118CE790E060E070E080
:109560004EE550E00E9406118CE790E060E070E06C
:109570004DE650E00E9406116CE17AE186E090E051
:109580000E9442498CE790E060E070E04CE050E0DF
:109590000E9406118CE790E060E070E041E050E04E
:1095A0000E9406118CE790E060E070E046E050E039
:1095B0000E9406116AE67AE080E090E00E9442494B
:1095C0000895DF93CF93CDB7DEB7A2970FB6F89487
:1095D000DEBF0FBECDBFDE011196E0EAF5E081E10E
:1095E00001900D928150E1F7DE015296E1EBF5E03A
:1095F00081E101900D928150E1F70E948C4ACE01E9
:1096000001960E943C4A82E00E94594A6AE67AE04A
:1096100080E090E00E944249CE0142960E943C4A7E
:1096200060E17EEA88E290E00E94424980E00E9488
:109630006B4A60E17EEA88E290E00E94424981E064
:109640000E946B4AA2960FB6F894DEBF0FBECDBF44
:10965000CF91DF910895E6E4F1E08081208190814F
:109660003081829586958695837022952F70822B06
:10967000832B92959F70892B0895DF92EF92FF9232
:109680000F931F93DF93CF9300D0CDB7DEB780E069
:109690006CE046E00E94134F89E18093C400109271
:1096A000C50082E08093C00080E00E94BD4F0E9410
:1096B000424E84B784B784B784B784B7E6E8FDE246
:1096C00022E432E4318320833A968DB79EB70A971D
:1096D000E817F907B8F300D000D086EC9EE0ADB7EC
:1096E000BEB712969C938E93119782EC95E01496D8
:1096F0009C938E9313970E94B17A0F900F900F90C6
:109700000F900E947F5E0E944D3D8DE695E060E0E7
:1097100070E00E94013E0E947E41E0910D06F091B2
:109720000E0609950E942B4B90E00E94BD5ECE0173
:1097300001960E94704D882359F000D086EA9EE081
:10974000EDB7FEB7928381830E94B17A0F900F909C
:109750008E010F5F1F4FC8010E94AE3B0E947A4DE1
:109760007C010E947F4DBC01C701A8010E94CA5222
:109770000E94D84C0E94AF520E94844D0E943754E0
:1097800000D089E99EE0ADB7BEB712969C938E9348
:1097900011970E94B17A00D0EDB7FEB7319605E976
:1097A0001EE0ADB7BEB712961C930E9311978A8137
:1097B000828313820E94B17AEDB7FEB73196ADB7BE
:1097C000BEB712961C930E931197898182831382E0
:1097D0000E94B17A0F900F9083E99EE0EDB7FEB73B
:1097E000928381830E94B17A0F900F900E94C35E92
:1097F000E0919006F09191060995E0917706F0913D
:1098000078060995E0913906F0913A060995E090BD
:109810007506F090760600918E0610918F060E94D4
:10982000AC52D82E0E943F542DB73EB72A5030403C
:109830000FB6F8943EBF0FBE2DBFEDB7FEB7319601
:1098400028E73EE0ADB7BEB712963C932E93119732
:10985000F382E28215830483D68217828087118681
:109860000E94B17AE0919A06F0919B062DB73EB71F
:10987000265F3F4F0FB6F8943EBF0FBE2DBF309707
:10988000D1F00995BC0100D000D085E69EE0ADB7CF
:10989000BEB712969C938E93119780E890E00E9439
:1098A000F876EDB7FEB7748363830E94B17A0F90A8
:1098B0000F900F900F9000D083E69EE0ADB7BEB73B
:1098C00012969C938E9311970E94B17A0F900F90ED
:1098D00089EB96E060E070E00E94013E8BE395E04A
:1098E0000E94695D00D08BE59EE0EDB7FEB79283E4
:1098F00081830E94B17A0F900F900F900F90CF91BB
:10990000DF911F910F91FF90EF90DF900895EF92FC
:10991000FF920F931F9380E8809361001092610083
:109920000E943D4B0E945D3D0E94DE4F80910625C6
:1099300090910725009729F0019790930725809330
:109940000625E0900825F090092500910A25109140
:109950000B250E947F4EE616F7060807190711F33C
:109960000E947F4E609308257093092580930A25F5
:1099700090930B25D7CF00D000D000D0EDB7FEB725
:10998000319625E53EE0ADB7BEB712963C932E93D7
:10999000119793838283758364830E94B17A8DB714
:1099A0009EB706960FB6F8949EBF0FBE8DBF089562
:1099B0000F931F93DF93CF93CDB7DEB7A2970FB668
:1099C000F894DEBF0FBECDBF8CE490E00E94FB7B1D
:1099D00089839A83982F9B50903108F08A839A81CB
:1099E0009095891709F470C000D081E09FE0ADB771
:1099F000BEB712969C938E9311970E94B17A8E01F6
:109A00000D5F1F4F0F900F90D80180E090E0FC0198
:109A1000EF51F14FE491ED93019688309105B9F73C
:109A2000F894CE0103966AE270E048E050E00E94AC
:109A3000017CD80180E090E0FC01E751F14FE49116
:109A4000ED9301968E309105B9F7CE01039662E34E
:109A500070E04EE050E00E94017C80E090E0FC016C
:109A6000E950F14FE491D801ED938D0101968A30D0
:109A70009105A9F7CE01039660E470E04AE050E05A
:109A80000E94017C8EE490E06DEC7BEA0E94197CE0
:109A900080E590E060E070E00E94197C82E590E053
:109AA00060E00E940B7C8AE490E060E070E00E943D
:109AB000197C8AE1898385EE8A8369817A818CE4C5
:109AC00090E00E94197C78948981A2960FB6F89450
:109AD000DEBF0FBECDBFCF91DF911F910F910895D3
:109AE000F8946AE270E042E050E00E94E37B7894F0
:109AF00080E008958EE490E00E94FB7B089580E56D
:109B000090E00E94FB7B089582E590E00E94F37B49
:109B100008952091142530911525409116255091D6
:109B2000172590E0A0E0B0E0280F391F4A1F5B1F07
:109B3000209314253093152540931625509317250F
:109B40002091102530911125409112255091132517
:109B5000280F391F4A1F5B1F2093102530931125B2
:109B600040931225509313252091B4262223A1F06F
:109B700020910C2530910D2540910E2550910F25F7
:109B8000280F391F4A1F5B1F20930C2530930D258A
:109B900040930E2550930F2508951F920F920FB6F4
:109BA0000F920BB60F9211242F933F934F935F9315
:109BB0006F937F938F939F93AF93BF93EF93FF9395
:109BC0008091FA0F9091FB0F01969093FB0F809379
:109BD000FA0F8091FC0F8F5F8093FC0F8091FC0F38
:109BE0008038A9F41092FC0F8091142590911525CE
:109BF000A0911625B09117250196A11DB11D809346
:109C0000142590931525A0931625B09317258091C0
:109C1000B4268823F1F08091FD0F8F5F8093FD0FB4
:109C20008091FD0F8038A9F41092FD0F80910C25D2
:109C300090910D25A0910E25B0910F250196A11DA3
:109C4000B11D80930C2590930D25A0930E25B09304
:109C50000F250E94C840009711F00E94C83FFF9155
:109C6000EF91BF91AF919F918F917F916F915F9194
:109C70004F913F912F910F900BBE0F900FBE0F9001
:109C80001F901895F8941092B60016BC83EF87BD0C
:109C900082E084BD94E095BD95B395BB80936E0042
:109CA000789408952091FA0F3091FB0F8091FA0F6C
:109CB0009091FB0F28173907A9F7C901089507C02C
:109CC00022E330E0000021503040E1F70197009797
:109CD000B9F708950F931F93CF93DF938C010E94E0
:109CE000524EEC010E94524E8C1B9D0B8017910727
:109CF000C8F3DF91CF911F910F910895089520919E
:109D000014253091152540911625509117258091E5
:109D1000142590911525A0911625B0911725281787
:109D200039074A075B0759F7B901CA0108951F921D
:109D30000F920FB60F9211241092E6050F900FBEEE
:109D40000F901F9018951F920F920FB60F920BB69F
:109D50000F9211242F933F934F935F936F937F93B1
:109D60008F939F93AF93BF93EF93FF93E091DC05A5
:109D7000F091DD058081E091E705F091E8053097ED
:109D800009F00995FF91EF91BF91AF919F918F914C
:109D90007F916F915F914F913F912F910F900BBEEB
:109DA0000F900FBE0F901F9018951F920F920FB635
:109DB0000F9211241092F3050F900FBE0F901F9079
:109DC00018951F920F920FB60F920BB60F92112497
:109DD0002F933F934F935F936F937F938F939F93B3
:109DE000AF93BF93EF93FF93E091E905F091EA05FC
:109DF0008081E091F405F091F505309709F009951F
:109E0000FF91EF91BF91AF919F918F917F916F9152
:109E10005F914F913F912F910F900BBE0F900FBE0E
:109E20000F901F90189590E02DE030E0829FF00198
:109E3000839FF00D929FF00D1124E452FA4FA281FE
:109E4000B3811C92A481B5816C93A681B78188ED02
:109E50008C93A085B1854C93128614861386089541
:109E600090E02DE030E0829FF001839FF00D929F03
:109E7000F00D1124E452FA4F81E08287A081B18174
:109E80006C933A9680818823E9F708951F93182FE1
:109E90008A3031F48091FE0F6DE00E94304F02C095
:109EA0008D3029F08091FE0F612F0E94304F80E0AD
:109EB00090E01F910895EF92FF921F93CF93DF934D
:109EC000182FE62EE7017E01F72EE7010CC08A303D
:109ED00021F4812F6DE00E94304F69916D3019F0AF
:109EE000812F0E94304F8881882389F7DF91CF919D
:109EF0001F91FF90EF9008950F931F93DF93CF93DF
:109F0000CDB7DEB7FE013A960FEF1FE0C80160E45F
:109F100070E0488559859F010E944D7B8F81B80173
:109F20000E945B4FCF91DF911F910F9108951F9376
:109F3000CF93DF93182FEB0104C0812F0E94304F85
:109F40002196FE0164916623C1F7DF91CF911F91A5
:109F5000089590E02DE030E0829FF001839FF00DA6
:109F6000929FF00D1124E452FA4F7487638708958D
:109F7000682F80E00E94304F08958093FE0F8EEC92
:109F800095E09093812D8093802D089584B7877FED
:109F900084BF88E10FB6F89480936000109260004F
:109FA0000FBE08952FE088E190E00FB6F894A895D1
:109FB000809360000FBE209360000895A8950895D7
:109FC00088E10FB6F89480936000109260000FBE95
:109FD0000895F89428E088E190E00FB6F894A895E9
:109FE000809360000FBE20936000FFCF80912725F3
:109FF00090E0FC01EE0FFF1F9695982F882797950C
:10A000008795E80FF91FE85DFA4D10820895809159
:10A010001F2580911F2590E008958091390181FDD1
:10A020000CC081E491E06FE140E00E94E055813096
:10A0300039F021E030E0813129F020E030E002C049
:10A0400021E030E0C90108958091390181FD12C0FD
:10A0500081E491E06FE140E00E94E055982F81514A
:10A06000823050F09F3141F0913041F081E09230E8
:10A0700031F402C081E0089580E0089580E0089501
:10A080000E9424508823E1F3089581E491E06FE178
:10A0900040E00E94E0550895E9E3F1E0808180818D
:10A0A0008D7F80838DE090E00197F1F782E491E06D
:10A0B0006FE140E023E00E94EA5583E090E00197E1
:10A0C000F1F708950E9440501092B4260E944C501F
:10A0D00080913901826080933901809137278823EC
:10A0E000E9F180919400909195002091482730915A
:10A0F000492782179307A0F4809114279091152780
:10A10000A0911627B09117278C57914EAF4FBF4F94
:10A110008093142790931527A0931627B0931727A1
:10A120008091940090919500821B930BA0E0B0E089
:10A130002091142730911527409116275091172709
:10A14000820F931FA41FB51F809314279093152788
:10A15000A0931627B093172710923727809139279D
:10A160008823E9F1809194009091950020914C27EB
:10A1700030914D2782179307A0F480911C2790916E
:10A180001D27A0911E27B0911F278C57914EAF4FCE
:10A19000BF4F80931C2790931D27A0931E27B09339
:10A1A0001F278091940090919500821B930BA0E053
:10A1B000B0E020911C2730911D2740911E2750911F
:10A1C0001F27820F931FA41FB51F80931C279093F6
:10A1D0001D27A0931E27B0931F271092392708959B
:10A1E0008091B426882381F080913F10882321F448
:10A1F0000E942450882331F481E08093C21021E032
:10A2000030E004C00E94625020E030E0C9010895AF
:10A210000F931F93182F883049F0863039F089301A
:10A2200029F0863119F0893109F041C08091390156
:10A2300081FD40C00E9440500E944550082F1817D1
:10A2400009F43BC0183019F40E944C5029C0193150
:10A2500041F48631A9F482E491E06FE140E029E025
:10A2600009C0163169F4893159F482E491E06FE153
:10A2700040E026E00E94EA55E3E0F0E03197F1F794
:10A2800082E491E06FE140E0212F0E94EA5508301E
:10A2900019F4E9E6F1E002C0E3E0F0E03197F1F70C
:10A2A0000E944550811749F023E430E008C022E4C1
:10A2B00030E005C024E430E002C020E430E0C90111
:10A2C0001F910F9108958091940090919500909323
:10A2D0004D2780934C2721E0209339278091390125
:10A2E00081FF15C02093B326809194009091950032
:10A2F00090934927809348272093372780913901ED
:10A300008D7F809339018091B3268823E1F786E120
:10A310000E94085181E08093B42608958091B4266C
:10A32000882351F480913F10882321F081E08093AD
:10A33000C11002C00E94635181E090E008951F9314
:10A34000DF93CF930F92CDB7DEB78FB7898380911C
:10A350003F10882331F5F8948091B426882351F07A
:10A360008091390181FD1BC00E9424508823B9F0DF
:10A3700080E003C00E948E5181E0909147019E30A1
:10A3800010F010E001C01FEF882311F00E94F05080
:10A3900016FF05C089818FBF21E030E004C08981AC
:10A3A0008FBF20E030E0C9010F90CF91DF911F9166
:10A3B00008958091C110882321F00E94635110926A
:10A3C000C1108091C210882321F00E946250109227
:10A3D000C21010923F100895EF92FF92CF93DF9337
:10A3E000B82FA92FF62FE72F81E080933F102091FF
:10A3F000F8263091F9264091FA265091FB262F5FDE
:10A400003F4F4F4F5F4F2093F8263093F9264093EC
:10A41000FA265093FB26862F8E5F87FF0CC0809113
:10A42000B1269091B22601969093B2268093B126E0
:10A43000CFEFDFEF0BC020E430E1C9016B2F7A2FA3
:10A440004F2F5E2F0E94117AC0E0D0E00E94D951B8
:10A45000CE01DF91CF91FF90EF9008959091390157
:10A4600091FD0AC0282F803108F02FE085E491E0AB
:10A470006FE040E00E94EA5508958093C41008956B
:10A480000E9445508250813130F4E82FF0E0EF5DBA
:10A49000F94F8081089581E0089508958FEF8093AA
:10A4A0004E018CE691E060EF44E022E00E94EA5524
:10A4B0008CE290E06EE041E025E00E94EA5580E801
:10A4C00080936F018091460180936D0184E491E057
:10A4D00060E245E021E00E94EA550895CF93DF93C2
:10A4E000CDEFD3E0CE010197F1F70E94D65510923F
:10A4F00028251092AA2510922C261092272510921A
:10A500002625E9E3F1E080818E7F808380818D7F45
:10A5100080838DE090E00197F1F7808181608083F6
:10A5200082E491E06FE140E023E00E94EA55219748
:10A53000F1F780915D0180915E010E944E5283E0AF
:10A5400096E060E070E00E94013E0E94635181E06D
:10A5500090E0DF91CF9108958091C3100895DF932B
:10A56000CF930F92CDB7DEB789830E9440502981E7
:10A570002093C31088E491E06FE140E00E94EA5527
:10A580000F90CF91DF9108950E94AF5286E00E9414
:10A590000851089580936201909363016093600174
:10A5A000709361014115510531F1FA018191809358
:10A5B0006B01DA0111968C9180936A01DF0111968B
:10A5C000818180936901FD01319611968C91809370
:10A5D0006801DF011196818180936701FD01319649
:10A5E00011968C911197809366018181809365010A
:10A5F000828180936401089583E096E00E94243E66
:10A6000081E080931F25809120259091212501963E
:10A61000909321258093202581E090E00895EF928A
:10A62000FF92CF93DF9350912725252F30E0F9013A
:10A63000EE0FFF1F3695322F222737952795E20F11
:10A64000F31FE85DFA4D4081442309F4CEC0209108
:10A65000390121FDCAC02091B426222309F4C5C0C6
:10A6600047FF16C00E94F64F8091E8269091E92698
:10A67000A091EA26B091EB260196A11DB11D809311
:10A68000E8269093E926A093EA26B093EB26ADC086
:10A690004330B0F40E94F64F8091E4269091E52675
:10A6A000A091E626B091E7260196A11DB11D8093E9
:10A6B000E4269093E526A093E626B093E72695C07E
:10A6C000C42FD0E022976C177D07B0F40E94F64F9C
:10A6D0008091E0269091E126A091E226B091E326B8
:10A6E0000196A11DB11D8093E0269093E126A093D1
:10A6F000E226B093E32679C0652F70E09B01220F1C
:10A70000331F7695762F662777956795260F371F27
:10A71000275D3A4DB90150E00E94117A209127251A
:10A72000822F90E0FC01EE0FFF1F9695982F88274F
:10A7300097958795E80FF91FE855FA4D808180932A
:10A740001825822F90E0FC01EE0FFF1F9695982FA1
:10A75000882797958795E80FF91FE85DFA4D1082D5
:10A760002F5F20932725233010F01092272580910A
:10A77000272590E0FC01EE0FFF1F9695982F882764
:10A7800097958795E80FF91FE85DFA4D808188233A
:10A7900011F00E94FC52609147016093192580914D
:10A7A0001E25882311F0681710F460931E2584E09D
:10A7B00070E00E94C0456091182583E070E00E941F
:10A7C000C0458091FC269091FD26A091FE26B09177
:10A7D000FF260196A11DB11D8093FC269093FD26B6
:10A7E000A093FE26B093FF2602C0C0E0D0E0CE01C9
:10A7F000DF91CF91FF90EF900895CF93DF93EC011D
:10A8000088819981009729F024E08B3F920739F5E0
:10A8100005C08BEF94E09983888325C0623819F5D1
:10A8200010921F250E943A450E94974460E870E00C
:10A830000E940F531816190644F40E949244E091A6
:10A840009406F09195060995E4CF80911C2590918E
:10A850001D25019690931D2580931C25DACF198222
:10A86000188283E001C081E0DF91CF91089591E0EB
:10A8700090933F100E942E520E94D95108958091CA
:10A88000390181FD07C085E491E06FE040E00E945E
:10A89000E055089580E10895CF92DF92EF92FF9204
:10A8A0000F931F93CF93DF93182F21E020933F1036
:10A8B0000091B4268091390181FF16C080919400E7
:10A8C00090919500909349278093482720933727AC
:10A8D0002093B326809139018D7F80933901809137
:10A8E000B3268823E1F700E00E9440508091B4260F
:10A8F000882309F441C0809139278823E9F1209108
:10A9000094003091950080914C2790914D27281705
:10A910003907A0F420911C2730911D2740911E2754
:10A9200050911F272C57314E4F4F5F4F20931C27BC
:10A9300030931D2740931E2750931F27209194008A
:10A9400030919500281B390B40E050E0C0901C2747
:10A95000D0901D27E0901E27F0901F272C0D3D1D45
:10A960004E1D5F1D20931C2730931D2740931E27EB
:10A9700050931F271092392789E10E94085186E0E1
:10A980000E94CB45009751F00E943F54C82F86E0AB
:10A990000E94CB4581500E942E5202C0C0E0D0E000
:10A9A000809194009091950090934B2780934A2733
:10A9B00081E080933827F8948091390182608093F8
:10A9C0003901809139018D7F80933901612F6E5F4C
:10A9D00080E490E10E941B5678948091AE2690917D
:10A9E000AF2601969093AF268093AE260E944050EA
:10A9F00082E491E060EE45E00E94E055182F86E089
:10AA00000E94CB45009719F08C2F0E942E520023F4
:10AA100019F00E94635102C00E9462508091382751
:10AA20008823E9F1809194009091950040914A2704
:10AA300050914B2784179507A0F480911827909187
:10AA40001927A0911A27B0911B278C57914EAF4F11
:10AA5000BF4F8093182790931927A0931A27B0937C
:10AA60001B272091940030919500241B350B40E06A
:10AA700050E08091182790911927A0911A27B09142
:10AA80001B27280F391F4A1F5B1F2093182730935D
:10AA9000192740931A2750931B271092382780912B
:10AAA000B426882361F08091940090919500909352
:10AAB0004D2780934C2781E08093392707C082E49B
:10AAC00091E06FE140E023E00E94EA550E94D951F5
:10AAD0001130E1F01330A9F48091F0269091F12625
:10AAE000A091F226B091F3260196A11DB11D80938D
:10AAF000F0269093F126A093F226B093F32612E06D
:10AB00000AC0153029F0173031F404C010E003C03A
:10AB100013E001C011E0812F90E0DF91CF911F91F0
:10AB20000F91FF90EF90DF90CF900895CF93DF9338
:10AB3000EB010E94EC519C01009731F4CE010E9480
:10AB40004C549C01009749F08091B1269091B22617
:10AB500001969093B2268093B126C901DF91CF91DF
:10AB600008950F931F938091B426882321F40E94A7
:10AB70008E5111E001C010E00E944550863111F065
:10AB8000813119F40091470109C086E491E06FE139
:10AB900040E00E94E055082F000F080F112311F02C
:10ABA0000E94F050802F1F910F9108951092C610AF
:10ABB0001092C510EFE6F0E08081806280830895F6
:10ABC000FC018081862390E002C0959587954A9587
:10ABD000E2F70895F894FC019081862F80958923EF
:10ABE00030E002C0220F331F4A95E2F72623282BBC
:10ABF000208378940895DC01119620917B01FC015B
:10AC00002083215030E0A9014F575E4FE0E8F1E08A
:10AC100061916D93E417F507D9F7FC01E058FF4FF8
:10AC20002F573E4FD9012C9120838F579F4F21E002
:10AC3000FC0120830895FC0160938001019663501C
:10AC4000860F911DA1E8B1E021912D93E817F90736
:10AC5000D9F708951F920F920FB60F920BB60F926D
:10AC600011242F933F934F935F936F937F938F9311
:10AC70009F93AF93BF93EF93FF938091470180938E
:10AC800019252091262530E0C901880F991F369596
:10AC9000322F222737952795820F931F885D9A4D73
:10ACA0000E94FB55809126258F5F80932625833057
:10ACB00010F0109226250E94FC52FF91EF91BF9157
:10ACC000AF919F918F917F916F915F914F913F9144
:10ACD0002F910F900BBE0F900FBE0F901F901895E5
:10ACE0001F920F920FB60F9211240F900FBE0F906C
:10ACF0001F9018951F920F920FB60F9211240F906C
:10AD00000FBE0F901F9018951F920F920FB60F92C3
:10AD100011240F900FBE0F901F9018951F920F9245
:10AD20000FB60F9211241092B3260F900FBE0F9002
:10AD30001F9018951F920F920FB60F921124109228
:10AD4000B3260F900FBE0F901F9018951F920F9271
:10AD50000FB60F9211248F9381E080931F258F915E
:10AD60000F900FBE0F901F9018951F920F920FB665
:10AD70000F9211241092B3260F900FBE0F901F90C8
:10AD800018951F920F920FB60F9211248F939F93D5
:10AD90008091C5109091C61001969093C610809333
:10ADA000C5109F918F910F900FBE0F901F90189517
:10ADB0000F931F93CF93DF938091BC269091BD2674
:10ADC000A091BE26B091BF260196A11DB11D809312
:10ADD000BC269093BD26A093BE26B093BF260E94AA
:10ADE0008959EC0187EC90E10E94C63E0BC0D80166
:10ADF0001296ED91FC911397309709F00995C801CF
:10AE00000E948C3F082F192F0115110581F72097FB
:10AE100019F0CE010E94363CDF91CF911F910F9126
:10AE200008950E94C35E0E943A450E94935785E7A9
:10AE300096E09093B7268093B6260E94865982E0CA
:10AE400090E060E074E040E05EE12FEF31E00E94CE
:10AE500047590895CF92DF92EF92FF920F931F937D
:10AE6000CF93DF936C01EB018A0187EC90E10E94A4
:10AE7000C63E0CC0D7011496ED91FC911597309702
:10AE800011F0CE010995C7010E948C3FE82EF92EE2
:10AE9000E114F10479F7C601BE01A8010E943E3C0D
:10AEA000DF91CF911F910F91FF90EF90DF90CF90A6
:10AEB0000895BC0187EC90E10E944D3F0895BC01CC
:10AEC00087EC90E10E94143F0895CF93DF93EC014B
:10AED0008091B8269091B926A091BA26B091BB2650
:10AEE0000196A11DB11D8093B8269093B926A09319
:10AEF000BA26B093BB26CE010E94A059009769F0F4
:10AF00000E94B444E0917906F0917A068AE297E5CE
:10AF1000BE01099521E030E002C020E030E0C90127
:10AF2000DF91CF91089589EC90E10E94C23E08958F
:10AF30000F93CF93DF93EC017B836A8318865F8343
:10AF40004E8389EC90E1BE010E944D3FE091CB1011
:10AF5000F091CC10309749F04C815D818A819B81C2
:10AF6000688520E030E001E00995DF91CF910F91F5
:10AF70000895BC0189EC90E10E94143F08950F935D
:10AF8000DC0118961C921897E091CB10F091CC1030
:10AF9000309759F012968D919C91139760E040E0A4
:10AFA00050E020E030E000E009950F9108950F9304
:10AFB000DC01AB0114962D913C91159781E0189618
:10AFC0008C93189715967C936E931497E091CB1001
:10AFD000F091CC10309739F012968D919C91139787
:10AFE00061E000E009950F9108950F93DC01E09175
:10AFF000CB10F091CC10309769F014962D913C91C4
:10B00000159712968D919C91139718966C91A901A2
:10B0100001E009950F910895E091CD10F091CE10C7
:10B02000309709F0099508959093CE108093CD1034
:10B0300008959093CC108093CB10089589EC90E103
:10B040000E94C63E0895EF92FF920F931F93CF93F5
:10B05000DF938C01EB017A0189EC90E10E94C63EFE
:10B0600015C0DC0112962D913C9113972C173D07CA
:10B0700059F41696ED91FC911797309761F0B8014D
:10B08000AE019701099507C00E948C3F282F392FE8
:10B09000C901009731F7DF91CF911F910F91FF9078
:10B0A000EF9008950895AF92BF92CF92DF92EF9202
:10B0B000FF920F931F93DF93CF9300D0CDB7DEB7EE
:10B0C0005B010E949744FC01008111811A8309836E
:10B0D0000C30110518F4EE24FF242EC000D000D04F
:10B0E0008DE396E0EDB7FEB79283818314830383EB
:10B0F0000E949F7A0F900F900F900F9020C00E9497
:10B100009744F701EE0FFF1FEE0FFF1FE80FF91F27
:10B11000C280D3800E9497440894E11CF11CF7017F
:10B12000EE0FFF1FEE0FFF1FE80FF91F4081518147
:10B13000C501B6010E942358E016F10600F30F90F6
:10B140000F90CF91DF911F910F91FF90EF90DF90C3
:10B15000CF90BF90AF900895CF93DF93CAEED0E128
:10B160006091001170910111CE014EED58E520E083
:10B1700030E00E948B410E94C05E6091001170918E
:10B1800001110E94F876BC01CE01409743EF58E5CB
:10B1900020E030E00E948B41DF91CF9108950F9322
:10B1A000013051F48091FA109091FB1090930111AD
:10B1B000809300110E94AC580F9108958091001166
:10B1C000909101112091FE103091FF10880F991F6E
:10B1D0002817390708F4C9019093011180930011D1
:10B1E0000E94AC580895EF92FF92CF93DF930E9494
:10B1F0003A450E949744E82EE7017E01F92EE701C7
:10B20000198218820E941E5826C028813981F901AE
:10B21000EE0FFF1FEE0FFF1FEC0FFD1FDC0112965C
:10B220004D915C911397538342832F5F3F4FF901F8
:10B23000EE0FFF1FEE0FFF1FEC0FFD1F14964D9139
:10B240005C91159751834083398328830E948C3FFA
:10B25000282F392FC901009721F0FC0120852223D6
:10B26000A1F688819981880F991F880F991F0296EE
:10B270000E94924488819981009721F08FEC90E19F
:10B280000E94093CDF91CF91FF90EF900895EF92DB
:10B29000FF920F931F93CF93DF93FC018B017A01F1
:10B2A000E9018FEC90E1BF014AE556E00E94EB3BDB
:10B2B0001093FB100093FA10F092FD10E092FC1036
:10B2C000D093FF10C093FE108FEC98E50E941958A0
:10B2D000DF91CF911F910F91FF90EF900895CF9341
:10B2E000DF93CAEED0E1CE010E941242CE01409718
:10B2F0000E941242CE014B970E94063CDF91CF91F3
:10B300000895809100119091011108950E944A3C86
:10B310000895EF92FF92CF93DF93E0915E06F09154
:10B320005F060995EC01009729F06A817B8181E035
:10B330000E94C045CE01DF91CF91FF90EF9008951C
:10B340000F931F93CF93DF938C01E0916006F091F0
:10B3500061060995EC01F8016281738181E00E9428
:10B36000C04521E030E0209711F420E030E0C90131
:10B37000DF91CF911F910F910895E0916206F091B6
:10B38000630609950895FC0120E030E004C0818146
:10B39000280F311D329680818823C9F7C90108958D
:10B3A000FC01818190E0308120E0822B932B02C050
:10B3B000880F991F6A95E2F7892F9927FA01EC59AE
:10B3C000F94F208130E08223932328E030E0241BD2
:10B3D000350B02C0969587952A95E2F708956F92EE
:10B3E0007F928F929F92AF92BF92CF92DF92EF9215
:10B3F000FF920F931F93CF93DF936C017B015A0150
:10B4000089012830310544F4CB01BA01A9010E9419
:10B41000D059F601808341C0390133E075946794B7
:10B420003A95E1F74115510521F04C01C0E0D0E01B
:10B4300016C0DB01FC01C0E0D0E08D918193219624
:10B44000C615D705D4F3A8014770507041155105B2
:10B4500021F1C7018C0F9D1F60E070E019C0C7018A
:10B460008C0F9D1FB50148E050E00E94D059F401B7
:10B4700081934F012196C615D7058CF3A80147701B
:10B4800050704115510549F0C7018C0F9D1FB50142
:10B490000E94D059CC0DDD1D8883DF91CF911F9183
:10B4A0000F91FF90EF90DF90CF90BF90AF909F9063
:10B4B0008F907F906F9008954F925F926F927F92DE
:10B4C0008F929F92AF92BF92CF92DF92EF92FF92B4
:10B4D0000F931F93DF93CF9300D000D0CDB7DEB78B
:10B4E0000E949744E82E092F82E090E00E94734466
:10B4F000009709F464C0EE2DF02F918180E0208147
:10B50000820F911D0E945E3C7C01009709F459C096
:10B510000E9497443C01F7014681242F30E02770B8
:10B52000307081E090E02115310511F480E090E069
:10B53000469546954695840F911D0E947344009749
:10B54000F1F1F70104811581CC24DD2453E0452E6F
:10B55000512C4C0E5D1E4E010894811C911C2AC07A
:10B56000F801A180BB24B60143E0759567954A9523
:10B57000E1F7660D771DA60147705070883150F0D5
:10B58000C40195010E94EF59F8018081B4010E9425
:10B59000D4450CC01C821B82C20195010E94EF5948
:10B5A0006B817C81F80180810E94C045CA0CDB1C44
:10B5B0000E5F1F4FF8018081882391F602C0EE24B0
:10B5C000FF24C7010F900F900F900F90CF91DF9144
:10B5D0001F910F91FF90EF90DF90CF90BF90AF90B1
:10B5E0009F908F907F906F905F904F900895FC0197
:10B5F00050E080E190E0861B970B821B930B02C00A
:10B60000440F551F8A95E2F78081852B80838181C5
:10B61000842B818308956F927F928F929F92AF9235
:10B62000BF92CF92DF92EF92FF920F931F93CF932F
:10B63000DF938C015B016A0179012830310524F424
:10B64000C801FA01408156C0390163E075946794DE
:10B650006A95E1F7A114B10421F04A01C0E0D0E0FD
:10B6600021C0DA01F80180E090E02D91219301964C
:10B6700086159705D4F39701277030702115310591
:10B68000D9F1F601E80FF91F408150E068E070E061
:10B69000621B730B02C0559547956A95E2F7800FC0
:10B6A000911F26C0F40141914F01C8018C0F9D1FCD
:10B6B000B50128E030E00E94F75A2196C615D7055B
:10B6C0008CF397012770307021153105A9F0F60130
:10B6D000EC0FFD1F408150E0C5010896821B930BC3
:10B6E00002C0559547958A95E2F7C8018C0F9D1FBA
:10B6F00060E070E00E94F75ADF91CF911F910F91A7
:10B70000FF90EF90DF90CF90BF90AF909F908F9081
:10B710007F906F9008954F925F926F927F928F9279
:10B720009F92AF92BF92CF92DF92EF92FF920F93D0
:10B730001F93DF93CF9300D0CDB7DEB78C01DC0130
:10B7400016964C911697842F90E08770907021E0A8
:10B7500030E0009711F420E030E04695469546959C
:10B760007901E40EF11CC70102960E94FF44009784
:10B7700009F453C00E949F44FC01D80112968C9199
:10B780001297808313968C9181830E949F44F2E0EC
:10B790006F2E712C680E791EC30160E070E0A70166
:10B7A0000E941A7AF801C480D58000E010E02E01D2
:10B7B0000894411C511C2AC0D60111968C901197F7
:10B7C00099247801E3E0F594E794EA95E1F7E60C33
:10B7D000F71C77E0A72EB12CA022B122883130F0DF
:10B7E0000E94DE45AC01C701B50107C00E94CB45F0
:10B7F0009A838983C701B501A20194010E940B5B62
:10B80000080D191DE2E0F0E0CE0EDF1ED6018C918E
:10B81000882391F621E030E002C020E030E0C90149
:10B820000F900F90CF91DF911F910F91FF90EF90AC
:10B83000DF90CF90BF90AF909F908F907F906F9050
:10B840005F904F900895E0919206F09193060995CC
:10B850000895E0913B06F0913C0609950895E0912A
:10B860009606F091970609950895E0919806F09153
:10B8700099060995089580E090E008950895E09173
:10B880001D06F0911E0609950895009731F0E0918C
:10B890001D06F0911E0609950895E0911F06F0918E
:10B8A00020060995089580E090E008950F931F9376
:10B8B000DF93CF93CDB7DEB7E0970FB6F894DEBF36
:10B8C0000FBECDBF0E94E9448C010E949744602FB7
:10B8D000AE014F5F5F4F0E948964882309F445C021
:10B8E00088A99801281B3109C9010E947344009757
:10B8F000E1F12E81222371F18A859B853BEA8D3C03
:10B90000930721F03FEF8F3F930779F5223041F005
:10B9100088E090E007C0019722912F3F41F00BC0D3
:10B9200082E090E0FE01E80FF91F3C96F4CF181674
:10B9300019068CF30FC089E1BE01645F7F4F0E943E
:10B94000D44589E10E94DE4565EC74E20E949C3B8F
:10B95000009759F088E1BE016A5E7F4F0E94D4458E
:10B96000E0917B06F0917C060995E0960FB6F8947D
:10B97000DEBF0FBECDBFCF91DF911F910F91089514
:10B98000AF92BF92CF92DF92EF92FF920F931F93ED
:10B99000DF93CF93CDB7DEB7E0970FB6F894DEBF55
:10B9A0000FBECDBF6C018B01FE01319680E3DF013C
:10B9B0001D928A95E9F781E089838CE00E94CB454E
:10B9C0008C831D821F828091041189878F5F8093F1
:10B9D000041183E0E82EE8868DEC9BEA9B878A873A
:10B9E00089E10E94DE4565E575E00E949C3B009779
:10B9F00031F082E08E838FEF8C878D8709C089E1DB
:10BA00000E94DE45BC01CE010C960E94933BEE8263
:10BA10008DEC9BEA9D8B8C8BCE01469665EC74E297
:10BA20000E94933B0E9497449FA78EA70E94E944DF
:10BA300088AB7E010894E11CF11CC7010E94806361
:10BA4000A82E90E00E94FF44009741F10E949F447D
:10BA5000BC01C7014A2D0E949E63A0901306B090BE
:10BA600014060E949F447C010E94F344BC01C7015C
:10BA7000F5010995C114D10489F0009721F08130B6
:10BA8000910561F404C0C80160E070E003C0C80122
:10BA900064E070E041E050E0F6010995E0960FB6F1
:10BAA000F894DEBF0FBECDBFCF91DF911F910F91F4
:10BAB000FF90EF90DF90CF90BF90AF9008950E94DD
:10BAC000C05E80930411E0911D06F0911E06099559
:10BAD0000895EF92FF92CF93DF93E82EE7017E0166
:10BAE000F92EE70104C060E070E00E94013E8991F8
:10BAF00099910097C1F7DF91CF91FF90EF90089552
:10BB0000EF92FF92CF93DF93E82EE7017E01F92EAB
:10BB1000E70102C00E94463D899199910097D1F7B3
:10BB2000DF91CF91FF90EF900895CF93DF93EC01D9
:10BB30007B836A830E94524E99838883DF91CF91E1
:10BB40000895FC018081918122813381820F931FAE
:10BB5000918380830895CF93DF93EC010E94524E2E
:10BB600099838883DF91CF910895CF93DF93EC0180
:10BB70000E94524E28813981821B930B019621E04D
:10BB800030E04A815B814817590710F020E030E02F
:10BB9000C901DF91CF910895EF92FF92CF93DF9388
:10BBA000FC01C281D38180819181C80FD91F0E947D
:10BBB000524EC81BD90BCE01DF91CF91FF90EF9071
:10BBC0000895CF93DF93EEE3F7E2C0E0D7E2A2E37C
:10BBD000B7E21192119219921992199219921D922B
:10BBE00087E2E635F807A9F7DF91CF9108950F9323
:10BBF0001F93CF93DF93FC01DC01AE5CB84D8C91B9
:10BC0000882339F10091940010919500EF01CC0F39
:10BC1000DD1FCC0FDD1FC050D94DDF01AA0FBB1FA8
:10BC2000A25CB84D8D919C9111979801281B390BFE
:10BC300040E050E0688179818A819B81260F371F1F
:10BC4000481F591F288339834A835B8311961C93AD
:10BC50000E93EE0FFF1FEE0FFF1FE050F94D6081B6
:10BC6000718182819381DF91CF911F910F9108950E
:10BC700060E070E0CB010895FC01EE0FFF1FEE0FB6
:10BC8000FF1FE050F94D4083518362837383089511
:10BC9000EF92FF920F931F93CF93DF9322E337E24C
:10BCA000C0E0D7E2EEE3F7E2D9018D919D01882350
:10BCB000C9F04091940050919500808191817A0162
:10BCC000E81AF90A00E010E088819981AA81BB8115
:10BCD0008E0D9F1DA01FB11F88839983AA83BB83EC
:10BCE0005183408324963296B7E22E333B07E1F628
:10BCF000DF91CF911F910F91FF90EF9008950E94D7
:10BD0000FD6208950F931F93FC01CB014091051133
:10BD100050910611338322831583048371836083DA
:10BD2000F0930611E09305114115510511F40E949D
:10BD3000176380E090E01F910F91089580910511A5
:10BD4000909106110097C1F0109206111092051102
:10BD5000DC0114966D917C9115971296ED91FC91F2
:10BD600013970995E0910511F0910611309721F094
:10BD7000808191810E94176308950E94E67708955B
:10BD80000E94E17708958CE996E00E943A3E84EAA9
:10BD900096E00E943A3E0895EF92FF92CF93DF9390
:10BDA0000E94A6440097C9F084EA96E00E945A3E99
:10BDB000E82EE7017E01F92EE701209731F10E947C
:10BDC000E944998388830E94E4449B838A83C70162
:10BDD00004960E9412448CAB18C08CE996E00E9435
:10BDE0005A3EEC017E01F92EE701209771F0C70160
:10BDF00002960E94294499838883B7016E547F4F2D
:10BE0000C7018E579F4F0E949645CE01DF91CF917B
:10BE1000FF90EF900895BC016E547F4F8E579F4F57
:10BE20000E9496450895CF93DF93EC018CE996E04C
:10BE3000BE010E94A53E009719F08CE996E009C06A
:10BE400084EA96E0BE010E94A53E009729F084EAAC
:10BE500096E0BE010E94803EDF91CF910895EF925F
:10BE6000FF92CF93DF93EC018CE996E0BE010E9434
:10BE7000A53E009779F068817981CE0102960E94F3
:10BE80006345BE016E547F4FCE018E579F4F0E9477
:10BE9000AB451BC084EA96E0BE010E94A53E009718
:10BEA000A1F00E943A45688179818A819B810E9434
:10BEB00063458CA990E00E94FF440E949F444CA9D6
:10BEC0002496BE0150E00E94117ADF91CF91FF903D
:10BED000EF900895EF92FF92CF93DF93EC018CE9FE
:10BEE00096E0BE010E94A53E009711F022960DC07B
:10BEF00084EA96E0BE010E94A53E009721F00A80E8
:10BF0000DB81C02D02C0C0E0D0E0CE01DF91CF9137
:10BF1000FF90EF900895FC0180819181089570E079
:10BF20006F5B7F4F660F771F680F791FCB010895F6
:10BF3000E62FF0E0EF5BFF4FEE0FFF1FE80FF91F5A
:10BF400080819181089508958DE597E10E94B04028
:10BF5000009721F08DE597E10E949B400895E091C4
:10BF60006A17F0916B17309711F00995089580E0EA
:10BF70000895EF92FF920F931F93CF93DF93EC01FD
:10BF80008A0188819981009731F023E08C309207F3
:10BF900009F006C12BC080E00BC0E82FF0E0EE0FE7
:10BFA000FF1FEE0FFF1FE55BF84E118210828F5FBF
:10BFB000843098F38093651780918C0E90918D0E4C
:10BFC00090935C1780935B170E943F3D80935627A8
:10BFD0008DE597E160E470E00E9485400E9418665C
:10BFE0008CE093E09983888381E0DDC0623009F4BE
:10BFF000B9C0633030F4662309F489C0613081F739
:10C000009CC0673819F0683859F741C0109266171C
:10C010004BE4E42E47E1F42E18C0F70182819381AE
:10C020008017910749F4808191810E945F67F70131
:10C03000118210821382128284E090E0E80EF91ED1
:10C04000809166178F5F80936617809166178430A2
:10C0500020F3E6E6FCE2848D958D8017910719F4B4
:10C06000158E148E118EB0969CE2E63EF90799F774
:10C07000ECEFFCE2818592858017910711F415821F
:10C0800014823D962DE2EE37F207A1F7A9CF87E1A2
:10C090004D35580709F0A4CFCA010E94B04000975F
:10C0A00009F49ECF109266172DC0F0E035E0EE0F38
:10C0B000FF1F3A95E1F7EA59F34D818D8823E9F0A6
:10C0C0008DE597E10E949B408091661790E025E006
:10C0D000880F991F2A95E1F78A59934D9093652C03
:10C0E0008093642C82E00E949367809157279091FF
:10C0F0005827009711F00E94AF5F809166178F5FFD
:10C1000080936617E0916617E43078F269CF4115A5
:10C11000510509F465CF5093652C4093642C83E05E
:10C120000E9493678091572790915827009711F0AC
:10C130000E94AF5F0E94A45F53CF4115510509F4DF
:10C140004FCF5093612C4093602C85E00E94936701
:10C150008091572790915827009709F441CF0E946A
:10C16000AF5F3ECF8091572790915827009709F4F1
:10C1700037CF80916827863031F48091802781FF06
:10C1800002C00E94A45F81E00E94936780915727BC
:10C1900090915827009709F423CF0E94E26120CFA5
:10C1A0001982188283E0DF91CF911F910F91FF9048
:10C1B000EF90089590936B1780936A1708952091DC
:10C1C0008C0E30918D0E60E0EBE4F7E113C04081FE
:10C1D00051814817590761F442815381421753072F
:10C1E00039F460936917118210820E945F67089585
:10C1F00034966F5F643058F360936917089540E098
:10C20000EBE4F7E116C0542F5F5F208131812115E7
:10C21000310569F4409368179183808320918C0ED7
:10C2200030918D0E338322830E947967089534966E
:10C23000452F443040F3409368170895FC018091E6
:10C240008C0E90918D0E958F848F778F668F0895C9
:10C25000FC0180918C0E90918D0E9287818774875E
:10C2600063870895CF93DF93EA010E94DB66FC01A8
:10C27000009741F080918C0E90918D0E928781876E
:10C28000D487C387CF01DF91CF9108950F931F9378
:10C29000DF93CF9300D000D0CDB7DEB78C01AB01D8
:10C2A0008FEF89838A838B838C83CE010196B801BB
:10C2B0000E943261FC01009711F015830483CF01C5
:10C2C0000F900F900F900F90CF91DF911F910F91D2
:10C2D000089589EB96E062E040E050E00E94F23D74
:10C2E00010925827109257270895AC0189EB96E0D9
:10C2F00061E00E94CF3D0895AC0189EB96E060E0DB
:10C300000E94CF3D08950F931F93CF93DF93EA01CF
:10C310000E9451668C01009761F080918C0E909183
:10C320008D0EF801958F848FD78FC68FC8010E941C
:10C330007C61C801DF91CF911F910F910895CF9338
:10C34000DF93A091642CB091652C109719F0ED014A
:10C350006C9605C0C091602CD091612C299680917B
:10C360005F2C86FF22C01092671740E0EBE4F7E1F4
:10C3700016C02081318114968D919C9115972817B4
:10C38000390759F482819381009739F040936717F8
:10C39000998388831B821A8206C034964F5F44308B
:10C3A00040F3409367170E94A45F888199810097AA
:10C3B00031F04A815B81609156270E94F23DDF9106
:10C3C000CF9108950F931F93CF93DF9380916827A8
:10C3D000863009F074C0809157279091582725E046
:10C3E0008030920709F06BC0C4E9D2E0D09358279F
:10C3F000C093572702E00093612714E91093622746
:10C4000010928427109283270E9410668095909541
:10C41000909384278093832710926A27109269272C
:10C420000E94FF658095909590936A278093692775
:10C430000E94AF5FD0935827C0935727009361277E
:10C44000109362279091622C8091632CE92FF82F32
:10C45000DF01A459BD4F8CE692E00D900192019747
:10C46000E1F787E797E26CE672E00E94A3658091AE
:10C470005B278093772780915C2780937827809132
:10C480005D278093792780915E2780937A27109289
:10C490008427109283270E94106680959095909330
:10C4A00084278093832710926A27109269270E941D
:10C4B000FF658095909590936A27809369270E94E5
:10C4C000AF5FDF91CF911F910F910895282F392FE2
:10C4D000F90120E030E080E0A8E112C0419198E04D
:10C4E000542F5827B52FB17050FD8A278695B1304B
:10C4F00009F48068915011F04695F2CF2F5F3F4FBD
:10C500002617370759F708951F920F920FB60F920B
:10C510000BB60F9211242F933F934F935F936F931A
:10C520007F938F939F93AF93BF93EF93FF938091EC
:10C53000940090919500909343278093422781E047
:10C540008093342780917100807D809371000E94D8
:10C550009E5E809134278823E9F180919400909128
:10C560009500209142273091432782179307A0F42A
:10C570008091082790910927A0910A27B0910B2755
:10C580008C57914EAF4FBF4F809308279093092748
:10C59000A0930A27B0930B27809194009091950067
:10C5A000821B930BA0E0B0E020910827309109276F
:10C5B00040910A2750910B27820F931FA41FB51F8C
:10C5C0008093082790930927A0930A27B0930B27FD
:10C5D00010923427FF91EF91BF91AF919F918F916E
:10C5E0007F916F915F914F913F912F910F900BBE73
:10C5F0000F900FBE0F901F9018959FB7F894E1E72A
:10C60000F0E08081807D808388B38F6288BB109248
:10C610009000E1E9F0E010821092920010929500F3
:10C62000109294008081856080839FBF08952FB70A
:10C63000F894909399008093980088B38F6288BB98
:10C64000E1E7F0E08081826080832FBF0895EF9260
:10C65000FF92CF93DF93FC01DB0185E0EB011992A0
:10C660008A95E9F7858190E083709070009711F0CA
:10C6700082E08C93878190E083709070009721F026
:10C6800082E012968C931297858190E0837090706F
:10C69000009799F0878190E083709070009769F01F
:10C6A00023893489818592852817390731F481E0FF
:10C6B000848312961C92129701C014828581837024
:10C6C0008250823030F4C82FD0E0CD53D94F8881CA
:10C6D00001C080E011968C931197E781E370E250DE
:10C6E000E23028F4F0E0ED53F94F808101C080E0A2
:10C6F00013968C931397DF91CF91FF90EF9008954D
:10C70000DF93CF9300D000D00F92CDB7DEB7BE013C
:10C710006F5F7F4F0E94276389819A81890F8D5FA8
:10C720009B81890F9C81890F9D81890F0F900F90AC
:10C730000F900F900F90CF91DF910895AF92BF921D
:10C74000CF92DF92EF92FF920F931F93DF93CF93DD
:10C7500000D000D000D0CDB7DEB78C017B01BE0188
:10C760006F5F7F4F4E830E942763C9809A81A92EF5
:10C77000BB24DB808C81682F70E095012C0D311D6E
:10C780002D5F3F4F2D0D311D260F371F5D81250F6A
:10C79000311D4E8150E0421753070CF4A8C0D80158
:10C7A00011964C91119750E041705070E3E0440FA6
:10C7B000551FEA95E1F712962C91129730E02170FF
:10C7C000307054E0220F331F5A95E1F7242B3C912F
:10C7D0003770232B13963C911397E32FF0E0E17011
:10C7E000F07045E0EE0FFF1F4A95E1F72E2B1496EF
:10C7F0003C911497E32FF0E0E170F07036E0EE0F1B
:10C80000FF1F3A95E1F72E2BF701208315964C91E7
:10C81000159750E043705070440F551F440F551F3B
:10C8200016962C91169730E02370307054E0220F4A
:10C83000331F5A95E1F7242B17963C9117973295A1
:10C84000330F330F307C322B318318962C9118978D
:10C850002283FC2DF23069F419962C91D70113969E
:10C860002C931397F801228514962C93149745E086
:10C8700001C043E0E92FF0E03B96E00FF11F542F99
:10C880000AC09701250F311DC290D901CC925F5F7C
:10C890000894A108B108A114B10499F7940FBD2D13
:10C8A000B23089F4F701E90FF11DD80153962C91AC
:10C8B000539720839F5FF701E90FF11D54962C9148
:10C8C000549720839F5FE82FF0E07596E00FF11FEB
:10C8D000292F08C0D701A20FB11D32913C932F5FC1
:10C8E0006150704061157105A9F7890F01C080E0A2
:10C8F00026960FB6F894DEBF0FBECDBFCF91DF9165
:10C900001F910F91FF90EF90DF90CF90BF90AF906D
:10C910000895BF92CF92DF92EF92FF920F931F93F1
:10C92000CF93DF937C01D62EEA01633008F4ADC0CB
:10C93000FC018081B82EB294B694B694B3E0BB22C9
:10C94000F1E0BF22F7019181292F269526952370CA
:10C95000C92EC294C694C694A3E0CA22382F377059
:10C960003883382F36953695369531703983382F80
:10C97000329531703A838295869581708B83BC8223
:10C980002D83892F829583708E83CF8282818887C1
:10C9900087010D5F1F4F222361F1F801918180E033
:10C9A000F7013381830F911D9A87898787010B5F78
:10C9B0001F4F223081F4CA010B9665E575E00E9495
:10C9C000933BF80181818B87F70185818C878701F3
:10C9D000095F1F4F16C02330A1F4F7013D96DA011D
:10C9E0001B9682918D93E017F107D9F7085F1F4FCF
:10C9F00008C0CA010B9665E575E00E94933B1A8654
:10CA00001986CC2089F1BB2059F4F801918180E08E
:10CA10002081820F911D9C8B8B8B0E5F1F4F04C05A
:10CA200089859A859C8B8B8BFC2DF23071F4CE011D
:10CA3000459665E575E00E94933BF80181818D8BF9
:10CA400080818E8B0E5F1F4F17C0FC2DF330A1F439
:10CA5000085F1F4FD801FE01759680E09E9191936B
:10CA60008F5F8830D9F708C0CE01459665E575E03F
:10CA70000E94933B1C8A1B8A802F8E199D2D981B28
:10CA80009FA71EA70DA7D81608F480E0DF91CF91CD
:10CA90001F910F91FF90EF90DF90CF90BF9008957E
:10CAA0009C0141505040460F571FDB0110C0FC91C4
:10CAB000E0E011968C911197BF01680F711D260F50
:10CAC000371F2617370710F42F5F3F4F1296A41712
:10CAD000B50768F3A417B50749F49C9180E0280FC7
:10CAE000391F2817390710F42F5F3F4FC9010895E8
:10CAF000CF93DF9390916227C92FD0E06497309154
:10CB0000612720E0C20FD31F9E01280F311DC901EC
:10CB10006BE677E248E050E00E94506563E777E219
:10CB2000AE010E945065009719F0382F292F02C0DE
:10CB30002FEF3FEFC901DF91CF91089590937B17BD
:10CB400080937A170895FC014381460F40935E2736
:10CB5000872F99272281280F20935D27A181A093F9
:10CB60005C27508150935B2730E02817390748F441
:10CB70008A2F8F5F80935C27882319F45F5F50931F
:10CB80005B27842F90E070708617970798F4809148
:10CB90005D278F5F80935D27882361F480915C27F8
:10CBA0008F5F80935C27882329F480915B278F5FB8
:10CBB00080935B270895BC018091642C9091652C33
:10CBC00008960E94A365E091642CF091652C8091F9
:10CBD0005B27808780915C27818780915D27828792
:10CBE00080915E27838708959C01AB0180E090E0EF
:10CBF000B9010E945065382F292FC901089580E09E
:10CC000090E06FE577E244E150E00E9450650097C4
:10CC100019F0382F292F02C02FEF3FEFC9010895D7
:10CC200086E00E947865089581E10E947865089504
:10CC300080E009C0E82FF0E0EE0FFF1FEA51F34D4E
:10CC4000118210828F5F8430A8F380E00BC0E82F40
:10CC5000F0E095E0EE0FFF1F9A95E1F7EA59F34DEA
:10CC6000118E8F5F843098F380E094E090937D176D
:10CC700080937C1740E08DE090E00EC0242F30E0E0
:10CC8000289FF001299FF00D389FF00D1124E450EA
:10CC9000F34D158214824F5F4A3080F3409378172A
:10CCA000089520917C1730917D172F5F3F4F4DE7FE
:10CCB0002030340710F020E030E1522F432FA0E065
:10CCC00013C0EA2FF0E0B5E0EE0FFF1FBA95E1F7D1
:10CCD000EA59F34DB18DBB2331F00480F581E02D8D
:10CCE000E417F50711F3AF5FA43059F730937D17C0
:10CCF00020937C171092781720E0E0E0F0E01EC04F
:10CD0000A22FB0E035E0AA0FBB1F3A95E1F7AA5970
:10CD1000B34D59963C915997332321F420937817BA
:10CD2000FD0110C0373049F4309731F05A964C91DC
:10CD30005A97328D341708F4FD012F5F243000F329
:10CD4000209378173097A9F122E0218F2091721754
:10CD500024872091731725872091741726872091A7
:10CD60007517278728ED34E0338B228B358B248B86
:10CD700021E030E0318B208B138E21E0228F23E0E5
:10CD8000208F168A20E1278B20917C1730917D1708
:10CD90003227232732273583248377836683DC0178
:10CDA0002D913D914D915C91139720833183428366
:10CDB0005383CF0108950F931F93CF93DF93209157
:10CDC0007C1730917D174DE050E02F5F3F4FADE76E
:10CDD00020303A0710F020E030E1B22FA32F10E00E
:10CDE00012C0C12FD0E0C49FF001C59FF00DD49FA9
:10CDF000F00D1124E450F34D0480F581E02DEA1785
:10CE0000FB0719F31F5F1A3061F730937D172093EA
:10CE10007C1710E02DE030E01AC0012F0F5FC12F0A
:10CE2000D0E0C29FF001C39FF00DD29FF00D1124FE
:10CE3000E450F34DDF0114964481558141155105AD
:10CE400029F410937817309749F433C0102F1A3013
:10CE500020F310937817E0E0F0E02BC020917C17CE
:10CE600030917D1732272327322711963C932E933A
:10CE700077836683009729F41082118212821382CD
:10CE800009C0DC012D913D914D915C91208331834E
:10CE9000428353838DE090E0C89FD001C99FB00DBD
:10CEA000D89FB00D1124A450B34D80E418968C93F4
:10CEB0001897CF01DF91CF911F910F91089540E016
:10CEC00013C0E42FF0E0542F5F5FEE0FFF1FEA5115
:10CED000F34D208131812817390729F440937817C1
:10CEE000118210820895452F443058F340937817EB
:10CEF000089540E013C0E42FF0E0542F5F5FEE0F81
:10CF0000FF1FEA51F34D208131812115310529F4AC
:10CF100040937817918380830895452F443058F3C8
:10CF2000409378170895EF92FF920F931F93CF933A
:10CF3000DF93C091642CD091652C843009F4F7C143
:10CF400007E817E21093632C0093622C10935A2782
:10CF500000935927833071F4898D90E08F70907021
:10CF60008330910509F074C088899989009709F088
:10CF70002FC78DC0823009F08EC0809175178F5FEA
:10CF800080937517882399F4809174178F5F80932D
:10CF90007417882361F4809173178F5F80937317E0
:10CFA000882329F4809172178F5F809372171092F3
:10CFB0005827109257271092FB2C1092FA2C898D2B
:10CFC000873011F0853041F48A8D8F5F8A8F8431EC
:10CFD00009F0FEC6198EFCC6882309F4F9C6288913
:10CFE00039892115310509F44EC09A8D292F215018
:10CFF0002A8F992309F0ECC69B8D983031F0282FA9
:10D000002150223048F4953039F4198E80E880930D
:10D010005F2C0E949F6195C5953048F423E030E075
:10D02000092E02C0220F331F0A94E2F701C020E349
:10D030002A8F9F5F9B8F90E08F7090708330910557
:10D04000E1F0843091054CF48130910509F461C31D
:10D050008230910509F0BCC60DC08630910509F4F7
:10D060000CC58830910509F408C58430910509F094
:10D07000AFC603C5109280274FC384E080935F2C16
:10D080000E949F6190C58F70833009F0A1C688E02F
:10D0900080935F2C4BC5853019F5E091602CF091A1
:10D0A000612C84819581009709F492C61092652CB9
:10D0B0001092642C0C5010401093632C0093622C3F
:10D0C00010935A27009359271092FB2C1092FA2C98
:10D0D000109258271092572788E080935F2C25C123
:10D0E0000852104080915F27853409F071C69091F5
:10D0F000612780E0209162277C01E20EF11C809183
:10D100005727909158278E159F0508F461C6F09215
:10D110005827E09257278091652790E08F73907091
:10D12000009709F055C680916627882309F050C6FC
:10D130008091F62C9091F72CC091C906D091CA0627
:10D140008C179D0759F44091F82C5091F92C20919F
:10D15000CB063091CC0642175307A1F020916F27E0
:10D16000309170272817390709F032C620917127AE
:10D17000309172278091F82C9091F92C281739075B
:10D1800009F026C60E94FF652FEF8F3F920709F036
:10D190001FC680916827863009F431C18131E9F1D9
:10D1A000813009F015C680917327883009F010C6C8
:10D1B0001092732780917527909176274FEF873FC4
:10D1C000940710F0099601C00896909376278093F3
:10D1D000752780916B2790916C27A0916D27B09156
:10D1E0006E2780936F2790937027A0937127B09339
:10D1F00072278091F62C9091F72CA091F82CB09189
:10D20000F92C80936B2790936C27A0936D27B09394
:10D210006E2780E4F8018087B8C5C7014C979093CA
:10D220005827809357278BE797E29093632C80933E
:10D23000622C8091792790917A27009739F00E948B
:10D240001466FFEF8F3F9F0709F0C2C52091752735
:10D25000309176272115310509F4BAC58CEF9CE28F
:10D260009093612C8093602C6091CB067091CC06DA
:10D270004091C5065091C6060091C7061091C80698
:10D2800039C084819581009781F12817390769F5A4
:10D2900086819781009739F0A0917327B091742708
:10D2A000A817B90711F5808191818C179D0729F482
:10D2B000A281B381A617B70739F18417950729F41E
:10D2C000A281B381A017B107F9F0A0916B27B091AB
:10D2D0006C27A817B90749F4A0916D27B0916E2764
:10D2E00082819381A817B90779F03D96F093612C5C
:10D2F000E093602CE091602CF091612C8DE2EE3790
:10D30000F80708F4BECF64C51092652C1092642C07
:10D3100082E080935F2C8BE797E290935A2780936B
:10D3200059271092FB2C1092FA2C0E949F61809139
:10D33000FA2C9091FB2C009709F44AC59C01245EBD
:10D340003F4F3093582720935727309361272093DE
:10D350006227E091602CF091612C20852093672753
:10D3600021E120936827089698278927982790938A
:10D3700078278093772710927A27109279278481D3
:10D3800095819093742780937327868197819093DA
:10D390007627809375278091F62C9091F72CA09199
:10D3A000F82CB091F92C80936B2790936C27A09365
:10D3B0006D27B0936E2780819181A281B381809384
:10D3C0006F2790937027A0937127B093722787E8F7
:10D3D00097E29093632C8093622C0E941466809550
:10D3E000909590937A2780937927009709F0CDC480
:10D3F0008FEF9FEF90937A2780937927C6C40E947E
:10D400001066EFEF8F3F9E0709F0E2C48091752709
:10D4100090917627009709F4DBC42091732730910F
:10D4200074272115310509F4D3C4C6E6DCE2498D21
:10D430004423E9F06C817D8186179707C1F46E81E2
:10D440007F812617370799F4E0916B27F0916C27BD
:10D4500068817981E617F70751F4E0916D27F09123
:10D460006E276A817B81E617F70709F46DC1A096E4
:10D47000FCE2C63EDF07D9F6209180272F732230C9
:10D48000B9F4909377178093761740E00DC0E42F9E
:10D49000F0E0EE0FFF1FEA51F34D208131814F5F25
:10D4A0008217930709F46EC0443088F340937817CD
:10D4B0008091802782FD8CC484E1F80181A388E2F9
:10D4C00090E0909358278093572780E580A3809120
:10D4D0007A2790917E27938F3091792790917D279D
:10D4E000928F368F2091782790917C27918F258F6E
:10D4F000909177279093781740917B27408F948F56
:10D500008F5F878F882361F4832F8F5F868F8823B7
:10D5100039F4822F8F5F858F882311F49F5F948F5A
:10D520008091732790917427909377178093761743
:10D530002091752730917627F801358B248B978BB6
:10D54000868B80916B2790916C27A0916D27B0916D
:10D550006E2780936F2790937027A0937127B093C5
:10D5600072278091F62C9091F72CA091F82CB09115
:10D57000F92C80936B2790936C27A0936D27B09321
:10D580006E27E8C31092781780E0C0E0D0E022C098
:10D59000E82FF0E075E0EE0FFF1F7A95E1F7EA590A
:10D5A000F34D918D992321F480937817EF0116C0E4
:10D5B000973079F4209721F0228D9A8D921748F4B4
:10D5C000C82FD0E065E0CC0FDD1F6A95E1F7CA599E
:10D5D000D34D8F5F8430E0F280937817209709F461
:10D5E000F7C3D093652CC093642C83E08A8F888F17
:10D5F0001E8A84E08F8B1B8E8091752790917627F1
:10D600009D838C8380917327909174279F838E8351
:10D6100080916B2790916C27A0916D27B0916E2718
:10D6200088839983AA83BB8381E0898F8091721755
:10D630008C87809173178D87809174178E87809166
:10D6400075178F8781E090E0998B888B80917A277E
:10D650008B87809179278A87809178278987809125
:10D660007727888781E090E00E94DB6580917F27A3
:10D67000282F30E0207F3070213531050CF449C06F
:10D6800082958F7090E00597880F991F880F991FDA
:10D690005091791740E034C0F901E15AF84D50A596
:10D6A000552329F4409378171092791732C05130DE
:10D6B00011F44F5F25C05230E1F461A56430C9F424
:10D6C000409378175093791732A520E083A590E016
:10D6D000822B932B9093771780937617F4E0893DF4
:10D6E0009F0710F088ED94E09B8B8A8B9D8B8C8B31
:10D6F00010C0215A384DF90121A5222331F0420FE3
:10D70000242F30E0281739073CF2409378175093C4
:10D71000791780E1809380278091802782608093B1
:10D72000802782E08093872784E0809388278093F6
:10D73000892788ED80938A278CE290E09093582780
:10D740008093572780E6B3C2D093652CC093642C96
:10D7500010925F2C8091802790E082FF03C0198E89
:10D7600080E24EC220917F2722952F70220F220F38
:10D7700020937817B701621B71099B012451304037
:10D78000309358272093572750E04F705070423005
:10D79000510539F4AC014F7350704231510551F4C9
:10D7A0002AC04130510531F4AC014F735070423002
:10D7B000510509F12115310531F49C0123703070B8
:10D7C00021153105C1F0309177272885321709F0EE
:10D7D00064C2309178272985321709F05EC23091F2
:10D7E00079272A85321709F058C230917A272B857C
:10D7F000321709F052C284FF4AC0688979896115DD
:10D80000710509F444C0CE010C960E94A3653091C5
:10D810007B2780915B273817D1F520917C27809159
:10D820005C272817A1F590917D2780915D27981797
:10D8300071F580917E2740915E27841741F53C87E2
:10D840002D879E878F878B8D8823D1F42E89888D95
:10D850009A8D891B922F969596959695891B280FE0
:10D860002E8B87FD81959F89392F36953695931B91
:10D87000980F9F8B822F869586958695890F888F26
:10D8800081E080935F2C888D8A8F198A188A298D70
:10D8900030E0C9018F7090708430910509F4B5C1F2
:10D8A0008530910564F482309105C9F1833091058A
:10D8B0000CF0B9C08130910509F08AC211C08630E0
:10D8C000910509F4E2C1863091050CF4BEC18730A0
:10D8D000910509F4E2C18830910509F079C28AC145
:10D8E00080915F2C80FF14C083E0898F80E4809357
:10D8F0005F2C198A188A8091572790915827009792
:10D9000009F410C122E420935F2C0E94DB650AC158
:10D91000809180278F73823009F05AC2FACE8091AD
:10D920005F2C80FF75C0809180278F73823109F052
:10D930006FC080917F27282F30E0207F3070213505
:10D9400031050CF449C082958F7090E00597880FDF
:10D95000991F880F991F5091791740E034C0F90141
:10D96000E15AF84D50A5552329F4409378171092A9
:10D97000791732C0513011F44F5F25C05230E1F4B5
:10D9800061A56430C9F4409378175093791732A594
:10D9900020E083A590E0822B932B909377178093C0
:10D9A000761774E0893D970710F088ED94E09B8B23
:10D9B0008A8B9D8B8C8B10C0215A384DF90121A583
:10D9C000222331F0420F242F30E0281739073CF290
:10D9D000409378175093791783E0898F8091772748
:10D9E0008887809178278987809179278A87809195
:10D9F0007A278B8781E090E00E94DB6582E4809348
:10DA00005F2C198A188A10925827109257278AC0BB
:10DA100080E280935F2C0E949F61E091642CF091E2
:10DA2000652C118E45CD8091802780FF2AC024FD72
:10DA300028C088899989009709F0CAC18091572721
:10DA40009091582701960E94DB6520915F2C822FD0
:10DA5000806180935F2C8091572790915827009781
:10DA600019F0226120935F2C0E949F6181E090E079
:10DA7000998B888B88E0898F1B8E81E1809380272A
:10DA80000FC185FF1CC05091852740E080918627FB
:10DA900090E0842B952B4091622C5091632C480F81
:10DAA000591F5093632C4093622C409157275091FB
:10DAB0005827481B590B509358274093572780915C
:10DAC000572790915827009749F024FD07C02091CF
:10DAD0005F2C226020935F2C0E94DB659091812750
:10DAE00080E020918227820F911D90937717809379
:10DAF00076172C893D892817390710F0009721F4F3
:10DB00003093771720937617809176179091771737
:10DB10009B8B8A8B80915F2C90E083709070009734
:10DB200009F456C11092FB2C1092FA2C0E949F61AE
:10DB300080915F2C85FF07C01092FB2C1092FA2C6D
:10DB4000198E84E19BCF84FF0AC01092FB2C1092A7
:10DB5000FA2C81E090E0998B888B84E08CCF209127
:10DB6000FA2C3091FB2C21153105E1F080FF02C029
:10DB7000198A188A88899989009781F48A899B89EA
:10DB80008217930720F49093FB2C8093FA2C8091BA
:10DB9000FA2C9091FB2C998B888B04C09093FB2CD2
:10DBA0008093FA2C1B8E8091592790915A2790933D
:10DBB000632C8093622C8091FA2C9091FB2C00971F
:10DBC00059F088899989009739F088969093582759
:10DBD0008093572788E10BC080915F2C81FFF8C0AC
:10DBE00088E290E0909358278093572780E18093B4
:10DBF00080275CC080915F2C80FFEAC0198E80E195
:10DC000080935F2C0E949F61E3C080915727909181
:10DC10005827009711F00E94DB6590918027809132
:10DC20005F2C90FF0BC080FF06C087E0898F1A8EA3
:10DC3000198A188A19C086E0898F16C080FF1EC015
:10DC400085E0898F198A188AC3C0809157279091DF
:10DC50005827009711F00E94DB658091802780FF94
:10DC60000DC087E0898F1A8E81E090E00E94DB650D
:10DC700080E180935F2C0E949F610FC080915727A5
:10DC800090915827009749F4A3C080915F2C80FFA2
:10DC90009FC087E0898F1A8E9BC080E1F80181A325
:10DCA00088E290E0909358278093572780E58093EF
:10DCB0007F27888580937B27898580937C278A8529
:10DCC00080937D278B8580937E278C858093772713
:10DCD0008D85809378278E85809379278F85809393
:10DCE0007A2786E0809368278C819D8190937427A2
:10DCF000809373278E819F819093762780937527D9
:10DD00008091F62C9091F72CA091F82CB091F92CE1
:10DD100080936B2790936C27A0936D27B0936E2709
:10DD200088819981AA81BB8180936F279093702706
:10DD3000A0937127B0937227898D84FF05C010923C
:10DD400082271092812706C084E08093812788ED86
:10DD50008093822780E48093672780915727909152
:10DD600058279093612780936227109286271092FC
:10DD7000852710928427109283270E941066809531
:10DD80009095909384278093832785E480935F27E1
:10DD900010926027109266271092652780917A175B
:10DDA00090917B17019690937B1780937A179093AD
:10DDB00063278093642710926A27109269270E9434
:10DDC000FF658095909590936A278093692704C09A
:10DDD000109258271092572710925F2CDF91CF9105
:10DDE0001F910F91FF90EF900895382F292FC901AF
:10DDF0000895382F292F40E050E0762767277627AF
:10DE000080E090E0CB0177276627262B372B482B25
:10DE1000592BB901CA010895AC01E0915927F0913D
:10DE20005A27222733272E1B3F0B215A334D6217C7
:10DE300073070CF49B011216130664F42093FA2C5A
:10DE40003093FB2C4E175F0729F0CF01BA01A901CF
:10DE50000E94117A08950F93DF93CF93CDB7DEB769
:10DE600060970FB6F894DEBF0FBECDBF002309F454
:10DE700059C029833A834B835C836D837E838F8370
:10DE80009887E0E2E01B29813A814B815C811E1674
:10DE9000BCF019861A861B861C868E2F992787FD53
:10DEA0009095909581959F4F04C0220F331F441F7A
:10DEB000551F8A95D2F72D873E874F87588B2AC0EA
:10DEC000CA01B901002E04C0660F771F881F991F71
:10DED0000A94D2F769877A878B879C87DA01C90110
:10DEE00004C0B695A79597958795EA95D2F72D81A9
:10DEF0003E814F81588504C0220F331F441F551F98
:10DF00000A95D2F7822B932BA42BB52B8D879E8756
:10DF1000AF87B88B29853A854B855C856D857E8575
:10DF20008F85988960960FB6F894DEBF0FBECDBF7F
:10DF3000CF91DF910F910895A0E1B0E0E2EAFFE612
:10DF40000C94647729833A834B835C836D837E834F
:10DF50008F839887A986BA86CB86DC86ED86FE8677
:10DF60000F87188B2D813E814F8158858D859E8529
:10DF7000AF85B889281739074A075B07C8F08217A9
:10DF80009307A407B50790F029813A814B815C8102
:10DF900089859A85AB85BC85281739074A075B07B1
:10DFA00038F082179307A407B50720F482E003C076
:10DFB00080E001C081E06096EAE00C9480772F92C7
:10DFC0003F924F925F926F927F928F929F92AF9209
:10DFD000BF92CF92DF92EF92FF920F931F93DF9346
:10DFE000CF93CDB7DEB763970FB6F894DEBF0FBE01
:10DFF000CDBF6C017F876E87FC01178216828381FB
:10E0000081FD04C06FC34C855D8504C01E0108946A
:10E01000211C311CF6019381EE85FF8593FD8591CE
:10E0200093FF8191FF87EE87882309F457C38532D8
:10E0300041F493FD859193FF8191FF87EE878532AF
:10E0400059F490E0B6014A8B5B8B0E94737A4A893F
:10E050005B895D874C87D7CF10E0FF2400E000325A
:10E06000B0F48B3269F08C3228F4803251F0833274
:10E0700071F40BC08D3239F0803349F401602CC04B
:10E080000260046029C0086027C0006125C007FD48
:10E090002EC0282F20532A3098F406FF08C0812F65
:10E0A000880F182F110F110F180F120F15C08F2D79
:10E0B000880FF82EFF0CFF0CF80EF20E00620CC059
:10E0C0008E3221F406FD0AC3006406C08C3611F4BA
:10E0D000006802C0883659F4EE85FF8593FD85916E
:10E0E00093FF8191FF87EE87882309F0B8CF982F9F
:10E0F0009554933018F40061805E06C0982F9556B1
:10E10000933008F09BC10F7E06FF16E06FE3E62E0A
:10E11000E022853619F4F0E4EF2A07C0863619F4B8
:10E1200020E8E22A02C011111150E7FE06C01C339C
:10E1300040F4912E939427E00BC0183030F4212F37
:10E1400006C027E03CE3932E03C027E017E09924A4
:10E15000CA0104969D878C87FA0160817181828152
:10E160009381A101092D0E9421795C016980262DEE
:10E1700030E0398B288B60FE03C0388933FF06C03E
:10E18000E1FC06C0E2FE06C000E205C00DE203C0ED
:10E190000BE201C000E0888999898C70907000972B
:10E1A000C1F1002311F084E001C083E08F1558F421
:10E1B000F81AE3FC09C080E290E0B6010E94737A8D
:10E1C000FA94C9F701C0FF24002329F0802F90E0C2
:10E1D000B6010E94737A888983FD03C002E31FE0C1
:10E1E0000EC00EE21FE00BC0A114B10409F0805272
:10E1F00090E0B6010E94737A0F5F1F4F05C0AE2CEE
:10E20000BB2490E1A922BB24F8018491882361F703
:10E2100062C2E7FE0EC09A0CF889F4FF04C08A813E
:10E22000813309F49A94191454F5292D293050F5A5
:10E230002DC0E6FC2BC0812F90E08A159B054CF089
:10E240003CEFA3163FEFB30624F080E8E82A01C0B4
:10E250001150112349F0E2E0F0E0EC0FFD1FE10F57
:10E26000F11D80818033A1F3E7FE10C0912E9394BD
:10E27000812F90E0A816B90644F41A1907C0992412
:10E28000939404C098E0992E01C010E0E7FE07C007
:10E290001A141B043CF495012F5F3F4F05C025E085
:10E2A00030E002C021E030E0002311F02F5F3F4F4B
:10E2B000112329F0812F90E00196280F391F8F2D0F
:10E2C00090E02817390714F4F21A01C0FF244E2CED
:10E2D0005524C20189709070009749F406C080E20D
:10E2E00090E0B6010E94737AFA94FF20C1F70023F0
:10E2F00029F0802F90E0B6010E94737A43FC09C098
:10E3000006C080E390E0B6010E94737AFA94FF2081
:10E31000C1F7E7FE46C03501B7FE02C06624772488
:10E3200025010894411C511C46185708420C531CE7
:10E33000F501E919F1094F01812F90E0002711271C
:10E34000081B190BFFEF6F16FFEF7F0629F48EE213
:10E3500090E0B6010E94737AA614B70434F08614D4
:10E3600097041CF4F201808101C080E308946108E5
:10E3700071080894411C511C601671062CF090E045
:10E38000B6010E94737ADECF6A147B0441F49A814D
:10E39000963320F4953319F4F889F4FF81E390E083
:10E3A00049C08A81813311F02FEE622290E0B601DC
:10E3B0000E94737A112389F08EE290E0B6010E94E8
:10E3C000737A02E0F101E00FF11D0F5F808190E0B0
:10E3D000B6010E94737A1150A9F744FE03C085E488
:10E3E00090E002C085E690E0B6010E94737AB7FC27
:10E3F00005C0A114B10441F464FE06C0B094A19418
:10E40000B108B3948DE201C08BE290E0B6010E94A6
:10E41000737A80E305C08F5FE6EFFFEFAE0EBF1E9D
:10E42000FAE0AF16B104BCF790E0B6010E94737A2F
:10E43000C501C096B6010E94737A4DC1833631F092
:10E44000833789F0833509F059C022C09A012E5FC5
:10E450003F4F3D872C87FA0180818983310181E01C
:10E46000A82EB12C13C09A012E5F3F4F3D872C87F9
:10E47000FA016080718006FF03C0612F70E002C066
:10E480006FEF7FEFC3010E94397A5C010F7714C0F0
:10E490009A012E5F3F4F3D872C87FA016080718083
:10E4A00006FF03C0612F70E002C06FEF7FEFC30172
:10E4B0000E94017A5C01006803FD1CC006C080E276
:10E4C00090E0B6010E94737AFA948F2D90E0A8161E
:10E4D000B906A8F30FC0F30107FD859107FF8191ED
:10E4E0003F0190E0B6010E94737AF110FA9408940B
:10E4F000A108B108A114B10471F7EDC0843611F080
:10E50000893661F507FF0BC09A012C5F3F4F3D87AD
:10E510002C87FA0160817181828193810CC09A01FC
:10E520002E5F3F4F3D872C87FA01608171818827DC
:10E5300077FD8095982F0F7697FF08C0909580956E
:10E54000709561957F4F8F4F9F4F0068A1012AE022
:10E5500030E00E94857B982E921841C0853721F4C7
:10E560000F7E2AE030E020C0097F8F36A9F0803787
:10E5700020F4883509F0B2C00BC0803721F088370D
:10E5800009F0ACC001C0006104FF09C0046007C00D
:10E5900004FF08C0066006C028E030E005C020E1A6
:10E5A00030E002C020E132E007FF0AC0CA01049651
:10E5B0009D878C87FA01608171818281938109C076
:10E5C000CA0102969D878C87FA016081718180E083
:10E5D00090E0A1010E94857B982E92180F7706FF8C
:10E5E00009C00E7F911630F404FF06C002FD04C07E
:10E5F0000F7E02C0E92C01C0E12E802F90E004FFC5
:10E600000CC0FE01E90DF11D2081203311F4097EBB
:10E6100009C0E39402FF06C004C08678907000979A
:10E6200009F0E394A02EBB2403FD14C000FF0FC02B
:10E63000EF1428F4192D1F0D1E19EF2C08C0192DE9
:10E6400006C080E290E0B6010E94737AE394EF1472
:10E65000C0F304C0EF1410F4FE1801C0FF24A4FEA0
:10E660000FC080E390E0B6010E94737AA2FE1FC043
:10E67000A1FE03C088E590E010C088E790E00DC0DF
:10E68000C50186789070009791F0A1FC02C080E2ED
:10E6900001C08BE207FD8DE290E0B6010E94737A23
:10E6A00006C080E390E0B6010E94737A1150911683
:10E6B000C0F39A94F101E90DF11D808190E0B6015B
:10E6C0000E94737A9920A9F706C080E290E0B60113
:10E6D0000E94737AFA94FF20C1F795CCF601268147
:10E6E000378102C02FEF3FEFC90163960FB6F89450
:10E6F000DEBF0FBECDBFCF91DF911F910F91FF9075
:10E70000EF90DF90CF90BF90AF909F908F907F90D1
:10E710006F905F904F903F902F9008955058BB2777
:10E72000AA270ED044C135D130F03AD120F031F4CF
:10E730009F3F11F41EF42AC10EF4E095E7FB20C1BF
:10E74000E92F46D180F3BA1762077307840795074C
:10E7500018F071F49EF55EC10EF4E0950B2EBA2F01
:10E76000A02D0B01B90190010C01CA01A0011124D7
:10E77000FF27591B99F0593F50F4503E68F11A1683
:10E78000F040A22F232F342F4427585FF3CF469514
:10E7900037952795A795F0405395C9F77EF41F1636
:10E7A000BA0B620B730B840BBAF09150A1F0FF0F00
:10E7B000BB1F661F771F881FC2F70EC0BA0F621FEC
:10E7C000731F841F48F4879577956795B795F795DC
:10E7D0009E3F08F0B3CF9395880F08F09927EE0F6E
:10E7E000979587950895A8D008F481E008950CD0F6
:10E7F000DEC0D6D040F0CDD030F021F45F3F19F02C
:10E80000BFC0511108C1C2C0E3D098F39923C9F326
:10E810005523B1F3951B550BBB27AA276217730726
:10E82000840738F09F5F5F4F220F331F441FAA1FDA
:10E83000A9F333D00E2E3AF0E0E830D0915050409A
:10E84000E695001CCAF729D0FE2F27D0660F771F48
:10E85000881FBB1F261737074807AB07B0E809F02A
:10E86000BB0B802DBF01FF2793585F4F2AF09E3FBF
:10E87000510568F085C0CFC05F3FECF3983EDCF3F4
:10E88000869577956795B795F7959F5FC9F7880F38
:10E89000911D9695879597F90895E1E0660F771F8A
:10E8A000881FBB1F621773078407BA0720F0621B1B
:10E8B000730B840BBA0BEE1F88F7E0950895E8946C
:10E8C00009C097FB3EF490958095709561957F4FB8
:10E8D0008F4F9F4F9923A9F0F92F96E9BB27939566
:10E8E000F695879577956795B795F111F8CFFAF476
:10E8F000BB0F11F460FF1BC06F5F7F4F8F4F9F4FA7
:10E9000016C0882311F096E911C0772321F09EE804
:10E91000872F762F05C0662371F096E8862F70E06A
:10E9200060E02AF09A95660F771F881FDAF7880F44
:10E930009695879597F90895990F0008550FAA0B9A
:10E94000E0E8FEEF16161706E807F907C0F0121602
:10E950001306E407F50798F0621B730B840B950B05
:10E9600039F40A2661F0232B242B252B21F408955A
:10E970000A2609F4A140A6958FEF811D811D0895F7
:10E9800097F99F6780E870E060E008959FEF80EC62
:10E99000089500240A941616170618060906089505
:10E9A00000240A9412161306140605060895092E6B
:10E9B0000394000C11F4882352F0BB0F40F4BF2BDA
:10E9C00011F460FF04C06F5F7F4F8F4F9F4F08951A
:10E9D00057FD9058440F551F59F05F3F71F0479510
:10E9E000880F97FB991F61F09F3F79F087950895F5
:10E9F000121613061406551FF2CF4695F1DF08C014
:10EA0000161617061806991FF1CF86957105610530
:10EA100008940895E894BB2766277727CB0197F9D8
:10EA200008950BD0C4CFB5DF28F0BADF18F09523D6
:10EA300009F0A6CFABCF1124EECFCADFA0F3959F8C
:10EA4000D1F3950F50E0551F629FF001729FBB27D5
:10EA5000F00DB11D639FAA27F00DB11DAA1F649F81
:10EA60006627B00DA11D661F829F2227B00DA11D34
:10EA7000621F739FB00DA11D621F839FA00D611DBA
:10EA8000221F749F3327A00D611D231F849F600DDB
:10EA9000211D822F762F6A2F11249F5750408AF014
:10EAA000E1F088234AF0EE0FFF1FBB1F661F771FA0
:10EAB000881F91505040A9F79E3F510570F060CFDC
:10EAC000AACF5F3FECF3983EDCF386957795679588
:10EAD000B795F795E7959F5FC1F7FE2B880F911DBE
:10EAE0009695879597F90895FA01EE0FFF1F3096D6
:10EAF0002105310599F16115710561F48038BFE395
:10EB00009B0749F168949038810561F08038BFEF28
:10EB10009B0741F0992342F5FF3FE10531052105AF
:10EB200011F1E8940894E795D901AA2329F4AB2FB1
:10EB3000BE2FF85FD0F310C0FF5F70F4A695E0F72A
:10EB4000F73950F019F0FF3A38F49F779F930CD0C3
:10EB50000F9007FC905808953EF018CF60E070E0E9
:10EB600080E89FE308954FE79F775F934F933F932C
:10EB70002F939ED02F913F914F915F9152DF05C00F
:10EB800019F40EF0FDCE46CF01CF2ADFC8F3963838
:10EB9000C0F707F80F92E8942BE33AEA48EB5FE7F7
:10EBA0004EDF0F920F920F924DB75EB70F92C0D00B
:10EBB000E0E2F1E016D04F915F91EF91FF91E59582
:10EBC000EE1FFF1F49F0FE57E0684427EE0F441F79
:10EBD000FA95E1F74195550B32D00F9007FE26C00C
:10EBE0000895DF93CF931F930F93FF92EF92DF92DD
:10EBF0007B018C01689405C0DA2EEF011EDFFE0157
:10EC0000E894A5912591359145915591AEF3EF0189
:10EC100097DDFE019701A801DA9479F7DF90EF9074
:10EC2000FF900F911F91CF91DF9108959B01AC014F
:10EC300060E070E080E89FE3DACDA2CEACC0D0DE29
:10EC4000E8F39923D9F3940F511DBBF39150504031
:10EC500094F059F0882332F0660F771F881F915087
:10EC60005040C1F79E3F510544F7880F911D96957E
:10EC7000879597F908955F3FACF0983E9CF0BB27CD
:10EC8000869577956795B79508F4B1609395C1F728
:10EC9000BB0F58F711F460FFE8CF6F5F7F4F8F4FC6
:10ECA0009F4FE3CFB8CE0EF076C070CE689468CE9A
:10ECB00097DEC8F39923D1F3C6F3DF93CF931F9365
:10ECC0000F93FF92C92FDD2788232AF02197660F23
:10ECD000771F881FDAF720E030E040E85FEB9FE322
:10ECE000883920F0803E30F021968F7718DDE8E4F7
:10ECF000F1E003C014DDE5E7F1E073DF8B01BE0155
:10ED0000EC01FB2E6F5771097595771F880B990BD6
:10ED1000D8DD28E132E741E35FE38FDEAF2D9801D4
:10ED2000AE01FF900F911F91CF91DF9109DD3FCE92
:10ED3000FA01DC01AA0FBB1F9B01AC01BF5728F4ED
:10ED400022273327442750781FC0B75188F4AB2FB0
:10ED50000024469537952795011CA395D2F30020F2
:10ED600069F0220F331F441FB395DAF30DD0D6CCD0
:10ED700061307105A0E88A07B94630F49B01AC0107
:10ED80006627772788279078309621F02083318373
:10ED90004283538308959F3F31F0915020F487952B
:10EDA00077956795B795880F911D9695879597F9F3
:10EDB0000895629FD001739FF001829FE00DF11DC5
:10EDC000649FE00DF11D929FF00D839FF00D749FE5
:10EDD000F00D659FF00D9927729FB00DE11DF91F91
:10EDE000639FB00DE11DF91FBD01CF0111240895EE
:10EDF000AA1BBB1B51E107C0AA1FBB1FA617B70761
:10EE000010F0A61BB70B881F991F5A95A9F780957C
:10EE10009095BC01CD01089597FB092E07260AD0D5
:10EE200077FD04D0E5DF06D000201AF470956195D7
:10EE30007F4F0895F6F7909581959F4F0895A1E231
:10EE40001A2EAA1BBB1BFD010DC0AA1FBB1FEE1F64
:10EE5000FF1FA217B307E407F50720F0A21BB30BAF
:10EE6000E40BF50B661F771F881F991F1A9469F72B
:10EE700060957095809590959B01AC01BD01CF0187
:10EE8000089597FB092E05260ED057FD04D0D7DF35
:10EE90000AD0001C38F450954095309521953F4F8D
:10EEA0004F4F5F4F0895F6F7909580957095619557
:10EEB0007F4F8F4F9F4F08952F923F924F925F92B7
:10EEC0006F927F928F929F92AF92BF92CF92DF927A
:10EED000EF92FF920F931F93CF93DF93CDB7DEB7DF
:10EEE000CA1BDB0B0FB6F894DEBF0FBECDBF099473
:10EEF0002A88398848885F846E847D848C849B84CA
:10EF0000AA84B984C884DF80EE80FD800C811B81D7
:10EF1000AA81B981CE0FD11D0FB6F894DEBF0FBE06
:10EF2000CDBFED010895AF92BF92CF92DF92EF92E5
:10EF3000FF920F931F93CF93DF93EC016881798148
:10EF40008A819B81611571058105910521F464E237
:10EF500079ED8BE597E02DE133EF41E050E00E9441
:10EF6000417779018A0127EA31E440E050E00E94CC
:10EF7000D9765B016C01C801B7012CEE34EF4FEF7D
:10EF80005FEF0E94D9766A0D7B1D8C1D9D1D97FF3A
:10EF900004C06150704080409048688379838A83C0
:10EFA0009B837F77CB01DF91CF911F910F91FF90D2
:10EFB000EF90DF90CF90BF90AF9008950E9493772D
:10EFC00008958DEC96E00E9493770895A0E0B0E05C
:10EFD0008093CD069093CE06A093CF06B093D00633
:10EFE00008952F923F924F925F926F927F929F92DD
:10EFF000AF92BF92CF92DF92EF92FF920F931F9347
:10F00000CF93DF933B01EA016115710519F0FB0114
:10F0100080839183209739F09E0122503040233223
:10F02000310508F0D5C0C82ED92EF60111916F0117
:10F030007F01812F90E00E94F9790097B1F71D328E
:10F0400031F4F60111917F019924939406C01B328B
:10F0500019F4F60111917F019924209719F0C0311C
:10F06000D105D1F4103389F4F7018081883711F08C
:10F07000883559F4F701118182E090E0E80EF91E1D
:10F0800092E0992AC0E1D0E007C0209729F410331C
:10F09000B1F0CAE0D0E02BC0CA30D10541F1C03197
:10F0A000D10521F0C830D105A9F409C02FEFA22E57
:10F0B0002FEFB22E2FEFC22E2FE0D22E20C0C8E0AD
:10F0C000D0E09FEFA92E9FEFB92E9FEFC92E9FE1B1
:10F0D000D92E15C09E01442737FD4095542F6FEF60
:10F0E0007FEFCB010E941F7759016A0108C089E9AF
:10F0F000A82E89E9B82E89E9C82E89E1D82E60E0CA
:10F1000020E030E0A9011E01442437FC4094542C37
:10F11000012F00530A3060F0812F81548A3110F49E
:10F12000075006C0812F81568A3150F5012F0755AF
:10F13000802F90E08C179D071CF56F3FE9F0A21619
:10F14000B306C406D506A8F0CA01B901A20191010F
:10F150000E94D9769B01AC01802F90E0A0E0B0E046
:10F16000280F391F4A1F5B1F281739074A075B07FB
:10F1700010F46FEF01C061E0F70111917F01C8CF7A
:10F180006114710481F0662339F00894E108F108F4
:10F19000F301F182E08207C091FE05C0C70102972A
:10F1A000F3019183808390FE07C050954095309580
:10F1B00021953F4F4F4F5F4F67FF0DC082E290E0B8
:10F1C0009093852D8093842D2FEF3FEFA90103C0ED
:10F1D00020E030E0A901B901CA01DF91CF911F9170
:10F1E0000F91FF90EF90DF90CF90BF90AF909F90E6
:10F1F0007F906F905F904F903F902F90089566277B
:10F2000077270C941E7CFC0188279927E89421918C
:10F210002032E9F3293010F02E30C8F32B3241F0C0
:10F220002D3239F4689404C00E946B7A820F911DCC
:10F23000219120532A30C0F31EF4909581959F4F61
:10F240000895283008F027E03327DA01990F311D9F
:10F2500087FD916000966105710539F432602E5F7B
:10F260003D9330E32A95E1F708959F3F30F08038D1
:10F270007105610509F03C5F3C5F3D93913008F0FA
:10F280008068911DDF93CF931F930F93FF92EF92AE
:10F29000192F987F9695E92F96959695E90FFF2758
:10F2A000E057F04F99273327EE24FF24A701E70109
:10F2B00005900894079428F4360FE71EF81E491F9E
:10F2C000511D660F771F881F991F0694A1F705909F
:10F2D000079428F4E70EF81E491F561FC11D770F2B
:10F2E000881F991F661F0694A1F70590079428F4BC
:10F2F000F80E491F561FC71FD11D880F991F661F83
:10F30000771F0694A1F70590079420F4490F561F24
:10F31000C71FD81F990F661F771F881F0694A9F76C
:10F3200084911095177041F0D695C79557954795DC
:10F33000F794E7941A95C1F7E6E3FFE06894159017
:10F34000159135916591959105907FE27395E1183E
:10F35000F10A430B560BC90BD009C0F7E10CF11EA3
:10F36000431F561FC91FD01D7EF4703311F48A95B8
:10F37000E6CFE894015030F0080F0AF40027021796
:10F3800008F4202F2395022F7A3328F079E37D9318
:10F390002A95E9F710C07D932A9589F606949795EA
:10F3A0006795379517951794E118F10A430B560B9B
:10F3B000C90BD00998F023957E9173957A3308F0A4
:10F3C00070E37C932013B8F77E9170617D9330F0E9
:10F3D000839571E37D9370E32A95E1F71124EF9013
:10F3E000FF900F911F91CF91DF91992787FD909505
:10F3F00008959111B1C3803219F089508550D0F72A
:10F400000895FC010590615070400110D8F7809577
:10F4100090958E0F9F1F08954EE757E10E94447A02
:10F420000895FB01DC0102C001900D924150504053
:10F43000D8F70895DC0101C06D9341505040E0F7CA
:10F440000895FB01DC018D91019080190110D9F321
:10F45000990B0895FB01DC014150504048F00190A8
:10F460000D920020C9F701C01D9241505040E0F7B5
:10F470000895FC016150704001900110D8F780950B
:10F4800090958E0F9F1F0895FA01A191B08100976A
:10F4900019F41097E1F0CD01DC01CD010D900020B1
:10F4A00011F4C00113C0FB012191222319F0201592
:10F4B000D9F7F3CFFB012191201519F41E92119673
:10F4C00006C02223C1F70D900020A1F7D001FA0158
:10F4D000A193B08308957AE0979F902D879F802D08
:10F4E000910D112408950F931F93CF93DF938C01F7
:10F4F000EB018B8181FF1BC082FF0DC02E813F81FC
:10F500008C819D812817390764F4E881F981019382
:10F51000F983E88306C0E885F985802F099500976F
:10F5200031F48E819F8101969F838E8302C00FEFFD
:10F530001FEFC801DF91CF911F910F910895DF93C5
:10F54000CF93CDB7DEB7FE01359661917191809171
:10F55000802D9091812DAF010E94DF6FCF91DF91BF
:10F560000895DF93CF93CDB7DEB7FE013596619155
:10F5700071918091802D9091812DDC0113962C91B9
:10F580001397286013962C93AF010E94DF6FE091D0
:10F59000802DF091812D2381277F2383CF91DF91CF
:10F5A00008956091802D7091812D0E94737A089545
:10F5B000EF92FF920F931F93CF93DF938C01E09113
:10F5C000802DF091812D838181FF1FC0C0E0D0E0AC
:10F5D0000AC0DB011896ED91FC91199709950097E7
:10F5E00011F0CFEFDFEFF80181918F016091802D55
:10F5F0007091812D882369F7DB011896ED91FC91BC
:10F6000019978AE00995009711F0CFEFDFEFCE014F
:10F61000DF91CF911F910F91FF90EF9008950F937D
:10F620001F93DF93CF93CDB7DEB72E970FB6F89425
:10F63000DEBF0FBECDBF0D891E898F89988D26E054
:10F640002C831A83098397FF02C080E090E801971A
:10F650009E838D839E01255E3F4FCE010196698D6D
:10F660007A8DA9010E94DF6F4D815E8157FD0AC02E
:10F670002F813885421753070CF49A01020F131F8C
:10F68000F80110822E960FB6F894DEBF0FBECDBFE4
:10F69000CF91DF911F910F9108950F931F93DF93E7
:10F6A000CF93CDB7DEB72E970FB6F894DEBF0FBE5F
:10F6B000CDBF8C01CB01BA0146E04C831A8309838C
:10F6C00097FF02C080E090E801979E838D83CE0172
:10F6D0000196A9010E94DF6F4D815E8157FD0AC02E
:10F6E0002F813885421753070CF49A01020F131F1C
:10F6F000F80110822E960FB6F894DEBF0FBECDBF74
:10F70000CF91DF911F910F910895FA01AA27283018
:10F7100051F1203181F1E8946F936E7F6E5F7F4FDE
:10F720008F4F9F4FAF4FB1E03ED0B4E03CD0670F5A
:10F73000781F891F9A1FA11D680F791F8A1F911DAD
:10F74000A11D6A0F711D811D911DA11D20D009F4FD
:10F7500068943F912AE0269F11243019305D31933F
:10F76000DEF6CF010895462F4770405D4193B3E028
:10F770000FD0C9F7F6CF462F4F70405D4A3318F0CF
:10F78000495D31FD4052419302D0A9F7EACFB4E080
:10F79000A6959795879577956795BA95C9F7009738
:10F7A0006105710508959B01AC010A2E06945795D9
:10F7B000479537952795BA95C9F7620F731F841F30
:10F7C000951FA01D0895DC01CB01FC01F999FECF26
:10F7D00006C0F2BDE1BDF89A319600B40D924150D9
:10F7E0005040B8F70895F999FECF92BD81BDF89ABF
:10F7F000992780B50895A8E1B0E042E050E00C946C
:10F80000E57BDC01CB0103C02D910E940C7C4150B3
:10F810005040D0F70895262FF999FECF1FBA92BD18
:10F8200081BD20BD0FB6F894FA9AF99A0FBE0196E1
:10F8300008950E940B7C272F0C940C7C6F927F9272
:10F840008F929F92AF92BF92CF92DF92EF92FF92F0
:10F850000F931F93DF93CF930F92CDB7DEB75B016A
:10F860006115710521F0DB018C9311969C93482F53
:10F87000592F6A01F601E1906F018F018E2D90E002
:10F880000E94F9790097B1F7FE2DFD3229F4D601D7
:10F89000ED908D0121E007C0BE2DBB3219F4F601B9
:10F8A000E1908F0120E068010894C108D108C601E9
:10F8B00060E370E143E050E029830E94AF7D29813D
:10F8C000009711F572E0E72EF12CE00EF11EC70152
:10F8D00063E370E145E050E00E94AF7D298100972D
:10F8E00029F467E0E62EF12CE00EF11EA114B1041C
:10F8F00021F0D5011196FC92EE9220FF0FC130E06D
:10F9000020E090E88FEF12C1C60168E370E143E0A8
:10F9100050E029830E94AF7D2981009731F060E09B
:10F9200070E0CB01662477240AC0A114B10409F465
:10F93000F9C00E5F1F4FF50111830083F3C03E2D08
:10F9400030533A30A0F52260E22FF0E0AF0148706A
:10F95000507022FF07C04115510571F50894611CD4
:10F96000711C2AC04115510519F0089461087108ED
:10F970006B017C0152E0CC0CDD1CEE1CFF1C5A9587
:10F98000D1F76C0D7D1D8E1D9F1D660F771F881F83
:10F99000991F630F711D811D911D6839F9E97F075A
:10F9A000F9E98F07F9E19F0738F0246005C03E3F71
:10F9B00039F423FD3FC02860D801ED908D01BFCF01
:10F9C000353311F03531B1F5F80131913D3211F493
:10F9D000206102C03B3241F4D80111963C9111974D
:10F9E000319642E050E002C041E050E030533A30FE
:10F9F00020F08F01041B150B1DC040E050E0BCE05F
:10FA000040385B075CF4DA01AA0FBB1FAA0FBB1FCB
:10FA10004A0F5B1F440F551F430F511D3191305347
:10FA20008F013A3060F324FF03C0509541955F4F3A
:10FA3000640E751EC22EDD2421FF08C0A114B1047E
:10FA400029F001501040F501118300830E945F747A
:10FA50007B018C01F3E0CF22DD2433E0C316D10417
:10FA600021F417FB109517F91095C801B70120E094
:10FA700030E0A9010E94F373882309F44AC077FE9D
:10FA800009C04FE4C42E40E1D42E709461947108F3
:10FA9000739404C037E6C32E30E1D32E26E0822EC5
:10FAA000912C90E2A92EB12C0FC0F6012591359131
:10FAB00045915491C801B7010E941175E62EF72EA9
:10FAC000082F192F6A187B086A147B0474F7B59401
:10FAD000A7940894810891088114910429F08CEF6F
:10FAE0009FEFC80ED91EF0CFB701C801282F220FF3
:10FAF000292F221F2F3F39F020E030E0A9010E947A
:10FB0000F373882331F482E290E09093852D809303
:10FB1000842D3E2D2F2D902F812F08C030E020E026
:10FB200090E803C030E020E090EC8FE7F901AC01F1
:10FB30006F2F722F852F942F0F90CF91DF911F91F0
:10FB40000F91FF90EF90DF90CF90BF90AF909F907C
:10FB50008F907F906F900895992788270895FB01D3
:10FB6000DC014150504088F08D9181341CF08B3580
:10FB70000CF4805E659161341CF06B350CF4605EB2
:10FB8000861B611171F3990B0895881BFCCFF894C3
:02FB9000FFCFA5
:10FB9200263A202573205B414444523D252D642E94
:10FBA200252D64205345513D252D642054544C3D50
:10FBB200252D7520525353493D252D75204C514911
:10FBC2003D252D75204452503D252D642E25303281
:10FBD200645D0A00523D252D75204C3D252D752072
:10FBE200533D252D64200054696D656F7574204165
:10FBF2004444523D252D642E252D64205345513D0C
:10FC0200252D6420525353493D252D75204C5149D1
:10FC12003D252D750A002845787450777229000019
:10FC220045554936343D00253032582D00253032B5
:10FC3200580A00534E3D00413A2025642025642095
:10FC42002564200A00433A20256420256420256487
:10FC5200200A007374617475733D307825303278F0
:10FC62000A2000312E30204669726D77617265205C
:10FC72005665722E2053312D352E302032303134DC
:10FC82002D30312D323800656570726F6D006F6EE8
:10FC9200006F666600666F7263655F69646C65001B
:10FCA20064656570004F6E00613100726573657442
:10FCB200006E6F6E6500613200765F696E00310022
:10FCC2003200330034006175746F00666C757368BE
:10FCD20000414444523D252D642E252D6420534578
:10FCE200513D252D6420525353493D252D75204CFD
:10FCF20051493D252D750A00707772733D25730AAF
:10FD0200007472696D007478743D25730A0074651D
:10FD120073740043683D252D642054785077723DFA
:10FD2200252D640A004572726F72205458204C656A
:10FD32006E6774683D25640A005458543D2573204B
:10FD42000049443D0025303278002050533D25645F
:10FD52000020543D252D362E3266002054313D259B
:10FD62002D362E32660020545F4D43553D252D35EC
:10FD72002E31660020565F4D43553D252D342E32DF
:10FD820066002050303D252D6C58002050305F54C5
:10FD92003D252D372E3366002050313D252D6C58E0
:10FDA200002050315F543D252D372E3366002055FB
:10FDB200503D252D6C58002052483D252D342E31C2
:10FDC200660020565F494E3D252D352E32660020B5
:10FDD200565F41313D252D352E32660020565F415A
:10FDE200323D252D352E32660020503D252D6C6486
:10FDF200002050413D252D372E326600263A20251F
:10FE0200730A00545820706B74206C656E203D207C
:10FE120025640A0025303258006C656E3D25640A5F
:10FE2200000100ED478A3C22FFCC3B22FFCC3B1A6B
:10FE320020090D00A0046162636465666768696AEF
:10FE42006B6C6D6E6F70261400003C000A00636DCF
:10FE5200642070726F63657373000000BE046D33BB
:10FE620000000000737464696E2070726F636573C2
:10FE720073000000D404120F0000000062726F6170
:10FE820064636173742070726F6365737300000042
:10FE9200EC04463400000000536C656570207072FB
:10FEA2006F63657373000000080502100000000014
:10FEB200506572696F6469632070726F63657373F2
:10FEC2000000002005B11600000000CA04E204FE92
:10FED20004310516050000790800001D00400008E5
:10FEE20007480710000000C23BB63B181000000094
:10FEF200004576656E742074696D6572000000615C
:10FF020005CD3F000000004374696D657220707278
:10FF12006F6365737300000077050B4100000000FA
:10FF2200020306070A0B0E0F020306070A0B0E0F47
:10FF32002843292032303132204865726A756C6656
:10FF42000055747665636B6C696E672020202020F3
:10FF52002000436F6E74696B6920322E35000000F9
:10FF6200000200000000464F00000000C600C5006D
:10FF7200C400C100C200000000CE00CD00CC00C908
:10FF820000CA0000000052463233302064726976A3
:10FF92006572000000F605FD53000000006E52EC91
:10FFA200514C5496550F539F510D5007508E51F09E
:10FFB20050000101010101010101010101010101E1
:10FFC200010052696D650032061157D856616461AD
:10FFD20074612E6E756D20776179206F757420744F
:10FFE200686572653A2025640A00535852585C5A73
:0EFFF2008B5BC3590080C0E0F0F8FCFEFF6E90
:020000021000EC
:10000000756C6C6D6163006D063E5C235C295C2F32
:100010005C355C3B5C736963736C6F776D61630027
:1000200083065F5DC05C565C3F5C455C535CBA0018
:10003000080007110F1135000200DF16E1165443C6
:10004000502F495020737461636B000000AC06B9F7
:100050005F000000000208FFFFFFFF00000000013A
:04006000000000009C
:00000001FF
